:020000040800F2
:100000000002002029050008C5040008810400083A
:10001000D5040008E5040008F5040008000000000D
:10002000000000000000000000000000450400087F
:100030000505000800000000290400081505000857
:100040008901000889010008890100088901000868
:1000500089010008890100082124000821240008E2
:100060002124000821240008212400088901000817
:100070008901000889010008890100088901000838
:100080008901000889010008890100088901000828
:10009000890100088901000889010008212400085D
:1000A0008901000889010008890100088901000808
:1000B000B9250008890100088901000889010008A4
:1000C00089010008890100088901000889010008E8
:1000D0008901000889010008D11F0008D71F000806
:1000E000212400088901000889010008890100080D
:1000F00089010008890100088901000889010008B8
:100100008901000889010008BF250008890100084D
:100110008901000889010008890100088901000897
:100120008901000889010008890100088901000887
:100130008901000889010008890100088901000877
:100140008901000889010008890100088901000867
:100150008901000889010008890100088901000857
:100160008901000889010008890100088901000847
:1001700089010008890100088901000800000000C9
:10018000000000008901000800F0C4B900F004BBC1
:100190007047000070B50C46064600F061F9094B47
:1001A000094A1D682919914202D8084A914204D28D
:1001B0000C2333604FF0FF3500E0196000F058F970
:1001C000284670BD0002002000000220905E002042
:1001D0001946104600F0ECBA1946104600F0F0BA85
:1001E000132303604FF0FF307047132303604FF079
:1001F000FF307047132303604FF0FF307047022930
:100200004FF0000303608CBF002001207047000006
:10021000114B70B500241C60104B114D18682E68EE
:1002200000F09CF80F4B53F820301B68A3F1080234
:1002300096420FD026B13179092904BF0A213171C4
:10024000092103F8041C33F9021C074B2A601980AA
:10025000012070BD204670BD980200206C03002074
:10026000A0020020A80200209C020020082930B52E
:10027000037919D9082B32D842791A4B53F82250F6
:1002800000F108042DB12D68856053F822502C60D0
:1002900000E0846043F82240134C4279012303FAC2
:1002A00002F22368134319E0082B18D945790D4B46
:1002B00053F825203AB11468A2420BBF00222468EB
:1002C00043F825201460427953F822303BB9064C9C
:1002D000012303FA02F2236823EA02032360017177
:1002E00030BD00BFA80200206C03002008B50A4BF7
:1002F0001B681A79082A02D95B7983420AD900F06F
:10030000BAF818B1054B01221A6008BDBDE80840D3
:1003100000F082B808BD00BFA002002098020020B3
:1003200008B500F09DF8094B094A1B88094D1BB21E
:10033000002442F82340084A286813682146013BFC
:100340001360FFF793FF2C6000F062F89C0200201E
:10035000E8020020A0020020A40200200023C2071F
:1003600002D440080133FAE718467047134423F0DB
:10037000030310B54FF077321C1F43F8042C6207BB
:1003800042BF4FF0883243F8082CA3F108044FF025
:10039000807304E909000F4B44F80C3C002344F837
:1003A000103C032344F8143C2246022344F8183C32
:1003B000012344F81C3C42F8201D0B2342F8043D65
:1003C000013B032BFAD120466FF0020340F8443D75
:1003D00010BD00BF21030008064B0749074A1868F3
:1003E000884203D1934201D20433F8E70348C01A8C
:1003F000704700BF00000020FEE7FEE7000200207B
:10040000EFF30880704700000048704700000020AC
:1004100000F02AF801DFFEE7024A536843F08053F8
:100420005360704700ED00E0EFF3098020E9F00F22
:1004300040F804ED02490968086000F003F8000084
:10044000A0020020FFF7E4FE04480068016801C92B
:10045000B1E8F00F81F3098800470000A0020020F6
:10046000EFF3108072B6704762B6EFF310807047FA
:1004700080F310887047EFF30580C0B2704700002A
:100480000D490E4A0E4B6846904203D8984201D956
:10049000002102E009468D460121042072460242F5
:1004A00002D1EFF3088001E0EFF309802DE9F00FAE
:1004B0006B4600F06FF800BF000200200000022031
:1004C0006005002008B50249042000F0BBFB00BF16
:1004D0009CF5000808B50249062000F0B3FB00BFF8
:1004E000A8F5000808B50249072000F0ABFB00BFE3
:1004F000BBF5000808B50249082000F0A3FB00BFC7
:10050000CDF5000808B50249092000F09BFB00BFAB
:10051000E1F5000808B502490A2000F093FB00BF8E
:10052000F3F500087047704708B5FFF7FBFF6A4610
:10053000114B1249934202D243F8041BFAE7104AC6
:10054000104B11498B4204D252F8040F43F8040BAC
:10055000F8E70E4B0E4A0021934202D243F8041BE7
:10056000FAE7FFF7E0FF00F04DFB0DF00FF9BDE8F3
:10057000084000F0A1BB00BF00000020FEE7FEE73E
:10058000602201080002002094020020980200204E
:10059000905E00202DE9F04F9A46494B8FB093466C
:1005A0009A6B03925A6B04929F6ADA6A05921A6BED
:1005B000DB6B0793434B06921A68434B9A420446FF
:1005C000884602D041480DF0CBFBB8F1000F05D0B2
:1005D0003F4800250DF0C4FB2E4626E094E80E00AF
:1005E000E068D4F81C9008902069099060690A902E
:1005F00019F4007F3748A6690D930CBF04F120055C
:1006000004F124050C920B910DF0AAFB089B0093BA
:100610000BA90EC930480DF019FBCDF800903346F8
:100620000A9A09992D480DF011FB2D480DF098FB01
:1006300039462C480DF00AFB05992B480DF006FBB6
:1006400006992A480DF002FB079929480DF0FEFA99
:100650003A0403D5039927480DF0F8FA3B0603D571
:10066000049925480DF0F2FA24480DF079FB59461B
:1006700023480DF0EBFAB8F1000F1BD121480DF023
:100680006FFB314620480DF0E1FA69461F4BC91A4D
:1006900003D549421E480DF0D9FA20468268C36846
:1006A00001698C4641698E46AD46514691E8F00F8E
:1006B0004168006801BE1749052000F0C3FA00BF79
:1006C00000ED00E000000020FEE7FEE701F6000874
:1006D00017F6000846F6000861F600089EF60008C6
:1006E000DCF60008E5F60008F5F6000805F7000856
:1006F00015F7000825F7000835F7000845F700084A
:100700004AF700085CF700088DF700085801002040
:10071000B5F70008E2F7000810B568B1012815D157
:10072000174A136823F003031360136843F400733C
:1007300043F0010313601BE0114B1A6842F00E02F4
:100740001A605A6842F480725A6011E00D4A1369C7
:1007500023F0040313610024FFF782FEBFF34F8FE1
:1007600030BFFFF785FE54B1BDE8104001F0D4BAA8
:10077000044A136943F0040313610124ECE710BD3C
:100780000070004000ED00E008B5FFF769FE0020B2
:10079000BDE80840FFF7C0BF034B044A4FF4E13106
:1007A000002001F08BBB00BF04020020A91A000842
:1007B0000A460146014801F082B900BF0402002048
:1007C00010B50A460C4601230146024800F0FAFB28
:1007D000204610BDC4030020002001F097BE000099
:1007E000034B1968024611B9084601F06FBE704705
:1007F000B403002010B5094A13685BB19C68816896
:100800008C4202D21A461B68F7E703D15C68416844
:100810008C42F7D90360106010BD00BFC0030020F8
:10082000F0B51F4E1F4D33681F4C013333601F4B13
:1008300000201A6818602B68226019460746B646E1
:1008400041B1DEF800C08E68664503D80F4601202E
:100850000968F5E700B1296007B9F0BD00213960EA
:10086000E2B133B151685868814294BF11461946CC
:1008700000E01146084612681B680AB903600BE0E5
:100880000BB9026008E055685E68B54294BF154632
:100890001D4605602846EEE72160F0BD2360F0BDEF
:1008A000B8030020C0030020BC030020B0030020D8
:1008B0002DE9F0412E4F2F4C01233B6023683BB9BB
:1008C000FFF7AEFFFFF788FF0130FBD0002502E005
:1008D000FFF782FF05464FF00008236823B9FFF7B2
:1008E0007BFF854214D91AE05E68FFF775FF8542E9
:1008F00008D923685E68FFF76FFFA8422CD3B04287
:10090000F7D329E08642F4D9361A132EE7D8F0E758
:10091000236843B9FFF760FF854206460BD9FFF70E
:100920007FFF0025D9E75E68FFF756FF063E1430CB
:100930008642D2D309E010F1140F04D3FFF74CFF25
:100940008642FBD9EBE74FF0FF3600233B60304691
:10095000BDE8F041FFF744BF23681A682260C3F87E
:100960000480C3F80880DA6818699047B5E700BFCB
:10097000B4030020BC030020144B1A6882420AD141
:1009800012681A6012B15068063801E04FF0FF306B
:10099000FFF726BF13461A6822B19042FAD10268C7
:1009A0001A6070470A4A13681BB1984203D01A466E
:1009B000F9E7084A05E00368136070479842FAD0E7
:1009C0001A461368002BF9D1704700BFBC03002002
:1009D000B0030020C003002008B500231846054AD4
:1009E000054901F0A5FD4FF0FF30BDE80840FFF7D5
:1009F000F7BE00BFB108000840420F0070B5084EB6
:100A0000FFF7EAFE34680546FFF7E6FE8542F7D8B1
:100A100000222346141843F100052046294670BDE4
:100A2000B8030020F8B504460D46FFF7D5FE0023B5
:100A300085420646236010D3A5F10A0383420CD2F7
:100A40000A35FFF7C9FE8542FBD3FFF7C5FE854295
:100A5000FBD8E368206998473EE0FFF701FD636833
:100A60000746002B34D1A368002B31D11B4B6560A6
:100A70001A681B68B54238BF0132A260A2689A4268
:100A800003D92046FFF7B6FE1EE0B54202D9144B4B
:100A900019460EE0134A136823B159688D4201D3F9
:100AA0001A46F8E7236014600EE05068854203D3CD
:100AB00013461A68002AF8D122601C600B689C4219
:100AC00002D1A81FFFF78CFE3846FFF7D1FC03E0E8
:100AD0002046FFF751FFC9E70020F8BDB80300200A
:100AE000BC030020B003002038B50446FFF7B8FC73
:100AF0006368054633B9A36823B92846BDE8384082
:100B0000FFF7B6BC2046FFF737FFF6E7C36870B5BE
:100B100004460D46C3B1FFF7E7FF092D0CD8FFF7D8
:100B20005BFE0646FFF758FE801B8542FAD8E36855
:100B30002069BDE870401847FFF74EFE291820468F
:100B4000BDE87040FFF76EBF70BD00002DE9F047B3
:100B500004460E4690461AB9BDE8F047FFF7D6BFE7
:100B6000FFF77EFC63680746E3B9A368D3B9DFF8F3
:100B70003CA0FFF731FEDAF800508146FFF72CFE6B
:100B80008145F6D8304408EB0502864288BF013221
:100B90006060A2602046FFF72DFE3846BDE8F047B2
:100BA000FFF766BC2046FFF7E7FEE0E7B80300204A
:100BB00030B587B0002302930D4D0E4C4FF4E13356
:100BC00003930D4B049302A94FF400632846059349
:100BD00000F04CFA2946204600F0E4FB0094074B55
:100BE000074802224FF4806100F064FC07B030BD7A
:100BF000C4030020040C002004040020F5F70008C2
:100C0000140C002008B50121094801F031FB012135
:100C1000084801F02DFB0121074801F029FB0121C3
:100C2000064801F025FBBDE8084000F021B900BFEF
:100C30000D0C02400C0C02400E0C02400F0C024046
:100C40007047000008B50F4B1A680C469AB901228C
:100C500003281A6003D171460B480CF0F7FF2146B8
:100C60000A480CF0F3FF00F0B7FF09480CF0EEFF64
:100C700008480CF0EBFFFFF7F3FBFFF7E1FFFFF78E
:100C800083FD00BF1410002012F8000816F80008B9
:100C90003EF8000832F8000808B501F02FFD0348BF
:100CA0000CF0D4FF01F012FD002008BD40F8000850
:100CB00008B500F073FFFCE71FB5FFF7D1FB0E4B43
:100CC0000E481B68029300240D4B00930F220C2347
:100CD0004FF48071019400F055F80A4B0A481B68E4
:100CE00002930A4B009307220C234FF4C061019436
:100CF00000F048F8FFF78CFB1802002018100020C5
:100D0000B10C00081C02002018110020990C0008EA
:100D100008B5FFF7A5FB094B1B681A79082A07D904
:100D20005A79074B53F8221011B1096843F8221081
:100D3000FFF79EFBBDE80840FFF76EBBA002002056
:100D4000A802002038B50B79082B03D908490320E5
:100D5000FFF778FF4C7901F1080203682BB113F813
:100D6000035CAC4201D31846F7E78B60026038BDE4
:100D700000F80008031F53F8042F9A42FBD0181AFA
:100D8000704700000F2A2DE9F74F05468B46914624
:100D90009A462AD810F003031BBFC3F10403ED18D1
:100DA0000B46CB1A303B23F003031AF0080F05EB78
:100DB000030405D02A46A24203D212600432FAE7A5
:100DC0002D600193FFF74CFB2749019B80460122D0
:100DD00051F8227016B25FB10132212AF8D1404693
:100DE000FFF746FB6FF08A003BE06FF0150038E03C
:100DF0001D490C9841F822402A46E6800D99FFF7DC
:100E0000B5FA0E9B194AA3624FF0FF33E3611368F2
:100E1000206001331AF0010F6562C4F82CB084F829
:100E200005902771A760E76027616761A761276266
:100E3000136004D001212046FFF718FA0DE00A21C3
:100E40002046FFF713FA1AF0040F06D14046FFF7C9
:100E50000FFB4846FFF74AFA02E04046FFF708FB5F
:100E6000304603B0BDE8F08FE8020020A402002065
:100E700008B501F0B5FE00F04FFFBDE8084000F0F6
:100E800084BE0221436818470020704710B5846B68
:100E900061B1944202D94FF0FF3010BD002383634B
:100EA00022461C3001F0EAFB8442F4D1204610BDFA
:100EB000022970B5144609D1052B0BD900F1100198
:100EC000062220460CF0BCFC062070BDBDE8704038
:100ED00000F006BE6FF0150070BD0000436B10B54A
:100EE0000446032B1AD8DFE803F0021102021C307B
:100EF00001F0D9FB10B9236B013305E000236362D5
:100F000084F82C30A3626363236310BD036B013349
:100F10000363BDE81040024800F0C6BD10BD00BF2D
:100F2000040200202DE9F74F1346154606460C46ED
:100F30000A464FF0000913F1FF3303D3516808321A
:100F40008944F8E706F13C0B012102AF584601F055
:100F500017FC7E2307F8023D01223946F06801F0B4
:100F600013F80834F5B154F8088C54F8043C08EB35
:100F7000030AD04514D018F8013BF0688DF807300B
:100F80007D2B05D07E2B06D001220DF1070104E058
:100F900002220A4901E00A49022200F0F5FFE8E7CF
:100FA000013DDEE701223946F06800F0EDFF5846CA
:100FB00001F016FC484603B0BDE8F08FA6F8000823
:100FC000A4F800082DE9F34102AD1F467E23044634
:100FD0000E46904605F8053DFFF74DFA28B9012168
:100FE00004F13C0001F0CCFB04E001222946E0685A
:100FF00000F0CAFF01222946E06800F0C5FF5FB19A
:101000007D2387F02007022201A9E0688DF80430D3
:101010008DF8057000F0B8FFB044464513D016F8BF
:10102000013BE0688DF804307D2B04D07E2B05D089
:10103000012201A904E002220A4901E00A49022230
:1010400000F0A2FFE9E701222946E06800F09CFFDA
:10105000FFF711FA18B904F13C0001F0C1FB02B02E
:10106000BDE8F081A6F80008A4F80008F7B50D4621
:10107000244B0360EA680B68C3600023044680F8D1
:101080002C3003634363836389681AB1504232EAA8
:10109000000003D01C490320FFF7D4FD6362E36323
:1010A000A362E161226200F00FFE02AE04F11007BC
:1010B00046F8040D0422314638460CF0C1FB00F01E
:1010C00003FE31460190022204F114000CF0B8FB3B
:1010D000237C0E4A03F00203237495E803002346A1
:1010E00000F0ECFE02A97E2301F8053DE068012234
:1010F00000F04AFF0223062239462046FFF762FF2E
:1011000003B0F0BD8CF8000800F8000811110008C9
:1011100090F82C20012A10B5044609D002D3022AE7
:1011200032D010BD7E2949D100234363036342E0DE
:101130007D2901D102233FE07E2921D1036B002BC1
:101140003CD0416B022906D003290AD091B98363B0
:10115000436898470EE00323062200F11001FFF7D1
:1011600031FF226B062A05D104F1160104F11C009F
:1011700001F084FA002384F82C306363236310BDEC
:10118000BDE81040FFF7AABE232912D005D82129B7
:101190000DD022290FD142630DE05D2903D05E29D5
:1011A00009D17E2100E07D21FFF798FE03E00123B5
:1011B00000E003236363012384F82C3010BD00009A
:1011C000F8B585682B685C6800231A4619462846DE
:1011D000A047061E69DD002319461846324600F076
:1011E0003DFB2B6804465F6828B90346014632463A
:1011F0002846B84752E08168002332462846B8475F
:10120000011E4EDD8E4202DD204600F0AFFB0022C3
:101210000E21204600F03CFB0646002841D087689E
:10122000BB895BBA48F2DD629BB293420CBF0223DA
:1012300000230021237414224FF0FF33084600F0EE
:101240000DFB054660B3836806221A705A700022AF
:101250005A719A711A7180685A800278062A03D1ED
:10126000B91D08300CF0ECFAA8684278062A05D1BE
:1012700003780833394618440CF0E2FA0C4B1A880C
:10128000AB6831465A80204600F09AF900236B6023
:1012900023465A680AB11346FBE75D602046F8BD55
:1012A00034460021204600F0CBFB0020F8BD00BFF3
:1012B0009C0200202DE9F041876886B00D46002988
:1012C00067D091F910304E68591C02D06FF04C0075
:1012D00064E04EB196F910104FF6FF7348F2DD62EC
:1012E000022908BF13465BBAAC68ADF81430227807
:1012F000062A05D104F1080102A80CF0A1FA08E0C1
:101300003B680DF10E02D3F8108002210623384607
:10131000C04723791A0612D45B0616D5002E3BD09F
:1013200096F91030022B0AD1B16833238DF80830BA
:101330008DF80930042224310DF10A000CE0062258
:10134000FF2102A80CF07AFB08E06278062ABDD1E2
:1013500021780831214402A80CF072FA01A928462C
:1013600000F002F9064660B18168019A02AB0B6099
:101370000E234B603B6838461B6898473546044649
:1013800001E06FF068042846002100F059FB204678
:1013900004E06FF0150001E06FF0850006B0BDE8D5
:1013A000F0810000034B0360034B43608160002029
:1013B000704700BFB5120008C1110008F0B5254EF6
:1013C00084683388838195B00821054604A801F01C
:1013D000F3FB3088204B6360A56000B200F082F818
:1013E000236820469B68984740F2032741F2342641
:1013F000684601F0DEFBBDF80230BB4213D0B3F506
:10140000017F08D240F202229342F1D12B68019968
:1014100028469847EAE70AD0B342E9D12368204634
:10142000DB689847E2E7236801995E6902E0236878
:1014300001991E690B894A6809782046B04740F235
:101440000523039002A96846ADF80A3001F080FB3D
:10145000CCE700BF9C0200205D14000813B5806833
:1014600079B941F234230190B0F90C10ADF8023093
:10147000684601F0F9FA002816DC0C480CF070FC04
:1014800012E0022910D143689847044660B1034630
:10149000074990F9100040F2012204F00FF80146CC
:1014A00010B9204600F0CCFA02B010BDA8F8000830
:1014B0000000FFFF30B585B0089C6CB1A5685DB138
:1014C0000293074B009301940823FFF75BFC00286D
:1014D000D8BF6FF0150001E06FF0120005B030BD0D
:1014E000BD13000808B50E4BB3F90020904211D08F
:1014F000B3F90210002A0CBF1A460022884209D014
:1015000021B90233002A08BF1A4600E022B1108038
:1015100002F02AF9002008BD6FF00B0008BD00BFE3
:1015200018170020074AB2F90030014613B10380B2
:10153000012000E01846B2F9023013B121F8103052
:101540000130704718170020064BB3F90020824283
:1015500005D0B3F902301B1A584258417047012098
:10156000704700BF1817002070B504460E4619B921
:1015700012490320FFF766FB10B90020306070BDF0
:1015800001460025496801350029FBD16FF00103B0
:10159000EA00204600F062F90028EED08368002BB4
:1015A000E6D00833A26843F8082CE268646843F880
:1015B000042C0833002CF5D1356070BD00F800080C
:1015C00010B504468C42084601D1646808E0234601
:1015D0005A682AB1904201D01346F9E742685A602E
:1015E0000021416000F02CFA204610BD70B555680E
:1015F00004460846EDB129464B680BB11946FBE796
:101600001CB91A490320FFF71DFB0028F9D0002A56
:10161000F7D043685360844206D023465E6826B103
:10162000B04219D03346F9E7144653684B60556011
:1016300015E0002CE5D00029E3D0002AE1D04B686A
:1016400053608C4206D02346596841B1884205D088
:101650000B46F9E7144602E05A60E6E75A600021BB
:10166000416000F0EDF9204670BD00BF00F80008B1
:1016700070B503461A4A072B88BF033310688CBF26
:1016800023F003030823002140B34468A34202D996
:1016900001460068F8E7E41A072C0344114E05D808
:1016A000046809B9146011E00C600FE0C6F1080588
:1016B0001D44B5F5C05F02D90021116003E009B9EE
:1016C000136000E00B60026883E81400064A9B1B6D
:1016D00011889BB2994201D2138070BD70BD00BFCA
:1016E00020170020241700201C170020012101488A
:1016F00001F046B8242F0020204A38B5831AB3F5EC
:10170000C05F39D21E4D2C68002324B1844202D21E
:1017100023462468F9E707298ABF0331082121F00D
:1017200003010460141AC1F5C0522244072A98BF6D
:10173000891841600BB9286011E05A6818601A4492
:10174000821A072A0BD818B90E490320FFF77AFA34
:10175000026841681A60C21A0A445A60184603684F
:1017600053B1426802449A1A072A05D81A680260DF
:101770001A1A5B681344436038BD00BF2417002069
:101780002017002000F800082DE9F84381461420B6
:101790000F4616469846FFF76BFF0446D8B15EB178
:1017A0003046FFF765FF054638B920461421FFF79C
:1017B000A3FF2846BDE8F88335460123C4F804900A
:1017C000A560E66084F81080236027B13246394670
:1017D00028460CF035F82046BDE8F883F8B50F4DE3
:1017E00004460026CCB1631BB3F5C05F03D30C499C
:1017F0000320FFF727FA94E88800012B09D1E1685C
:10180000A0682660FFF778FF14212046FFF774FFD9
:1018100001E0013B23603C46E4E7F8BD24170020CB
:1018200000F8000808B5FFF761FF094A094B13608B
:10183000182100221A705A709A70DA701A71597150
:101840009A71DA710448BDE8084000F0C9BF00BFD2
:101850002017002024170020242F0020B2F5C05F9D
:10186000F8B505460E4614461F460DD8FFF73EFF55
:1018700022463B4631462846FFF786FF044603488A
:1018800000F0AEFF2046F8BD0020F8BD242F002058
:1018900007292DE9F84388BFCF1C0D468CBF27F0E0
:1018A0000307082704469146FFF720FF2DB124B116
:1018B000E3689D4201D8A3682BB92B4800F090FF44
:1018C0000020BDE8F8831420FFF7D2FE064600286A
:1018D000F3D0E3689D422ED0AF4202D85A1B072AAC
:1018E00029D82846FFF7C4FE074610B91421304610
:1018F0000BE0E068401BFFF7BBFE804640B91421B7
:101900003046FFF7F9FE29463846FFF7F5FED4E7E3
:101910002A46A16838460BF093FFE268A168521B83
:10192000294440460BF08CFFE168A068FFF7E4FE15
:10193000C4F8088005E0A7689D4214BF7B19002306
:10194000A360E36808485B1BE3606368736001237E
:10195000B760F56086F810903360666000F040FF75
:101960003046BDE8F88300BF242F0020072970B55A
:1019700088BFCE1C04468CBF26F0030608260D4601
:10198000FFF7B4FE1CB922490320FFF75BF9E368B7
:10199000A06813B90028F6D106E00028F3D01D4A4C
:1019A000821AB2F5C05FEED29D422CD02DB930B173
:1019B0001946FFF7A1FEA56024E09D4202D8991BBD
:1019C000072917D82846FFF753FE064620B91248C4
:1019D00000F006FF0C2070BDA16829B1E268AA42A0
:1019E00028BF2A460BF02CFFE168A068FFF784FEB1
:1019F000A66007E0033323F003039E4202D2304483
:101A0000FFF77AFEE560044800F0EAFE002070BDB2
:101A100000F8000824170020242F002038B50446C1
:101A20000D46FFF763FE24B123682B4423606468EE
:101A3000F9E70248BDE8384000F0D2BE242F00206C
:101A400010B50446FFF752FE2046FFF7C7FE0248D6
:101A5000BDE8104000F0C4BE242F002038B5044675
:101A6000FFF744FE0CB1E26822B90E4800F0B8FE60
:101A7000002038BD2368012B0FD994F91030A168DC
:101A80006068FFF781FE054610B12368013B2360C3
:101A9000044800F0A5FE284638BD024800F0A0FE2C
:101AA000204638BD242F002038B50446043000F00D
:101AB000FAFD0546204600F093FE284638BDF8B5ED
:101AC00004460E461746051D3A463146284600F0A4
:101AD000D5FD20B90121204600F052FEF4E7F8BD03
:101AE000082973B50C46154621D003D8081F0128D4
:101AF0000CD905E024293FD0252904D011290FD085
:101B00006FF0850039E00220108036E0022B03D010
:101B10001B490320FFF796F806222A8018462CE07E
:101B2000012BF5D940F2DC531380022025E0072B6E
:101B30001FD903686A461E6902210623B0479DF833
:101B4000003083F002032B709DF801306B709DF81C
:101B50000230AB70FF23EB70FE232B719DF8033036
:101B60006B719DF80430AB719DF80530EB71204628
:101B700003E06FF08A0000E0012002B070BD00BFFA
:101B800000F800086FF08500704708B5002000F0ED
:101B900049FA0120BDE8084000F044BAF8B50D4B01
:101BA0001E68C6F307221D4622B9F4B2003418BFDE
:101BB000012400E00224FEF753FC2B689E420746F6
:101BC00002D12046FEF7A8FD3846BDE8F840FEF7F2
:101BD0004FBC00BF200200202DE9F04F2C4B2D4AB6
:101BE0001B882D492D482E4EDFF8CCB08BB00DF15F
:101BF000280906F1800A29F8043D0CF027F8FEF7C1
:101C0000EBFB0546FEF700FC0446FEF7F9FB2A460F
:101C1000009023464FF4007122480CF017F825EA93
:101C2000E5754FF4007856F8044B14B32779E26A4F
:101C30005BF82730606A079390440692FFF79AF8A2
:101C4000069AB4F90610079B101A22680592626A78
:101C500004920390E26A029262790192082FD4BF43
:101C60004F4609F1010700970544A26A0E480BF0A0
:101C7000EDFFB245D7D10D4B02958DE808010C4A16
:101C80000C4819460BF0E2FF0BB0BDE8F08F00BF27
:101C9000CEF80008FCF8000802F9000807F900086F
:101CA000EC0200204FF9000899F90008D5F9000866
:101CB000D7F90008DBF90008D0F800080146014810
:101CC00000F0B2BC282F0020124BF0B593E834008E
:101CD000D8681E691C6084EA050122F000424A406F
:101CE00082EA420280EA500050405969D86040F3CD
:101CF000000782EA802239404A4004EB12249A60AD
:101D00009A693E40604044F30004754014405D60B1
:101D10006040F0BD282F002038B5FEF7A1FB1B4C1A
:101D20000023E360054600F037F84FF41443A36046
:101D3000A268164B12F00C0FFAD1154A40F2057149
:101D4000116081221A601A6842F480321A601A689F
:101D500012F4003F0D4AFAD00E4B5360136843F063
:101D6000807313601168094B8901FBD59A6842F0B2
:101D700002029A609A6802F00C02082AFAD100F076
:101D800017F82846BDE83840FEF772BB003802401D
:101D9000003C0240042A4007044B1A6842F001024A
:101DA0001A601A689207FCD5704700BF00380240DD
:101DB000044B9A6812F00C0F1EBF1A6822F0010241
:101DC0001A60704700380240034B044A00280CBFD9
:101DD00010461846704700BF00BD010580DE800236
:101DE00004281CD8DFE800F003080D1217000D4B83
:101DF0001A6C1143196412E00A4A536C1943516476
:101E00000DE0084A136B1943116308E0054A536B50
:101E10001943516303E0034A936B19439163BFF382
:101E20004F8F704700380240042821D8DFE800F0C7
:101E300003090F151B000F4A136C23EA01011164FB
:101E400070470C4A536C23EA010151647047094AF8
:101E5000136B23EA010111637047064A536B23EAAF
:101E6000010151637047034A936B23EA01019163B7
:101E7000704700BF0038024038B514230C4A434372
:101E8000D4582568AA0608D50A4B616803EBC0023E
:101E9000C9B253F83030506898472B0748BF636881
:101EA000054B1B681BB1BDE83840FEF731BF38BD9C
:101EB00054FA0008442F00209802002001282DE940
:101EC000F04780460D46174603D92B490320FEF7FD
:101ED000B9FEDFF8B090294A142404FB009442F8BC
:101EE0003070E66802EBC00201215360304600F01A
:101EF000BFF9304600F080FA3046617C00F054FAB9
:101F00004E464FB1D4F808900021484600F0B0F991
:101F1000217C484600F048FA142303FB08F806EB3E
:101F2000080999F812A0D9F804105046FFF758FF95
:101F300056F808400023E360504623616361FFF7D1
:101F400043FFB0FBF5F080B2A06077B199F8133091
:101F500001215AB203F01F0301FA03F352090849A1
:101F600041F8223042F22C0301E042F20803E36020
:101F70000020BDE8F08700BF00F80008442F0020D3
:101F800000E100E054FA0008012838B505D80E4CED
:101F900014230A4403FB004309E00C490320FEF725
:101FA00051FE25682D06FCD511F8015B65608A425B
:101FB00001D01C68F5E714235843034B1A581368E3
:101FC0005B06FCD538BD00BF54FA000800F80008D5
:101FD0000020FFF751BF0120FFF74EBFF8B5104CAE
:101FE00004EB401401216768384600F041F9A66807
:101FF0000021304600F03CF9E5680121284600F058
:1020000037F9247D3846214600F0CEF92146304686
:1020100000F0CAF921462846BDE8F84000F0C4B9EE
:1020200088FA000801282DE9F041044603D9104937
:102030000320FEF707FE0F4BDFF83C80002543F836
:1020400020506401FFF7CAFF08EB04031E7F9F695D
:1020500030463946FFF7C4FE58F8043039461D6053
:102060003046DD615D60BDE8F041FFF7DDBE00BFD9
:1020700000F80008542F002088FA0008012870B5E5
:102080000C4621D84A1C22D021F0FF0313F5807F93
:1020900011D114F0FF041AD10E4B03EB40152E6939
:1020A000731C14D00121304600F0E2F8297D30463F
:1020B00000F07AF906E00121204600F0D9F8204628
:1020C00000F09AF9002070BD4FF0FF3070BD6FF046
:1020D000010070BD88FA0008042B2DE9F84304467E
:1020E0000E461546984603D917490320FEF7AAFD68
:1020F0001648DFF860906701012100EB840000F0D2
:102100003FFB09EB07031C7F99692046FFF768FE38
:102110000F4B59F8071004EB84041C4416F5807F1C
:1021200014F8082045EAC20545F004050D6015BF06
:102130000B684B6843F4407343F0040314BF0B6017
:102140004B600020BDE8F88300F80008542F002001
:102150007CFA000888FA00080B4A430110B50446CF
:10216000D018D3588169007F00221A605A6822F083
:1021700004025A60FFF758FE044800EB8400BDE8F3
:10218000104000F02DBB00BF88FA0008542F00203B
:102190002DE9F843089E099F884691461D4623B9BC
:1021A0001EB931490320FEF74DFD304B400118F5B3
:1021B000807F1C58236843F04003236005D0B8F1AA
:1021C000FF3F02D0404600F020F9A6B92F44AF42AD
:1021D00006D0A3689E07FCD515F8013B2373F6E7EC
:1021E000A3689807FCD5A3681906FCD4A368DA078E
:1021F00020D5E368FAE70DB1002319E030463744F3
:10220000B84217D0A3689B07FCD52573A368DE07E7
:10221000FCD5237B00F8013BF2E7A2689007FCD5D0
:10222000EA5C2273A268D107FCD5227BF254013309
:10223000BB42F2D1A3689A07FCD5A3681B06FCD465
:10224000B9F1000F0ED1B8F1FF3F0BD0236818F59C
:10225000807F23F04003236004D04046BDE8F8436C
:1022600000F0CAB8BDE8F88300F8000888FA000852
:10227000F8B50D460126C0F3832120F00F0400F0CD
:102280000F0706FA01F10220FFF7AAFD07FA06F090
:102290000323216883406FEA030C01EA0C012160EB
:1022A000216805F0030E0EFA00FE4EEA01012160DE
:1022B000E2680CEA0202E260E168C5F38102824052
:1022C0000A43E2606268BE4022EA0606666062680F
:1022D000C5F30015BD4015436560A2681343A360B4
:1022E0000020F8BD2DE9F04100F00F0415462B4AFF
:1022F00042F8343002EBC402069B5360064688461F
:10230000C0F383274FF480410120FFF769FD414668
:102310003046FFF7ADFF042C214B03DCA11D012249
:102320008A4003E0092C03DC4FF400021A6002E04B
:102330004FF480725A601B4B0120996800FA04F236
:10234000D24311409960996805EA000E0EFA04FE26
:102350004EEA01019960D9680A40DA60C540DA683E
:10236000A54004F00C0404F1804404F59C341543AA
:10237000DD6006F00302A56892000F21914025EA76
:102380000101A160A1689740B0400F43A760586168
:102390001A68104318600020BDE8F0815C2F00200F
:1023A00000E100E0003C014020F00F0300F00F02CC
:1023B000F0B51E6857000325BD4026EA05051D60DF
:1023C0001D680224072A04FA07F444EA050494BFAE
:1023D000002201221C6003EB820300F007001C6A4C
:1023E00080000F22824024EA02021A621A6A8140A7
:1023F00041EA02001862F0BD20F00F02012300F054
:102400000F0003FA00F09061704720F00F0200F017
:102410000F001030012303FA00F0906170470000B4
:10242000104B2DE9F0415E691A680F4F16400024E9
:102430004FF001081D4608FA04F31E4206D06B61F6
:1024400007EBC40357F83420586890470134102C28
:10245000F1D1064B1B681BB1BDE8F041FEF758BC3B
:10246000BDE8F081003C01405C2F00209802002074
:102470002DE9F843124ADFF8508003010746D5588A
:102480002E69EB6800241E4008EBC0090223A3401C
:102490001E4209D0EA68D9F8040022EA0303EB607F
:1024A000214658F8373098470134042CEED1054BBB
:1024B0001B681BB1BDE8F843FEF72ABCBDE8F883F2
:1024C000C8FA000898020020DC2F0020032910B56C
:1024D00016D80D4B00011C181B586068024001F112
:1024E0000C0003EB800042601869022202FA01F13D
:1024F00020EA01021A61DA681143D960002010BD98
:102500004FF0FF3010BD00BFC8FA00080001024BB9
:102510001B58586A704700BFC8FA0008034B0001F7
:102520001A58136843F0010313607047C8FA000893
:1025300001282DE9F8430546884630D81A4E1B4934
:102540000401371941F8302097F80C9001EBC001D5
:1025500048464B60B968FFF743FC36597B68002456
:10256000346048467460F362FFF72EFC104B7A7BB0
:1025700013F809305843B0FBF8F3013BB36251B292
:10258000012302F01F02736149099340094A28465A
:1025900042F82130FFF7C2FF2046BDE8F8834FF034
:1025A000FF30BDE8F88300BFC8FA0008DC2F002028
:1025B000E8FA000800E100E00020FFF759BF012021
:1025C000FFF756BF30B5036845688468C168056089
:1025D00085EA040223F00043534083EA430381EA7F
:1025E000510183EA010242F3000583EA8223C260BB
:1025F0000169426929402A404C405340446083604D
:1026000030BD036823F0004363B9436853B983685E
:1026100043B9C36833B9542149224E234FF0590CB2
:1026200080E80E107047000038B5036943604369C5
:102630008360836901600446C3600F4801256B1EF7
:1026400003F0030305F0030254F8233054F822107A
:1026500083EA937300FB035301354B40082D44F884
:102660002230ECD12046FFF7CCFF2046FFF7AAFF2F
:10267000013DFAD138BD00BF6589076C70B51346BE
:102680007BB18568C468A5420BD084680668651C68
:1026900085604568013D2C40013B345D01F8014BEC
:1026A000EEE7D01A70BDC368426830B584681B1B62
:1026B000934208D0C3680468013A5D1C1340C560AA
:1026C000E154002030BD4FF0FF3030BD00B508218F
:1026D000A1B0074800F070FA06480BF041FB06482D
:1026E0000BF03EFB80226946002005F0D3FE00BFC0
:1026F000EC2F0020EAFA000811FB000808B50020C2
:10270000FFF7DCFAFEF768F9FFF78CF803F03EFA02
:1027100000F06CFC05F050FA00F008F8FEF748FAFB
:1027200001F01EFABDE8084005F0E6BA13B50E4CFC
:102730000E490F4808F0EEF80D49204603F050F816
:10274000002806DA0B48002102B0BDE810400BF06B
:102750007DBA0094084B094802224FF48061FEF7CD
:10276000A9FE02B010BD00BF6834002030FB000895
:102770002C34002048FB000882FB00082C3000208D
:1027800070B505460C46FDF76BFE2B6806462BB967
:102790004FF0FF332B60FDF76BFE18E0CCB10F4B11
:1027A0001C6802212046FDF761FD2B68013305D12D
:1027B00004F108032B600023A36003E021462846B0
:1027C000FEF7C0FA3046FDF753FEFDF725FE012067
:1027D00070BDFDF74DFE204670BD00BFA002002079
:1027E00070B50446FDF73CFE256806461DB16B1C1E
:1027F00005D100232360BDE87040FDF739BE2846AF
:102800000A2150F808392360FDF730FD236813B919
:102810004FF0FF33236015F8034C3046FDF728FED8
:102820002046BDE87040FDF761BD0000F8B50546E3
:102830000E46FDF715FE364B364A1B881BB207467F
:1028400052F82320D2F820E0BEF1000F1AD05469CC
:102850009369A34216D9631C5361D3691C4046B9DE
:10286000136933B9631C04D13846FDF701FE2046D5
:10287000F8BD002C0ADB0EEBC40393E8030085E8E7
:10288000030004E04FF0FF34002EE9D0D560166954
:1028900076B333681361002C0CDB95695169D369F9
:1028A000691A8B42A9BF691C4FF0FF351D40916129
:1028B0000EEBC505736893E8030085E8030016F87E
:1028C000043C052B09D0002373600A21A6F10800FF
:1028D000FDF7CCFC16F8034C00E00F243846FDF75A
:1028E000C7FD0E2C02D82046FDF700FD0120F8BDE3
:1028F000002C09DA10460321FDF7B8FC3846FDF735
:10290000B7FDFDF789FDF1E73846FDF7B1FDEDE7CD
:102910009C020020E802002010B583694469C26966
:102920001C1BA24201DA002010BD5C1C1340846114
:10293000F9D4026A03C902EBC30383E80300012050
:1029400010BD00002DE9F8431E46264B53F82150D8
:10295000254B1B880380074691462DB93046FDF76D
:1029600087FD4FF0FF3439E02B79032B28D01F4B24
:1029700001462846D3F80080FFF7CEFF044638B161
:102980003046FDF775FD98F80430052B25D122E07F
:10299000B9F1000F03D13046FDF76AFD1EE098F84B
:1029A0000430C8F80C70052B0CBF052104214046EB
:1029B000FDF75CFC414605F11000FEF7C3F907E0A6
:1029C00003C8EB6883E803000A212846FDF74EFCA4
:1029D0003046FDF74DFDFDF71FFD01242046BDE803
:1029E000F88300BFE80200209C020020A002002023
:1029F00038B50446FDF734FD074B1B882380074B91
:102A0000214605461868FFF787FF04462846FDF76C
:102A10002FFD204638BD00BF9C020020A0020020F0
:102A200008B50F4B53F82130B3B1212202801A7937
:102A3000032A0BD103C8DA6882E8030018460A218A
:102A4000FDF714FC074B0120186008BD014618462D
:102A5000BDE80840FFF760BF4FF0FF3008BD00BF82
:102A6000E80200209802002070B504460D46FDF7EC
:102A700002FD28B129462046BDE87040FFF7D0BFCF
:102A8000094B1B881BB29D4204D12046BDE8704013
:102A9000FFF7AEBFFDF7E4FC2946034601222046BE
:102AA000BDE87040FFF74EBF9C02002070B50446A1
:102AB0000D46FDF7E0FC064628B129462046BDE854
:102AC0007040FFF7ADBF0A4B1B881BB29D4204D17B
:102AD0002046BDE87040FFF78BBFFDF7C1FC3246D2
:102AE000034629462046BDE87040FFF72BBF00BFD4
:102AF0009C0200202DE9F041124F3B881BB293420B
:102B000006460C46154603D10F490320FEF79AF8F6
:102B1000FDF7A6FC3A880D4B12B2804653F822709E
:102B200005213846FDF7A2FB96E80300FC6043460A
:102B300084E80300012229462046BDE8F041FFF762
:102B400001BF00BF9C02002000F80008E80200203E
:102B500070B504460D46FDF783FCB4F90020114B17
:102B600053F8224006461CB90F490320FEF76AF8C5
:102B70002379052B04D0FDF77BFC4FF0FF3070BDAF
:102B800095E80300E36883E803000A212046FDF787
:102B90006DFB64793046FDF76BFC2046FDF7A6FB24
:102BA000012070BDE802002000F800080021FFF7B6
:102BB0003DBE0121FFF73ABE08B5074B4A1E1B6810
:102BC0001140186203D005490320FEF73BF8596114
:102BD0009961DA6108BD00BFA002002000F800087A
:102BE0000F4BD3F8882042F47002C3F888200D4AB6
:102BF0009A60102283F822200021DA7701F16040E8
:102C000000F561400131522980F80023F6D11A699C
:102C100042F010021A615A6942F400725A61704718
:102C200000ED00E00000000810B508220949044644
:102C30000AF0D4FD48B12378FF2B08D1607800F06A
:102C40000F00831E5842584110BD012010BD0020C6
:102C500010BD00BFD5FD00080021FEF7F1BE38B55C
:102C6000CBB2002114460246084602F0C5FD0546D7
:102C700018B92046FFF7F0FF0FE094F91030013348
:102C80000AD1A36882681B7903F03F0321462046DE
:102C90001371FEF795FC04466C60284638BD0000B1
:102CA00038B58B68588005460C4600F075FC18B99D
:102CB00013490320FDF7C6FF636800221BB1D968E2
:102CC0005B680A44FAE7B0F89031934204D2204698
:102CD000BDE83840FFF7C0BFB0F88E31DB0708D53C
:102CE000234640F202220749012002F0E7FB30B9F7
:102CF000EDE72146284602F01AFC0028E7DD38BD42
:102D000000F800080000FFFF2DE9F0478C68064638
:102D10000F46154600231AB1D16852680B44FAE7F2
:102D20005BBAA380A379FF2B0AD12B7C023BDBB2D9
:102D3000022B03D8214AD35CFF2B00D13B23A37184
:102D4000E37943B90EB9402304E0304600F024FC97
:102D500090F89231E37104F10808102218494046B6
:102D60000AF03CFD8246D0B904F118091549102239
:102D700048460AF033FD014630B9102240460AF0B9
:102D80005DFE0123E3750AE049465246304600F0F5
:102D90001DFE014618B1102240460AF051FD394689
:102DA000284602F0C7FD002804DA831C08BF002073
:102DB000BDE8F0870020BDE8F08700BF91FB000868
:102DC00025FE000835FE00082DE9F04F89B090F986
:102DD0001030013302AF054689460AD18368B3F942
:102DE0000260FEF73BFE00284ED043680546984639
:102DF00001E0804600264046FEF730FE04460028EB
:102E000042D04545836818BF68601A461B7ED0F8DB
:102E1000048008BF0546FF2B0CD1002E40F08C80AB
:102E200007F1100A5046FEF77DFB7860002840F05D
:102E3000978029E01346183310226A497B601846B0
:102E40000AF0CCFC48B17968002E3DD107F10C00A6
:102E500000F030FD064600283BD0B9F1000F06D047
:102E6000424621463046FFF74FFF00280CDB214643
:102E70000022CB6849681A440029FAD10223084687
:102E8000FEF7ECFC064608B928461AE08368984627
:102E9000E268A16840460AF0D3FCE36864684246F1
:102EA0001A449046002CF3D12846FFF7D5FE4E4B2E
:102EB0003146B3F9000002F047FB002800F38E8092
:102EC0003046FFF7C9FE89E0304600F0CBFC002811
:102ED000C3D107F1180B08230BF80D3D32467B6870
:102EE000594607F1100004F0DDF80028EA4608DC36
:102EF00000957B683246594607F1100002F0D8F879
:102F000048B10646B9F1000F09D042462146FFF705
:102F1000FBFE002803DA2846FFF79EFE0AE0F97A56
:102F20002A4607F11000FFF79AFE014610B130461D
:102F3000FFF7B6FED54651E0B9F1000F06D0424684
:102F400021463046FFF7E0FE00289DDBAA68137992
:102F500043F04003137129463046FFF7A1FE3DE0E0
:102F60007B682846591EFEF759FDB9F1000F20D0A5
:102F70002846FEF773FD0446D0F804B0002883D03D
:102F80000246D8F804309B450AD058463A60FEF70E
:102F900065FD3A68506050B1DBF804B00246F0E7D6
:102FA00021463AF91600FFF7AFFE002801DA204665
:102FB00087E7002122460846FFF751FE044668B124
:102FC000A2683AF91600137943F0400313712146C1
:102FD000FFF766FE7B680136B342C6D11C37BD469B
:102FE000BDE8F08F35FE0008AC3400201FB50F4C53
:102FF000B4F9003063B90E4A01930E4B029200936C
:10300000042208234FF480610B48FDF7BBFE2080AB
:103010000A480B4B0360012303710523836008F00A
:103020003DFEB4F9000004B010BD00BFAC34002078
:103030008CFB0008C1320008AE3400207834002038
:10304000B0380020292B2DE9F84381460F4614465D
:103050001D4606D03A2B06D0112B0CBF04230023AB
:1030600002E0022300E00323292D3B7401D03A2D16
:1030700003D1A74259D1012605E0A74202D06368D7
:103080009F4252D100267B6893F91000022805D098
:1030900016B301212046FEF7C1FC1DE0294602F0CF
:1030A0002DFC18B986F0010836B101E04FF0000898
:1030B00001212046FEF7B2FC234640F201221E49C0
:1030C00097F9100002F0FAF910B92046FFF7C4FD95
:1030D000B8F1000FDCD00AE0234640F20122294675
:1030E000022002F0EBF910B92046FFF7B5FD06B358
:1030F000292D07D03A2D18D121464846BDE8F8437E
:1031000008F054BF00232374616839B191F910307D
:10311000022B03D12046FEF753FAF5E7022323746E
:103120002046BDE8F84300F00BB804490320FDF742
:1031300089FDBDE8F88300BF0000FFFF00F800082C
:103140002DE9F047044618B95B490320FDF77AFDE5
:103150004FF0FF3102F0FFFB18B18368B3F9025062
:1031600000E005462746264696F91030022B08D186
:10317000F368282B05D1B3681B7803F0F003602BAC
:1031800008D0D6F804803746B8F1000F6ED0464616
:10319000EAE73C46D6F80880E368B8F8041049BA74
:1031A00089B2994203D22046FEF7E0FB0FE02246A7
:1031B0000023D068034492F91000022803D1283B71
:1031C000994204D95DE05268002AF2D1F7E708F18C
:1031D00018091022394948460AF000FB002855D04A
:1031E0004846FFF721FD494600B135B9002000F0FF
:1031F00061FB002D08BF054602E0284600F032FBC7
:10320000B0FA80F04009002840D008F10800FFF72C
:103210000BFDB0BB4846FFF707FD90BB98F80730A1
:10322000013BDBB288F807305BB33046FEF716FC93
:1032300038B34FF0FF31204602F08DFB014610B14C
:103240002046FEF7BDF9214600250846FEF706FC9C
:1032500018B92846FFF700FD13E0416845600546B0
:103260000029F2D1BDE8F047FFF7AEBDA3681B7897
:1032700003F0F003602B04D12046FEF7EFFB074676
:1032800068B92046BDE8F047FFF7E6BC98F806307D
:10329000224639462846BDE8F047FFF7D3BE022252
:1032A0002821FEF7F5FA87F81080064600287FF4FB
:1032B00070AF3846E6E700BF00F8000835FE0008AA
:1032C00010B5102298B00DEB020000210AF0B6FBF9
:1032D000544B0593544B08211B88ADF81C3008A8AB
:1032E000FFF76AFC04A9022002F0BCFA40F20523B1
:1032F000ADF80A3000246846FFF75BFCBDF80230E9
:103300006FF400721344222BF5D801A252F823F077
:103310009D330008A5330008AF330008AF33000821
:10332000F7320008F7320008F7320008F7320008D9
:10333000F7320008F7320008F7320008F7320008C9
:10334000F7320008F7320008F7320008BF330008F0
:10335000F7320008CB330008DB330008E333000802
:1033600013340008F7320008D3330008F73200089E
:10337000F7320008F7320008F7320008F732000889
:10338000F7320008F7320008F7320008EB33000884
:10339000F3330008FB3300080B3400080198FFF7F3
:1033A000CFFEA8E701210198FFF70EFDA3E76FF01C
:1033B000850302A968460393FFF7CAFB9BE7019ABE
:1033C000537F23F00803537795E7019801F01EF827
:1033D00091E7019801F0AAF88DE7019802F060F8F2
:1033E00089E7019802F05FF885E7019803F0D2FDC4
:1033F00081E7019803F024FE7DE7019B587C00F0F3
:103400000F0002F02FFC047475E7019804F0A2F895
:1034100071E701980023021D1946B0F91E0001F062
:10342000E5FB68E70000FFFF9C0200200121FFF799
:10343000A7B9000008B5102203490AF0CFF9B0FA85
:1034400080F0400908BD00BF25FE000810B5082225
:10345000094904460AF0C2F948B12378FF2B08D184
:10346000607800F00F00831E5842584110BD0120C3
:1034700010BD002010BD00BFD5FD00082DE9F843A8
:1034800000F5C475044628468846FFF7CFFF00269E
:103490004FF0380909FB06474146384604F023FE41
:1034A00030B31022002138460AF0C8FA00233B74DA
:1034B000B4F88E3103F00603062B12D198F80030D1
:1034C000FF2B0ED04046FFF7C1FF50B9032328461B
:1034D00084F89431FFF784F92046BDE8F84301F001
:1034E000DFBF04F027F83A46214604F0B7F902E0BE
:1034F0000136072ECED12846BDE8F843FFF770B954
:1035000003885BBA23F03F031B041B0C4FF6C06219
:10351000934209D00378FF2B08D1407800F00F00C8
:10352000052818BF0E207047052070470E207047F1
:103530002DE9F0470025804691461F460C462E4651
:103540004FF0010A3FB13A780AFA05F31A421AD04D
:10355000237CDB0717D42046FFF76CFF98B9494658
:10356000204604F0D5FD37B999F80030FF2B02D082
:10357000637C834207D8B04205D9B8F1000F01D06F
:10358000C8F8004006460135072D04F13804D9D1AA
:103590003046BDE8F0870000094AB2F98C31834219
:1035A00005D0B2F96C33834207D1012300E0002338
:1035B0004FF4F07000FB032070470020704700BFFD
:1035C00050390020B0F88E3113F0010F10B40246CC
:1035D00009D011B143F0020301E023F00203A2F885
:1035E0008E3110BC704710BC01F01EBFB0F88E3198
:1035F000DB0701D503F068BF01F0DABE2DE9FF4714
:10360000002605468846924699463446AF194146FB
:10361000384604F068FD002840F0A1803846FFF7E6
:1036200009FF10B1002C08BF3C463836B6F5C47F00
:10363000ECD12746002C00F0928010224146204613
:103640000AF0FEF8237884F811A0FF2B84F810907C
:1036500016D0B5F88E31D90712D501F015F981468B
:1036600070B105F5C4763046FFF7BAF8B5F98C01AC
:103670004B464A46214601F0B7F93046FFF7D6FEE1
:1036800098F80030FF2B04D1237C43F0010323740E
:1036900061E04046FFF7DAFE8146C8BB4FF0FF33DA
:1036A0006361A36103F046FF05F5C47682463046A8
:1036B000FFF796F801212846FFF798FF3046FFF7FD
:1036C000B5FE22462946504604F09AF8B5F88E31E8
:1036D00003F00603062B1FD13046FFF781F8B5F83B
:1036E0008E31DA0706D54B464A464946B5F98C0174
:1036F00001F07CFAB5F88E31DB0705D4032385F899
:103700009431284601F0CCFE3046FFF78FFE03E0EF
:10371000237C63F07F032374B5F88E3103F0030339
:10372000012B18D040F2FF220023CDE900234FF0F7
:1037300080730293FF238DF80C3098F80D308DF8CC
:103740000D30B8F80E30ADF80E30802200236946F7
:103750002846FFF753FF40F211236386646338461F
:1037600004B0BDE8F08700001A4BB3F98C219042F9
:1037700070B505462DD0002AB3F96C230CBF1C464A
:103780000024904225D02AB903F5F073002C08BF1D
:103790001C4600E0ECB104F5C4763046FFF746FE67
:1037A0004FF4A063A4F89031402384F892310023B1
:1037B000A4F88E31A4F88C51802207492046FFF7E7
:1037C0001DFF3046FFF70CF82046BDE8704000F0C2
:1037D000BBBE70BD50390020F5FD00082DE9F04159
:1037E0000D4617469846FFF7D7FE044610B900204D
:1037F000BDE8F0810029FAD00846FFF71BFE00283B
:10380000F5D1802FF3DC04F5C4763046FFF70EFEC9
:1038100043463A4629462046FFF7F0FE0446304626
:10382000FEF7DEFF2046BDE8F081000038B50D460A
:1038300060B90A4CB4F98C3113B12046FFF71EFE73
:10384000B4F96C3343B12946054801E0FFF7A4FE03
:10385000BDE83840FFF712BE38BD00BF5039002028
:10386000303B00202DE9F8438946FFF795FE0446DA
:10387000E8B100F5C4763046FFF7D8FD002504EB2B
:1038800005084946404604F02EFC074628B130465C
:10389000FEF7A6FF4046BDE8F8833835B5F5C47F8E
:1038A000EDD13046FEF79CFF3846BDE8F883BDE811
:1038B000F88300002DE9F041124E04460F46002522
:1038C000B0463946B6F98C011CB1FFF7CBFF20603A
:1038D00001E0FFF7C7FF38B14FF4F07303FB058534
:1038E000B5F98C01BDE8F0810135022D06F5F076C1
:1038F000E7D1002014B12060BDE8F0812046BDE88A
:10390000F08100BF503900202DE9F74302AD0026B9
:103910001B4C45F8046D8946804604F5C470FFF7DA
:1039200085FD33464A4621462846FFF701FE0746F5
:1039300028B1019BC8F80030B4F98C6100E006465C
:103940000F4C04F5C470FEF74BFF04F55A70FFF7F7
:103950006DFD00234A4604F5F0712846FFF7E8FDA7
:10396000B84284BF019BC8F80030064888BFB4F94C
:103970006C63FEF735FF304603B0BDE8F08300BF4F
:1039800050390020B83C00202DE9F34102AC00275B
:10399000884644F8047DFFF7FFFD00F5C475064630
:1039A0002846FFF743FD20463B4642463146FFF797
:1039B000BFFD044628461CB1FEF712FF019802E045
:1039C000FEF70EFF204602B0BDE8F0812DE9F04F72
:1039D00087B00F461546FFF7DFFD00F5C47380463C
:1039E00018460193FFF722FD0122002102A80AF0E8
:1039F00025F84646C3464FF0FF3A00244FF0010930
:103A00009BF80020FF2A12D05846FFF713FD70B92B
:103A100045B99DF8081009FA04F20A438DF8082008
:103A2000A24604E05846FFF711FD0028F1D1013409
:103A3000072C0BF1380BE3D1BAF1FF3F00F0878080
:103A400004AD22460021284609F0F8FF3B78FF2B01
:103A500004D197F8019009F00F0309E03846FFF709
:103A6000F5FC20B93846FFF74BFD009001E002233A
:103A700000934FF000094C469DF80810012303FA0B
:103A800004F2114232D039463046B34604F02BFBE3
:103A9000002855D13046FFF7D9FC18B93046FFF75A
:103AA0002FFD00E00220009B834208D12A5D0432F2
:103AB000D2B22A554A4588BF4FF004090AE009D915
:103AC0002A5D0232D2B24A4513462A5538BF4B46C8
:103AD0005FFA83F9B2694AB12A5D0132D2B24A452E
:103AE00013462A5538BF4B465FFA83F90134072C39
:103AF00006F13806C0D10122002102A809F09EFF7C
:103B000000209DF80820014601246E5C4E4504BF4C
:103B100004FA01F0024301F1010104BFD2B2012015
:103B20000729F2D108B18DF8082006A8002340F833
:103B30000C3D3A4602AB4146FFF7FAFCDDF80CB00B
:103B4000BBF1000F05D1382202FB0A8B01E04FF0D8
:103B5000000B0198FEF744FE584607B0BDE8F08F11
:103B60002DE9F04F8DB005A8FDF7DCFC0026DFF84D
:103B7000688103900DF112053746B346039B9E42C0
:103B800000F0A58035F9020FFFF706FD0446002876
:103B900000F0998000F5C47A5046FFF747FC0123F6
:103BA000B5F90000009300220DF1110317218DF8E3
:103BB00011B001F0D7FC86302AD09DF91130012BCD
:103BC00026D108230DF13009ADF818304FF6FF73F8
:103BD00029F8103DB8F88E31B5F9000043F0030321
:103BE000A8F88E3102230093002206AB052101F0D4
:103BF000DFFC0223B5F90000009311214B4600229F
:103C000001F0B0FCBDF82010B5F9000003F092FE01
:103C10004FF00809B5F90000CDF8009006AB00227E
:103C2000494601F09FFC00280FDB4A4606A90AA876
:103C300009F006FE4A46274908A809F001FE0023BC
:103C4000402208A92046FFF7D9FC0223B5F900005D
:103C5000009300220DF11203112101F083FC0028D2
:103C600006DBBDF81230B3F5A06F28BFA4F8903181
:103C700000231A462421B5F90000CDF800B001F068
:103C800071FCB4F88E310028CCBF43F0800323F0E0
:103C90008003A4F88E315046FEF7A2FD0121204694
:103CA000FFF790FCB4F88E31DB070CD53FB93946ED
:103CB00008A803F083FD39462046FFF797FC20460D
:103CC00003F04EF90127013608F5F07856E70DB0FC
:103CD000BDE8F08FD5FD0008503900202DE9F341F3
:103CE0000746884616461C4608F046FB054640B97E
:103CF000032300933246A3B24146384608F0C2FA85
:103D000020E0437F03F00703012B01D103210DE0E5
:103D1000027FA3B29A4200F114070CD031462C77EF
:103D20002246384609F08CFD0321284602B0BDE842
:103D3000F04100F0BDBE22463946304609F04EFD46
:103D40000028EBD102B0BDE8F08100002DE9F04F72
:103D50001D46D37991B0FF2B8046069116461A9FD7
:103D600040F0B4806B78002B40F0B080172F40F209
:103D7000AD802B7AFF2B00F0A98002F1080955498C
:103D80001022484609F02AFD70B105F108014046AD
:103D9000FFF768FD0590002800F098800023183F89
:103DA0001C4619469A461BE00D224B4906F11800A5
:103DB00009F014FD002800F08980E6E70AF11802F6
:103DC00005EB020BAA5C012A0DD0212A08BF5C4634
:103DD0009BF801200AEBC20A1FFA8AFAA7EBC20776
:103DE000002FEBDC0BE008AB2A78069800933146F5
:103DF0005B4601F03BF8031E68DB5946E8E74046A6
:103E000007930691FFF7C8FB0699079B18B933493A
:103E10000320FCF717FF08AA002942D0002C40D04D
:103E2000B0F88E1101F0030103293AD129780293E9
:103E300001924B460A4600943146404603F00CFA84
:103E4000002304F108020F21074603F0EBF90546B1
:103E500017B91022494620E0237A83F002038DF837
:103E60002830637A8DF82930A37A8DF82A30E37AE6
:103E70008DF82B30237B8DF82C30637B8DF82D3023
:103E8000A37B8DF82E300822E37B8DF82F300AA912
:103E90000EA809F0D5FC124908220CA809F0D0FCA4
:103EA00009E049464046FFF719FF102249460CA891
:103EB00009F0C6FC0025337E0095A3F1FF025342B2
:103EC000534105990CAA404600F002FD11B0BDE82F
:103ED000F08F00BF25FE000815FE000800F800085E
:103EE000D5FD00082DE9F04F89B003F1080992468D
:103EF000059149461D468046129E08F03DFA9AF803
:103F00000730FF2B40F0DF806C78002C40F0DB8026
:103F1000172E40F2D8802B7AFF2B00F0D480002897
:103F200000F0D180183E2746002E27DD07F1180348
:103F300005EB030BEB5C022B0DD0212B16D10023DC
:103F40002A7802930193CDF800B04B465146404683
:103F500003F082F90AE006AB2A78059800935146EF
:103F60005B4600F0CAFF041EC0F2AD809BF8013032
:103F700007EBC307BFB2A6EBC306D5E74FF0FF318F
:103F8000059801F0E8FC08B1876800E0074649465B
:103F9000404608F0F1F90646002800F09480437F7F
:103FA00003F00703022B38D127B13B7813B17B789C
:103FB000002B3BD106A9A6F81E802246347706F1D5
:103FC000140009F03DFC2B79404F59064CBF0721E6
:103FD0000321304600F06CFD95F90430002B737F0F
:103FE0004FF00005B4BF43F0080323F008037377D4
:103FF000A8463468002C66D0236833606168256069
:10400000B7F9000001F093FA002803DC0021606892
:10401000FDF716FDC4F80480EBE7002F4BD03B788A
:10402000002B48D07B78002B45D002E0002CC1D17A
:1040300049E0002C3DD0337F9C4209D0224606A99E
:1040400006F1140009F0CAFBB0FA80F0400900E064
:10405000002007462B799A0602D40FB154B11EE016
:1040600044B1A6F81E803477224606A906F1140052
:1040700009F0E6FB2B795B0601D5072101E01FB1B2
:104080000321304600F014FD95F90430002B737FB6
:10409000B4BF43F0080323F00803737713E0737F82
:1040A00003F00703072B0ED10321304600F000FD7B
:1040B00009E02746CEE724B9377F003718BF01272C
:1040C000C8E70027C6E709B0BDE8F08FAC34002090
:1040D0002DE9F04F87B01546984681460291109F12
:1040E000FFF75AFAB0F88E319A07064669D5EB7990
:1040F000FF2B66D198F80140002C62D1072F60D9C0
:1041000005F10803083F0DF1100A0393002F1FDD8E
:1041100004F1080308EB030B18F80330012B0FD14F
:1041200098F800200298CDF800A05B46294600F0E0
:104130009DFE031E45DB524603994846FFF7CEFD20
:104140009BF8013004EBC304A4B2A7EBC307DDE77F
:10415000B6F88E3113F0040F05F1080528D013F0DE
:10416000010F194B194C18BF1C46FDF7ADFD06F5A4
:10417000E27780463846FCF7B7FCB6F88E31DB07AD
:1041800016D52946484608F0F7F888B1B8FBF4F18F
:1041900040F21523A6F8DA310D4BC6F8DC01B3F96D
:1041A000003006F5EC7204FB1181384606F070FB16
:1041B0002946484608F0E0F818B1437F23F0080389
:1041C000437707B0BDE8F08F80841E0020A1070070
:1041D000AC3400202DE9F04F89B09246059181461C
:1041E0001E46FFF7D9F90AF1080B05460822844953
:1041F000584609F0F3FA002840F0FF809AF808309A
:10420000FF2B00F0FA809AF80730FF2B40F0F58082
:104210007378002B40F0F180129B0F2B40F2ED8061
:104220005946484608F0A8F8074650B90B230093B2
:10423000024603465946484608F024F8074668B93E
:10424000DBE0437F190706D5F28852BA92B212B961
:1042500023F0080301E043F008037B77F3889CB266
:1042600064B15CBA674B68491B88A4B21BB207F102
:104270003402614307F1200006F00AFB33790BB1E9
:1042800085F89231B5F88E31C3F30D02A5F88E2171
:1042900073791B0203F440431343A5F88E31B068D1
:1042A000A8B1D5F89C3190FA80F898450FD0FDF769
:1042B0000BFD0A22B0FBF2F303FB1200053008FBF2
:1042C00000F0C5F89C81B0FBF2F0C5F8A001F368DE
:1042D00013B11BBAC5F8A43105F5C470FEF780FA16
:1042E000129B103B0393002302930493039B002B28
:1042F00058DD029B103306EB0308F35C052B1CD042
:1043000004D8012B0DD0032B1ED03FE0222B2AD046
:10431000232B3BD14346129A3146484603F052F9CB
:1043200034E006AB0093327805984346514600F0DE
:104330009DFD031E049329DA5FE04246317848462A
:1043400000F015FE10BB58E042463178484600F0B8
:104350002BFE002851D0D8F804301BBAB3B19C42D0
:1043600028BF1C4612E04146307803F047F8002889
:1043700043D0B8F806305BBA9BB23BB13C22B4FBE9
:10438000F2F2934202D23C2202FB03F498F801308D
:10439000029A02EBC30292B20292039AA2EBC30307
:1043A0000393A3E7049B06AA59464846FFF796FCE9
:1043B00005F5D470FCF798FBB5F88E31DA071CD5FB
:1043C00004EB4404042C88BFA1084FF0000498BFFC
:1043D0000121384685F8934102F0F8FE3B1D1A464C
:1043E0002146B7F91E0000F0FFFAB5F88E319B07A1
:1043F00003D501212846FFF7F9F809B0BDE8F08F91
:10440000D5FD00089C02002040420F002DE9F0413C
:10441000437F03F00703022B86B0044601D0052B2F
:104420007DD194F8B420B4F91E50012A73D9022B1F
:1044300011D14FF080730493FF238DF81430637C07
:104440008DF8153040F2FF200021638AADF8163058
:10445000CDE902010BE0211D03C902AB83E8030093
:1044600004F10C0393E8030006AB03E90300013AEF
:1044700084F8B4202DBB01AE3046FDF753F804F1AB
:1044800004080746BD4208D036F9150002AB424683
:10449000002100F0A9FA0135F4E7224B04F13C05B4
:1044A000B3F900602846FCF71FFB40F21223A4F882
:1044B000523004F1500233461B49284606F0E8F911
:1044C0002DE02846FFF768F80646221D02AB06F5E8
:1044D000C475B4F91E00002100F086FA01212846B7
:1044E000FEF74EF90F4BD6F8A471B3F9008004F132
:1044F0003C063046FCF7F8FA40F21223A4F852309A
:104500003046434604F15002394606F0C1F92846C8
:10451000FEF766F903E0211D284607F055FF06B0B7
:10452000BDE8F081AC34002040420F00437F03F02F
:104530000703042B03D0072B04D1032100E005213E
:1045400000F0B6BA7047000038B500F5C4750446EF
:1045500001212846FEF714F9FDF7B6FB0A210A4BA4
:10456000B0FBF1F202FB11000530C4F89C3143436B
:10457000B3FBF1F3C4F8A031044BC4F8A4312846CE
:10458000BDE83840FEF72CB980C3C90140420F0096
:1045900010B5044608462378FF2B14D000221823B8
:1045A000872107F06DFD002270B183681A715A717E
:1045B0009A71DA7121686268DA609960A168E268CC
:1045C0005A61196110BD002010BD38B50B78FF2B62
:1045D00005460C46104616D000221823882107F005
:1045E0004FFD002280B1836825F01F051D71DA712F
:1045F0009A715A7121686268DA609960A168E2680C
:104600005A61196138BD002038BD08B50022082361
:10461000852107F035FD28B1836800221A715A718F
:104620009A71DA7108BD10B5002304461046CA1D00
:1046300002F0F8021946FDF711F920B182681470F2
:10464000C368DB08537010BDF8B516460F461A460E
:10465000B11CFFF7E8FF044660B18568C268023507
:10466000023A0021284609F0E9F93246394628463F
:1046700009F0E6F82046F8BD13460A460146012037
:10468000FFF7E2BF13460A4601460220FFF7DCBFF0
:104690002DE9F04180460F4616461D4600221023A4
:1046A0008621079807F0ECFC60B1069B846827F030
:1046B0003F0776BA2DBA1BBA84F804806771E6808A
:1046C000A560E360BDE8F0812DE9F041074688462A
:1046D00016462021079A03201C46FFF7A4FF054633
:1046E000C8B1806824BA0021846028F03F0800F136
:1046F000100436BA017341738173C173877080F8F7
:10470000038046601022204609F098F93A4606993F
:10471000204603F023FD2846BDE8F08110B50A4687
:10472000044608210520FFF77EFF28B18368002298
:1047300024BA9A70DA705C6010BD000008B51022CF
:10474000034909F04BF8B0FA80F0400908BD00BFFA
:1047500025FE000810B508220949044609F03EF874
:1047600048B12378FF2B08D1607800F00F00831E3A
:104770005842584110BD012010BD002010BD00BF9F
:10478000D5FD000870B506460846194607F002FD3B
:104790000446A0B18368FF22DA7100231A46194645
:1047A000184601F029F8054620B921462046FCF7B5
:1047B00007FF02E083685E804460284670BD70BDDC
:1047C0000021FDF73DB90000F7B51F46537C802B53
:1047D00005460E46144603D911490320FCF732FA68
:1047E0001046FFF7ABFF08B1002017E02046FFF7A7
:1047F000B1FF0028F8D1217CCB07F5D43388607C49
:10480000626913F0010F14BF002680268DE8900026
:10481000A3693143FFF758FF2860012003B0F0BDC2
:1048200000F8000830B585B0022300930D460DF165
:104830000E0300220521044600F094FE002803DB4D
:10484000BDF80E30062B10D80823009300222B460B
:104850000221204600F086FE002802DBADF80E00A3
:104860000EE00023ADF80E300AE00823009300228A
:104870002B460321204600F075FE0628E4DDEDE717
:10488000BDF80E0005B030BD38B5002007F0C0FD02
:10489000044660B1637F03F00703013B012B04D999
:1048A0000A4B00221A60201D38BD2046EEE7074D56
:1048B000286807F0ADFD034618B907F0A9FD0346C7
:1048C00010B12B60181D38BD204638BD103D0020AA
:1048D0002DE9F7430A9C0F46994680461646FEF797
:1048E0005BFEB0F88E31990701D4002507E0404601
:1048F000FEF752FEB0F88E315A07F6D580253046C5
:10490000FFF71CFF38B110223349304608F098FFFA
:104910000223737001E045F04005B9F1000F0BD0A0
:1049200069464046FFF77EFF30B1C1B22246684675
:10493000FFF7A8FE68B1044624B13B7CDB0758BFF3
:1049400045F02005224639462846FFF73EFE8146BF
:1049500008B920463BE00146002332464046FFF7B7
:1049600011FF054608B9484631E03B7CDFF87490FA
:1049700013F0010F23D0FDF7A7F9184BB0FBF3F7A5
:10498000314607FB1307404607F0F6FC044618B90A
:1049900013490320FCF756F900F158063046FCF79E
:1049A000A3F840F20223A4F86E302567B9F900306D
:1049B00004F16C023946304605F06AFF09E0014611
:1049C000B9F9000000F0B3FD002802DC2846FFF72B
:1049D000F7FE03B0BDE8F083E5FD000840420F009C
:1049E00000F80008AC3400202DE9FF4707460D46CB
:1049F00090469946FEF7D0FD824618B92A49032011
:104A0000FCF720F935B92A4641463846FEF7DEFF65
:104A1000054668B102A93846FFF704FF064650B1C3
:104A2000C1B2002202A8FFF727FE044620B935E0F4
:104A30000646044600E00446BAF88E31DB0714D57A
:104A4000082E0AD00823009300226B440321384625
:104A500000F088FD80B208281FD1234602AA0F214A
:104A6000002002F0DFFBC0B1044621464046FFF7BC
:104A70008FFD064688B101462B464A463846FFF769
:104A800081FE044608B9304608E0084B0146B3F9F8
:104A9000000000F04CFD002802DC2046FFF790FEED
:104AA00004B0BDE8F08700BF00F80008AC34002077
:104AB0002DE9F041437F23F007030B43052904460A
:104AC000437720D0072903D004294BD1264E05E097
:104AD000B0F91E00FEF760FDD0F8A061234B04F191
:104AE0003C05B3F900702846FBF7FEFF40F21723A0
:104AF000A4F8523004F150023B4631462846BDE846
:104B0000F04105F0C5BEB0F91E00FEF745FD0323D8
:104B1000064684F8B430231D1A4606F5C475B4F968
:104B20001E000021FFF760FF01212846FDF728FE47
:104B30000E4BD6F8A471B3F9008004F13C06304660
:104B4000FBF7D2FF40F21223A4F85230304643461E
:104B500004F15002394605F09BFE2846BDE8F041BD
:104B6000FDF73EBEBDE8F081404B4C00AC34002068
:104B70002DE9F3411B4D002918BF0D46002229469F
:104B80008046FEF723FF074670B169464046FFF7AF
:104B900049FE38B1C1B200226846FFF76DFD0446F8
:104BA00018B91AE0044600E004462046FFF72DFD40
:104BB000064688B101463B462A464046FFF7E2FDDD
:104BC000044608B9304608E0074B0146B3F9000037
:104BD00000F0ADFC002802DC2046FFF7F1FD02B03A
:104BE000BDE8F08105FE0008AC3400202DE9F04F4F
:104BF0008BB0002791468A46039302900797FEF7F1
:104C0000CBFC964B064600F5C47801214046B945D9
:104C100008BF9946FDF7B4FDB6F88E5115F00105B1
:104C20001BD1344606F5C777B3465C4500F0ED80EE
:104C3000627C9BF811309A4240F0E480594620464D
:104C400003F066FA637C834200F2DC8000E01D46DC
:104C50003834A045E8D1079D4FE002F06BFC0546D3
:104C600000284AD0846906F5C77BECB163689E4290
:104C700018D1AB699C4200F0D780A268996892F87D
:104C800011E0487C864540F0E3801046059304928D
:104C900003F03EFA049A059B527C824200F2D880CF
:104CA00000E01F462468E0E74FF0010B05EBD4035A
:104CB0009A7D04F007030BFA03F31A420CD0E0B21A
:104CC00000F0D0FF428A417C0346007C009702F04E
:104CD00033FD079060B107460134102CE6D12A4617
:104CE000A98A28693B4602F04DFD0546079020B988
:104CF0004046FDF775FD384681E0B6F88E311B075A
:104D000007D52946B6F89001FFF708FD0790F8B1DE
:104D10000546BAF1000F0FD14046FDF761FD494647
:104D200001220298FEF752FE012182464046FDF71D
:104D300027FDBAF1000F10D008A90298FFF772FD05
:104D400058B1C1B22A4608A8FFF796FC079018B9D7
:104D50004046FDF745FD3DE00546B6F88E2102F0E0
:104D60001004A4B20CB196F8924102F020039BB259
:104D70004BB1D6F8A0313A498B4206D84FF47A7B32
:104D8000B3FBFBFB03E09B4601E0DFF8DCB002F085
:104D90004007BFB22FB1D6F8A4714FF47A73B7FBB6
:104DA000F3F7039B13B9B6F89A2100E000224046BE
:104DB0000392FDF715FDB6F88E11039A01950912BD
:104DC000204600975B4601F0C001FFF761FC0446F6
:104DD000079008B9284612E0014653464A46029811
:104DE000FFF7D0FC0146079008B9204607E01D4BAD
:104DF000B3F9000000F09BFB00282BDC0798FFF7BD
:104E0000DFFC27E00BF1380B0FE72B462246394633
:104E100007A8FFF7D9FC00283FF41AAF079B002B27
:104E20007FF415AF28460DE03B46A268594607A817
:104E3000FFF7CAFC00283FF435AF079B002B7FF437
:104E400030AF3846FFF7BCFC4046FDF7C9FC01E037
:104E50001B680FE70BB0BDE8F08F00BFF5FD000841
:104E600000A493D6AC34002080EE3600F8B51E4680
:104E70009F1C5B780446154613B96FF01500F8BD0A
:104E800001F10800FFF75AFC0028F6D17CB394F931
:104E90001030013304D1A3681C78022C04D001E047
:104EA0006468F3E7082C06D17378012B14D0022B29
:104EB000E3D1082411E0853D022D1BD884B9727816
:104EC00008236FF0010413FB024402FB036616F88B
:104ED000013D2BB9013CFAE70224853D022D09D89A
:104EE00022463946069808F0ABFC2046F8BD853DC1
:104EF000022DE4D96FF08500F8BD70B51D465B78D2
:104F00000446164613B96FF0150070BD01F1080094
:104F1000FFF714FC0028F6D1882E27D1A91CA4B1D4
:104F200094F91030013304D1A3681C78022C04D00A
:104F300001E06468F3E7082C06D16B78012B0ED0F2
:104F4000022BE0D108240BE054B96C78E408023C51
:104F5000E4B20B1913F8013C13B9013CF8E7022441
:104F60002246049808F06CFC204670BD70BDF8B570
:104F700017460D46FEF710FB7C78012C06460FD134
:104F8000862D0FD100F5C47521462846FDF7F8FBA4
:104F90007B681BBAA6F890312846FDF721FC01E09A
:104FA0000020F8BD2046F8BD2DE9F0415378042BD0
:104FB00086B00746154671D186294ED102F11008F8
:104FC0004046FFF7C7FB0646002846D13846FEF7A5
:104FD000E3FAB0F88E31DA0703D595F90330002BE8
:104FE0003BDB41463846FEF73DFC044618B1427CA7
:104FF000AB789A422AD06B6843B31022002102A8F2
:1050000008F01CFDEB785B0616D4AA78414602A88E
:1050100003F0A4F8EB78AA7803F0C00302A938469D
:10502000FEF7DCFB0446002839D03846FEF7B4FA18
:10503000012102F049FA09E00821009104AB0022A5
:10504000384600F08FFA0028DFDA28E06B6833B9C1
:105050001CB121463846FEF7E9FB01261FE01BBACA
:105060006361AA68013312BAA2610CD00E4B696861
:105070000E481B8809BA41431BB204F1300204F107
:105080001C0005F005FC237C23F07F03DBB22374B6
:10509000EA7822F03F0213432374DEE7002630460D
:1050A00006B0BDE8F08100BF9C02002040420F0026
:1050B0002DE9F04391B01D4604460F46ADF8162089
:1050C000002308227649DDF860800693284608F020
:1050D00085FB18B9002D33D0284634E02B78FF2B00
:1050E00004D16B7803F00F03022BF3D010230022BE
:1050F000079302930CAB0C9203920093019507ABBC
:1051000008AA0DF11601674806F05EFD002804DBD1
:10511000079B102B01D108A8A8B9BDF91600294694
:1051200028B906A8FEF7F0FBADF8160002E0FEF77E
:105130002BFC0690069B1BB193F91030002BC9DBAA
:10514000FFF7A2FB00B105462946BDF9160007F09E
:1051500013F9064638B1437F03F007035A1E012AAC
:1051600000F291808DE002230093BDF916003346D2
:105170003246294607F086F8044600B98DE04A4BCE
:1051800003EBC6077A6882B953F83690B9F1000F7D
:105190000BD1C7F8048001214046FCF73FFC424B8D
:1051A00043F83690236823B909E00136202EE7D171
:1051B00006E01A680AB11346FBE71F6000E02760AB
:1051C000002340F2FF22CDE90C234FF080730E93B1
:1051D000FF238DF83C306B7B8DF83D30BDF91660B8
:1051E000EB89ADF83E301EBB07AF3846FCF79AF9A5
:1051F0008046464508D037F916000CAB2A460021F8
:10520000FFF7F2FB0136F4E7284B04F13C05B3F954
:1052100000602846FBF768FC40F21223A4F85230E5
:1052200004F1500233462249284605F031FB28E0BC
:105230003046FEF7B1F906462A460CAB06F5C475B2
:105240000021BDF91600FFF7CFFB01212846FDF72D
:1052500097FA164BD6F8A471B3F9008004F13C0616
:105260003046FBF741FC40F21223A4F8523030469E
:10527000434604F15002394605F00AFB2846FDF783
:10528000AFFA002009E0032B02D10421FFF710FC44
:1052900032463946204607F0F1F811B0BDE8F083F8
:1052A000D5FD000878340020143D0020AC340020E7
:1052B00040420F002DE9F047044600F5C4778946C7
:1052C00038460121FDF75CFAB4F89AA1B4F8985178
:1052D000BAFA8AF84FEA581815B1B4F896611EB9AF
:1052E0002E490320FBF7AEFCFCF7EEFC94F894315A
:1052F000761B012BB0FBF6F101FB160005440ED91D
:10530000013B84F89431BAF1000F04D194F8943140
:10531000012B07D81BE0102D28BF102502E0BAF1A1
:10532000000FF3D004F5E2763046FBF7DDFB40F2E8
:105330001323A4F8DA311A491A4BC4F8DC41B3F943
:10534000003004F5EC726943304605F0A1FA3846A6
:10535000FDF746FA254610221349284608F03EFA82
:10536000B8B108221149284608F038FA38B12B782C
:10537000FF2B0ED16B7803F00F03022B09D12B7C8E
:10538000DB0706D443464A462946B4F98C01FFF7A9
:105390002DFC3835AF42DED1BDE8F08700F80008BB
:1053A00040420F00AC34002025FE0008D5FD000867
:1053B00070B504460E46B0F88E51B9B105F004053B
:1053C000ADB27DBB00F5C47601213046FDF7D8F9BA
:1053D000B4F88E3143F00403A4F88E31032384F82B
:1053E00094313046FDF7FCF9294616E06B0719D5D4
:1053F00000F5C47501212846FDF7C2F9032384F89E
:105400009431B4F88E31A4F89A6123F00403A4F81F
:105410008E312846FDF7E4F931462046BDE870405C
:10542000FFF748BF70BD000038B504460D46B0F820
:105430008E3121B39A072FD4012380221749B0F966
:105440008C0104F5C475FEF7C9F901212846FDF762
:1054500097F9B4F88E3143F00203A4F88E314FF47B
:105460001673A4F89631C823A4F898314FF4E16379
:10547000A4F89A312846FDF7B3F9012107E09B070C
:105480000AD50649B0F98C01FEF7D0F92946204625
:10549000BDE83840FFF78CBF38BD00BF05FE0008EF
:1054A0000021FFF707BF10B50446B0F91E00FEF754
:1054B00073F8211DBDE81040FFF7FCBE2DE9F34154
:1054C0000446884617461D4600F018FA064650B3B3
:1054D0004146204600F000FA711E04462846FCF7BB
:1054E0009DFA04B3237A53B1012B17D1E068ADF8CC
:1054F000027000226946019506F0C6F807E0B4F98B
:105500000C10ADF8027068460195FDF7CFFA00283F
:1055100004DD204600F006FA0446E2E700212846B2
:10552000FCF78EFAF5E7304602B0BDE8F08107B52A
:1055300040F20223019101466846ADF80230FDF7C2
:10554000B5FA03B05DF804FB07B540F20123019101
:1055500001466846ADF80230FDF7A8FA03B05DF8E1
:1055600004FB000000B589B006930A9BADF81C301F
:105570004FF401738DF81410ADF81620ADF8063015
:10558000024605AB03A901A80293FDF7B3FABDF8E3
:105590000E2040F205239A4203D004490320FBF772
:1055A00051FB049809B05DF804FB00BF00F8000847
:1055B00000B589B006930A9BADF81C3040F2032376
:1055C0008DF81410ADF81620ADF80630024605AB84
:1055D00003A901A80293FDF78DFABDF80E2040F251
:1055E00005239A4203D004490320FBF72BFB0498C0
:1055F00009B05DF804FB00BF00F80008F0B584684E
:10560000A68BE3898FB006F02800ADF8183040F083
:1056100001000D4611B96FF015004BE091F9103003
:10562000013342D189680B790A7813F0C00F03BFA8
:1056300002F108035B184F781F4B18BF02270AB10D
:10564000083107E0720747BF04F11201082204F194
:105650001001022294F81AE00EF10106A6760390DA
:1056600008AEBDF81800ADF80800ADF804000097CA
:10567000CDF810E0304602F0CFFB07460028CAD034
:10568000284607A9FBF770FF054688B181682368A3
:10569000079A1B6881E8C00020469847002104460D
:1056A0002846FCF7CDF9204604E06FF04C0001E0FD
:1056B0006FF068000FB0F0BDD3FD00082DE9F04396
:1056C00087683B685C68002387B01A4619463846ED
:1056D000A047041E15DD0023224619461846FCF794
:1056E000BDF8054668B13B6881685E6822466B4636
:1056F0003846B047B0F1000805DC00212846FCF729
:105700009FF9002465E0BE8B06F00206B6B2002EBB
:105710005AD1A86802F014FC044608B9014637E0E3
:105720000146C0EB080832462846FCF7B1F881462E
:1057300008B90146E2E7866801AA04A9304602F0EA
:1057400075FC01AA044602A9304602F01DFC002C9B
:1057500001DA00241BE00028FBDBC1B2E3B204AA9B
:1057600002A800F049F806460028F2D0022C0CD11D
:105770009DF81030FF2B08D19DF81130FF2B01BF91
:105780008268137963F07F031371344626B90021D0
:105790002846FCF755F91CE0B3689DF801209A7182
:1057A0009DF800205A710D4A12885A803B7B2B7459
:1057B00049462846FBF704FF002373602B465A68CE
:1057C0000AB11346FBE75E6041462846FCF7CEF877
:1057D0002C46204607B0BDE8F08300BF9C020020A5
:1057E000034B0360034B436081600020704700BFA0
:1057F000FD550008BD5600082DE9F041174603F19C
:1058000008020A440E46002180461D4608464FF015
:10581000FF33FCF723F800220446F8B183681E70BA
:105820005D705A805A719A711A71B8F1000F08D0E0
:105830003EB180680278B24203D14146083007F099
:10584000FFFF5FB155B1A0684378AB4206D1037842
:1058500008332A463946184407F0F2FF2046BDE8CF
:10586000F081000008B50B7A53B9B1F90C200B4B4D
:1058700053F822301B6A1BB909490320FBF7E2F9F0
:10588000C3B2042B9FBF074B53F820200A6043F894
:10589000201094BF00206FF0150008BDE802002022
:1058A00000F80008143E0020C3B2042B11D8094AA6
:1058B00052F820308B4206D11B6842F820307047E6
:1058C000914204D013461A68002AF9D101E00A680F
:1058D0001A607047143E0020C3B2042B09D8064B4F
:1058E00053F8200020B143688B4203D00068F9E7E9
:1058F00070470020704700BF143E0020C3B2042B45
:105900000BD8074B53F8203000202BB15A681B6886
:105910008A4208BF0130F8E770470020704700BF97
:10592000143E002028B14368006810B142689342D9
:10593000FAD1704749B190F91030032B03D0042BF2
:1059400006D102F00DB906F0ABBB6FF01500704741
:105950006FF00100704728B190F910308B4201D0F0
:105960004068F8E770470021FCF76AB82DE9F0417C
:105970009EB0102200210AA808F060F8804B0B931B
:10598000804B08211B88ADF834300EA8FDF714F9C0
:105990000AA90120FFF766FF40F20523ADF81A308F
:1059A00040F2032440F2012504A8FDF702F9BDF8F6
:1059B0001230B3F5017F09D8A34280F0D880AB4202
:1059C0000CD040F2022293426ED0EDE740F2252245
:1059D0009342E9D1059800F0EDF9E1E7059D2846ED
:1059E000FCF73CF8044600287ED00121FFF7B3FF06
:1059F000054608B1C3681BB92046FFF7B4FFCFE7DF
:105A000083681B78412B11D1FCF728F80546002844
:105A1000F2D001221146FBF73BFF01460028EBD0F4
:105A20002046FBF7CDFD0223044631E003F0D80207
:105A3000C02A03D1204600F0B1FAB1E703F0E00339
:105A4000602BD9D10021022328220846FBF706FF4C
:105A5000089010B9089890B9CEE703AB00930023E3
:105A600021461A4608A800F0DFFC01460028F1D0C4
:105A700001222046FBF70CFF014618B90898FFF7F2
:105A800072FFB9E72046089AFBF7B0FD00230446F1
:105A90002B7440F20122234639490220FFF70EFD04
:105AA00000287FF47DAFA7E7059DEDB1EB68072BDC
:105AB0001AD96B68C3B193F91030022B14D1284660
:105AC000FBF7CCFF044678B18768B7F9020001F014
:105AD0004DFF61688046002619B1CB6849681E44B5
:105AE000FAE7B8F1000F01D1284686E798F80430AC
:105AF00023B1204600F086FF70B97DE701231A46E6
:105B00000846FBF7ABFE00283FF476AF63684360BE
:105B10006060836841221A70626800231AB1D168FC
:105B200052680B44FAE7B8F80210994208D32146AC
:105B3000B7F90200FFF7FBFC00283FF731AF5BE746
:105B4000114B596800297FF457AFB6F5006FBFF4C9
:105B500053AF79889A8108A840F2252219805C60A9
:105B60009E60ADF822200993FCF742FF18E76FF022
:105B7000850306A904A80793FCF7EAFF10E700BF16
:105B80000000FFFF9C020020283E00201FB50A4CA9
:105B9000B4F9000000280DDC084B029300230193A8
:105BA000074B0093032208234FF480610548FBF75D
:105BB000E9F8208004B010BD3842002094FB0008B2
:105BC0006D590008383E002038B50E4B142404FBF4
:105BD00000340546638A63B10020FCF797FC0A4B4A
:105BE000B0FBF3F0094B53F82530834206D800236D
:105BF0006382637C23F01003637438BD1B1A6382D5
:105C000038BD00BF3A420020008793037C43002048
:105C10002DE9F041012180461048114DFCF7B0FDFF
:105C2000002426462746E0B2FFF7CEFF2B7C53B177
:105C30004146284602F06CFA2B7C834203D8B842D6
:105C400084BF2E4607460134102C05F11405EAD115
:105C50000248FCF7C5FD3046BDE8F081BC4300209A
:105C60003A4200200F2838B5044615D801210B48C8
:105C7000FCF786FD2046FFF7A7FF094B142000FB29
:105C8000043506482C7C1CB1FCF7AAFD284638BD1B
:105C9000FCF7A6FD204638BD002038BDBC430020DF
:105CA0003A4200202DE9F8430F280646884615465B
:105CB0001F469DF820903FD8002A40D0012121485E
:105CC000214CFCF75DFD002F4FF0140303FB06434E
:105CD00008BF4FF00009802D88BF80225F828CBFF3
:105CE0001A741D74B9F1000F02D046F0100300E0E1
:105CF0003346142000FB064441466374204602F0FC
:105D0000F2F9014640B91022204607F097FE227CA6
:105D10004146204602F022FA0020FCF7F7FB0B4B2D
:105D2000B0FBF3F00A4B0744064843F82670FCF733
:105D300057FD2046BDE8F8830020BDE8F8831046F3
:105D4000BDE8F883BC4300203A420020008793035B
:105D50007C4300200021FBF773BEF8B50E460178A6
:105D60004378174601F10802024405460830FFF760
:105D700043FD0446E0B18368B5F902205A802A79D0
:105D80001A716A795A71AA799A71B7424FF0000173
:105D90003A464FF0010328BF32460846FBF75EFD46
:105DA000054620B92046FFF7D5FF2846F8BD6060BC
:105DB0002046F8BD2DE9F04F054685B0B0F900004A
:105DC00001F0D4FDD5F80480D8F8044083464FF0A4
:105DD000000A1CB1E36864689A44FAE7BBF1000F5B
:105DE00005D14046FFF7B6FFC5F804B0D0E0B5F8DE
:105DF0000C90B9F1000F42D1674FAE683B88D8F8DC
:105E0000080001333B80CAEB06039AB2BBF80230AC
:105E1000043B134403F0F8039B1A1FFA83F909F1BA
:105E200004025146FFF799FF034600283AD0426822
:105E3000D2F808A076BAAAF800609AF8002062F0BA
:105E40003F028AF800203A8852BAAAF80220D8F80D
:105E50000470002F7CD0FA68B9680093C4EB09067F
:105E6000964228BF1646201D344432465044A4B200
:105E700007F0E6FCA145009B6AD97F68E9E7D145B8
:105E800080F08280BBF80260D8F80800AF68053E59
:105E900006F0F806C9F10501721D5144FFF75DFFD8
:105EA000034628B96868FFF755FF00236B606FE071
:105EB00042689268511D009179BA1180117861F0A1
:105EC0001F01117034494F440988CAEB070A49BAC7
:105ED0004FEADA0A518082F804A0D8F80470FFB1C2
:105EE000A1451BD0FA68A11889B2894513D2C4EB29
:105EF00009041FFA84F9C9EB0204B442B968009896
:105F0000019328BF34462246494407F099FCA4B2C5
:105F10007F68019B05E07F680C46E0E7002400E015
:105F20003C46A64214D99FB1FA680193C4EB060817
:105F30009045009BB96828BF9046181944444246D2
:105F4000A4B207F07DFCA642019B01D07F68EAE77E
:105F50001946BBF900000093FFF7E9FA0028009BFF
:105F600002DC1846FFF7F6FE002C9BD0AB890395A8
:105F70001C44AC8140F2252302A8ADF80A30FCF79E
:105F800037FDFAF7C5FE03E04046FFF7E3FE6C601D
:105F900005B0BDE8F08F00BFC043002010B5826897
:105FA000137803F0F803C02B044606D0E02B0DD184
:105FB0001379C268DB00053A02E0C2680023043AA4
:105FC00060682146806800F013F82046BDE8104064
:105FD000FFF7C0BE002203682BB119689A80DA80EF
:105FE0001A600160F7E7436070470021FBF728BDA6
:105FF0002DE9F04F8FB081460020924604911F4654
:106000008E68AA4DFCF782FAA94A834605F19008EA
:106010002C46606858B1A368C3EB0B03934206D9C2
:106020000292FFF7E2FF2046FFF7D4FF029A2434E2
:106030004445EED199F800B009F1080307930BF13C
:1060400008034B44069399F80130029333885BBAF6
:10605000C3F30A03059373885BBAADF826300020BA
:106060009BB20A93FCF752FA002308901C46039354
:106070006A68A846002A00F02581D26805999142F5
:1060800023D1EA8B0A998A421FD12A7F93451CD1DA
:106090006A7F0299914218D15A4607990B9305F1EC
:1060A0000C0007F09BFB0B9B78B9029A069905F14F
:1060B000140007F093FB0B9B38B97C4C039A242304
:1060C00003FB0244089BA3604EE014B96A6802B95E
:1060D0002C463BB1A9689A68521A76498A4294BF05
:1060E000A8469846039B0133042B039305F124052E
:1060F00001D04346BCE784B9B8F1000F03D16E4923
:106100000320FAF79FFDD8F804000028F7D0FFF726
:106110006CFF4046FFF75EFF444600210223059ACC
:106120000846FBF79BFB6060002800F0DD80836879
:1061300000210020C3E90001089BA3605A4607998B
:1061400004F10C0007F07CFB029A069904F114009C
:1061500007F076FB9DF808306377BDF82630E383BF
:10616000002384F81CB0238425680FBB3379412BAE
:1061700003D105360AF1FF331FE003F0E003602B83
:1061800006F1040618D10EAB204643F8047D50F802
:10619000042F0093D2680499042300F045F90028E5
:1061A0007CD00D9A28320AEB020306441B1A05E044
:1061B00005365346002201E053463A466068C168FE
:1061C00003EB070E8E456AD81FFA87FE0EF1FF31EA
:1061D000194489B26DB1B5F804804145C0F08280A0
:1061E000B5F806C0E6457DD8C6456FD161456DD18D
:1061F00078E01FFA83F80EF1FF314144DFF8C0A0C8
:1062000089B2AC460AEBCC05B5F806B0BBF1000F7D
:1062100011D1ADB1E98021682960A5F804E0218C95
:10622000256080684144174421849A1A31463844D5
:1062300007F006FB04E00CF1010CBCF1340FE1D1D6
:106240006368228CDB689A424ED1637F217F04F120
:10625000140204F10C00FFF7CFFAF8B18368B9F922
:1062600002205A8099F804201A7199F806209A7130
:1062700099F805205A710023436063682BB15A686E
:106280000AB11346FBE7586000E0606063680B49A1
:1062900040F201220220FFF711F910B96068FFF700
:1062A000A4FE2046FFF796FE1EE000BFC443002078
:1062B000C0C62D00FEFFFF7F00F800080000FFFFB2
:1062C00054440020002C7FF404AF01E7FFF78DFE5B
:1062D0002046FFF77FFE3B46524604994846FFF7AB
:1062E00087FE01E02D6875E70FB0BDE8F08F00BFB5
:1062F000037823F00F0343EA11130370437803F08C
:106300000F0343EA01114170704700000822014960
:1063100007F096BAD5FD00081022002107F08EBBC9
:1063200010B508220949044607F058FA48B1237805
:10633000FF2B08D1607800F00F00831E58425841AF
:1063400010BD012010BD002010BD00BFD5FD00080C
:1063500073B51546194A04460E46106851686B46D7
:1063600003C32CB3637CDB0624D4227C802A1DD09B
:10637000402A1FD9D208D11F501C2944C2F10F0254
:10638000304407F02BFAA8B9237CD9080D44725C7D
:1063900015F8080C03F0070302A90B44424013F858
:1063A000083C1A420CBF0120002004E0012002E05A
:1063B000204600E0002002B070BD00BF98FB00083E
:1063C0000023042A10B54370037016D0082A02D0A7
:1063D000022A26D118E00B7883F0020303704B7871
:1063E00043708B788370CB78C3700B7903714B79D2
:1063F00043718B798371CB7911E00B7883F00203C1
:1064000003704B7843700223FF240022C470FE24E3
:10641000827004714271CA5C82710B445B78C371F3
:1064200010BD184610BD00002DE9F74F1E464B6801
:1064300000920F46D3F808A0D1F808B0019018B91F
:10644000C0490320FAF7FEFB019B1B68002BF7D025
:10645000DA68272AF4D90BEB06089D6898F9013011
:10646000002B2B7803F00F0343F060032B701BF815
:10647000063003F01803ACBF02240324082B27D0F6
:1064800017D8002B52D118F804102846FFF730FF18
:1064900008EB04014B7803F00F026B7813436B7029
:1064A0008978AA78E31C0A43AA7018F803200434F8
:1064B00029E0102B2AD0182B38D100212846FFF7CD
:1064C00017FF6B7823F00F036B700023AB702CE089
:1064D00018F804309B099B0043F060032B706B7825
:1064E00003F00F01697018F8043003F00F0308EB94
:1064F00004020B436B705178AA78A31C0A43AA705C
:1065000018F803200334EB7813430EE018F8041056
:106510002846621CFFF7ECFE6B7823F00F036B70CC
:106520000023AB70EB70144600E0EB701BF80630F4
:106530005B075CBF18F80430AB711BF8063003F042
:10654000030358BF0134022B08D0032B08D0012BC2
:1065500007D018F80430EB71013403E0402300E069
:10656000FF23EB7198F8013003F0400202F0FF09BD
:1065700072B118064ABF98F802000020000913F013
:10658000300905D0FFF76EFB8146002800F031820C
:1065900098F8013003F07003302B42D00FD8102B45
:1065A0001CD0202B26D0002B40F08C8008EB04015F
:1065B000102205F1080007F043F9103482E0502B57
:1065C0003BD006D8402B7DD105F10800FFF7A4FE93
:1065D00078E0602B45D0702B62D073E005F10800A5
:1065E000FFF794FE082208EB040105F1100007F004
:1065F00027F934E005F10800FFF788FE4FF0FF327D
:106600000023EA746FF001022A752B746B74AB746B
:106610006B75022208EB040105F1160007F010F972
:106620003CE0514605F1100011F8082BFFF7C8FEB9
:1066300005F10800FFF76AFE44E0B9F1000F3FF4EE
:10664000FFAE082208EB040105F1100007F0F8F88E
:1066500099F81020494605F1080001F07FFD083443
:1066600030E0B9F1000F3FF4EBAE4FF0FF32002302
:10667000EA746FF001022A7508EB040102222B7400
:106680006B74AB746B7505F1160007F0D9F899F8C7
:106690001020494605F1080001F060FD023411E0C8
:1066A000B9F1000F3FF4CCAE514605F1100011F8DE
:1066B000082BFFF785FE99F81020494605F10800E0
:1066C00001F04CFD98F8013059070FD51A064ABF62
:1066D00098F80200002000F00F0013F00B0F05D017
:1066E000FFF7C0FA8146002800F0838198F8013056
:1066F00003F00F030C2B00F27C81DFE813F00D0098
:106700001600250042007A015100610082000D0050
:106710009400A600B800C60008EB0401102205F1A1
:10672000180007F08DF81034D9E005F11800FFF7D4
:10673000EDFD082208EB040105F1200007F080F8C8
:106740003CE000BF00F8000805F11800FFF7DEFD8F
:106750004FF0FF32002385F823206FF0010285F807
:10676000242085F8203085F8213085F8223085F8FE
:106770002530022208EB040105F1260007F060F83D
:106780003DE09AF800109AF801200831514405F1D3
:106790002000FFF715FE05F11800FFF7B7FD9EE09A
:1067A000082208EB040105F1200007F049F899F8E8
:1067B0001020494605F1180001F0D0FC08348EE0A5
:1067C0004FF0FF32002385F823206FF0010285F897
:1067D000242008EB0401022285F8203085F82130BE
:1067E00085F8223085F8253005F1260007F028F8D5
:1067F00099F81020494605F1180001F0AFFC023469
:106800006DE09AF800109AF801200831514405F122
:106810002000FFF7D5FD99F81020494605F1180032
:1068200001F09CFC5BE005F11800FFF775FDFF230C
:106830002B7618F804306B76611C0522414405F173
:10684000230006F0FDFF063449E005F11800FFF7CC
:1068500063FDFF232B7618F804306B76611C03224E
:10686000414405F1250006F0EBFF043437E005F163
:106870001800FFF751FDFF232B7602236B7618F8E3
:10688000043085F82730013429E005F1180099F823
:1068900010A0FFF741FD99F81030402B84BF402332
:1068A00089F81030FF232B7618F804306B7608EB4C
:1068B000040349465B78AB7699F81030EB7699F88B
:1068C000102005F1580001F049FC211D042241442B
:1068D00005F1240006F0B4FF063489F810A0009BEF
:1068E00013B9FB681B1B01E0009B283B5BBAAB8024
:1068F0001BF806305B077ED518F8043003F0F80368
:10690000F02B78D1019BBD68D3F800A0009BDAF88A
:106910000890344404F1010815F804B04BB900990B
:10692000042308220846FAF799FF002865D08268F8
:1069300002E009F1280200200BF00303022B14D01F
:10694000032B1FD015F808101170012B05EB040361
:106950009978517004D0D978917005341B790FE083
:10696000DB780434A3F5805318E015F80830A3F55C
:1069700080535BBA13802B19043499789170DB78BB
:10698000D3700DE015F808301909A1F5756149BA01
:1069900003F00F0302341180A3F575635BBA5380D3
:1069A0001BF0040F03D00021FBF74AF825E02B5D14
:1069B0009371A31C2C446178D17118B1F968083126
:1069C000C91A01E00099283949BA9180112189F842
:1069D00006109288A9F8042018B1019AC0F804A002
:1069E000106053B19C1B0C9B0C9A1B6808331360FE
:1069F00001E0002003E0204601E00024F3E703B0BB
:106A0000BDE8F08F2DE9F04F4268D0F80890966805
:106A1000D268002189B0824601230846FAF71EFF9A
:106A2000029038B38568AB4960232B7006F1080BE0
:106A300000236B701022584606F0D0FE38B158463D
:106A4000FFF7E6F8804610B1437CD90601D44FF039
:106A50000008337EFF2B00F0628206F11800FFF77A
:106A6000D7F80746002800F05A82437CDA0640F146
:106A7000568201E0029858E2B8F1000F04D098F86D
:106A800011301B0703D15FB17B7C1C0708D06B78EA
:106A900063F07F036B700023AB70032401E0474673
:106AA000022431683378727821F4704121F0FF01BB
:106AB0001B01A9B943EA121313F0FF0F2B7803D17E
:106AC00043F018032B7036E043F010032B707378FB
:106AD00031781B09621C43EA01132B5594B22AE05A
:106AE0005BB203F030011209114304F101010ED130
:106AF0002B7843F008032B7032688BB2317812BACE
:106B00008910C2F3034242EA81122A5509E0134375
:106B10002B55326889B212BAC2F30342A31C6A54DD
:106B20009BB2326812BA120AEA549C1C01339BB21F
:106B30000022EA54A4B2B379112B6DD1DAF80430F3
:106B4000586883681A88B3F802E052BA92B222F009
:106B50000F0C1FFA8CFC4FF2B0018C451AD19EFA33
:106B60009EF121F00F010904090C614512D10322A5
:106B7000B271598849BA1FFA81FE198849BA89B297
:106B80000EEB011101F5AA61197099795970D97943
:106B9000997026E09EFA9EFE0EF47F4EBEF5704F71
:106BA00004D10122B2715A8852BA0CE002F47F4239
:106BB000B2F5704F0ED10222B2711A8852BA1A7011
:106BC0009A785A70DA789A709A79DA70DA791A7152
:106BD000052206E00022B2719A791A71DA795A71A7
:106BE0000622B17961F00F01C2F1080EB1711A44A9
:106BF000C168C3EB020CCEEB01018C4504D212F844
:106C00000E1002F8011BF3E7FAF7B0FE2B7843F001
:106C100004032B70012303E0621C2B5594B2002364
:106C20000393F379402B07D0FF2B0AD0012B0CD113
:106C30002B7843F0010302E02B7843F002032B7022
:106C400006E02B7843F00303F9E7621C2B5594B25E
:106C500010222049584606F0C1FD18B96B7843F060
:106C6000400335E0B8F1000F0CD06B7843F04003DF
:106C70006B7098F8112010070AD0AB7843EA021322
:106C8000AB7005E05846FFF74BFB002800F0408151
:106C900008AB0020002163E9040199F80020082ACC
:106CA00000F224814FF48A71D140C90740F11E815E
:106CB00009F108011846FFF783FBDDE90423716938
:106CC0003069994208BF904206D16B7843F0300397
:106CD0006B7021E025FE000804AA59464046FFF7E4
:106CE00037FB0028F1D13369B3F17F4F05EB040086
:106CF0006B7840F00381B28A52BA92B2B2F57E4FFD
:106D000040F0FC8043F020036B70022206F1160174
:106D100006F096FD0234A4B2337EFF2B72D16B785D
:106D200043F008026A70728BCABBF269BABB328C3C
:106D3000AABB727E022A0FD1326A6AB9B28C5AB9E2
:106D400096F8262042B943F00B036B7096F8272083
:106D50002A55631C9CB2B4E0728C8AB996F8242040
:106D600072B943F00A036B70737E2B55601C0322CB
:106D700006F1250115FA80F006F062FD04349FE06B
:106D800096F82220002A40F0948043F009036B70AB
:106D9000737E2B55601C052206F123012CE0B38B7A
:106DA000ADF81030F38BADF81230338CADF81430F1
:106DB000738CADF8163004A8FEF72AFF002878D0AF
:106DC000437CDB0675D5027CF37E9A4271D16B78E9
:106DD00043F004036B70437C13F00F031EBFAA78CB
:106DE0001343AB70737E2B55631C9BB2B27EEA5487
:106DF000A01C042206F1240115FA80F006F020FD03
:106E000006345DE01FB199F801303BB951E006F15D
:106E10001800FFF785FA0028F5D14AE057B16B78E2
:106E200043F004036B707B7C13F00F031EBFAA7842
:106E30001343AB7099F8001099F8012008314944C8
:106E400004A8FFF7BDFADDE90423716A306A9942AC
:106E500008BF904204D16B7843F003036B7030E0BD
:106E600004AA06F118013846FFF772FA0028F2D199
:106E7000336AB3F17F4F05EB04006B780FD1B28C0E
:106E800052BA92B2B2F57E4F09D143F002036B7051
:106E9000022206F1260106F0D3FC023410E043F092
:106EA00001036B70082206F1200106F0C9FC0834CA
:106EB00006E02819102206F1180106F0C1FC103472
:106EC000A4B2039B1BB1631CB2792A559CB2214624
:106ED0000298FAF74BFDDAF804105046FAF770FB07
:106EE000029A43685360426001201EE00821B9F90C
:106EF000020000910022FEF735FBDEE643F01003AE
:106F00006B70082206F1100106F09AFC083402E7C3
:106F100028191022594606F093FC1034FBE6B8F10C
:106F2000000F3FF4BCAD0027A9E509B0BDE8F08F24
:106F300010B508220949044606F050FC48B12378F0
:106F4000FF2B08D1607800F00F00831E5842584193
:106F500010BD012010BD002010BD00BFD5FD0008F0
:106F600038B5B0F88E31DB07044603D40849032056
:106F7000F9F768FE00F5C47528460121FBF700FC0F
:106F8000002384F893312846BDE83840FBF728BC3D
:106F900000F80008F8B5B0F88E31DB07044603D4DA
:106FA00024490320F9F74EFE00F5C476012130464E
:106FB000FBF7E6FB94F89331022B03D8013384F8F6
:106FC000933116E0DD1EFAF77FFE0123AB403B2B29
:106FD000B0FBF3F505FB13009EBF94F8933101332A
:106FE00084F89331092804D93C2828BF3C20054661
:106FF00000E00A2504F5D4773846F9F775FD4FF41B
:107000000873A4F8BE310C490C4BC4F8C041694365
:10701000B3F9003004F5DE72384603F039FC30462F
:10702000FBF7DEFBB4F98C010021BDE8F840FDF769
:107030009FBD00BF00F8000840420F00AC340020A4
:1070400038B50446B0F91E00FCF7A6FAB0F88E3148
:10705000DA0703D411490320F9F7F4FD637F1B0716
:107060000BD4002005F0D4F9B0B9B4F91E00FCF738
:1070700093FABDE83840FFF773BF251D1022084979
:10708000284606F0ABFB0028EBD02946B4F91E00D9
:10709000BDE83840FDF76CBD38BD00BF00F8000802
:1070A00025FE00082DE9F04380468DB0184689463C
:1070B00017461E46FFF73CFF0446B8B91023069357
:1070C000029308AD07AB079003900093019606ABBF
:1070D0002A460DF116013C4804F076FD002806DB37
:1070E000069B102B0CBF2C46002400E000243146E8
:1070F000384605F041F90546002C5FD030B93146DD
:10710000BDF9160005F038F90546E0B1B5F91E00E5
:10711000FCF742FA18B1B0F88E31DB0706D56B7F69
:1071200003F03003302B08BF344600E0344644B946
:107130003046FFF7FDFE48B334460CB9002040E06E
:107140000DB1A64205D02146384605F015F9264670
:1071500005463046FFF7ECFE28B1DDB16B7F03F04A
:107160003003202B16D06B7F03F03002202AE5D0AD
:1071700003F00703032B03D104212846FDF798FCF5
:107180002A464946404605F079F91AE0FDF77CFBAE
:107190000446D2E70FB9384613E007A8FAF7C2F958
:1071A000082289F80020B118404606F049FB98F8FB
:1071B000003083F0020388F80030ECE70028B7D0F5
:1071C000A4E70DB0BDE8F0837834002070B50E461A
:1071D00018B911490320F9F735FD0029F9D0B0F9A4
:1071E0001E00FCF7D9F900F5D47504462846F9F7D6
:1071F0007BFC4FF40873A4F8BE310849084BC4F86F
:10720000C04104F5DE7271432846B3F90030BDE891
:10721000704003F03DBB00BF00F8000840420F0083
:10722000AC340020F8B507460D46164610211A4624
:107230002120FDF7F8F9044660B1806800236DBA9B
:107240000822877043710371C370C58031461044B2
:1072500006F0F6FA2046F8BD2DE9F04F85B08046DD
:107260000E9E7578022D0F4692461C4640F0B8805F
:107270000823009300226B440321FEF773F90028D2
:10728000C0F2AE804046FCF787F921468146404671
:1072900005F072F8BAF1870F04464ED0BAF1880FA4
:1072A00040F09E80B9F88E31D90740F19980DDE930
:1072B0000223D6F80CB0D6F808A05B4508BF5245AB
:1072C00040F08E80002800F08B80B578012D2ED004
:1072D0000BD3022D40F08480404607F1080105F0F1
:1072E00073F84846FFF73CFE7AE009F5C4790121BE
:1072F0004846FBF745FAF6883D4B04F13C07384613
:1073000076BAB3F90080B6B2F9F7EEFB394940F22C
:107310001223013EA4F852303846434604F150028D
:10732000714303F0B5FA4846FBF75AFA5BE007F100
:1073300018014046FCF77AFA52E0B9F88E319A0704
:107340004ED0B378002B4BD1083710222A4938464B
:1073500006F044FA002843D0D4B1637F9B060CD5D5
:10736000D4F8AC20D4F8B03052EA030105D0F1686B
:10737000B0688B4208BF824234D1B6F80690B9F1AA
:10738000000F05D13946404605F01EF84D462AE06B
:10739000F3882BB384B9032300930F9A109B3946CB
:1073A000404604F06FFF0446E8B1324600F1AC03FA
:1073B00052F8080F516803C3637F0E4823F030036F
:1073C00043F030036377F188094B49BA89B24143EE
:1073D000B3F9003004F1A40204F1900003F058FA6C
:1073E000002500E00125284605B0BDE8F08F00BF6C
:1073F000AC3400200087930325FE000813B58A787B
:107400004B78402A01D8022B00E0032B0ED18628AE
:107410000ED1C878CB88C0F300145BBA00949BB23D
:10742000083100F00F00FEF73DFC01E0002000E015
:10743000012002B010BD000008B50146074800F069
:1074400052FE48B910220649044806F0C7F9002840
:10745000024818BF002008BD004808BDF4450020C0
:1074600025FE00082DE9F047154D002680468A4686
:1074700017463446A9465146A86800F049FEB8426E
:107480000BD3AB685B7C9F4207D16B68434504D14B
:107490000C2000FB0690BDE8F0874CB9A86808B93D
:1074A0002C4605E01022074906F098F90028F7D08D
:1074B0000136022E05F10C05DDD12046BDE8F0872E
:1074C0002C46002025FE000838B5044619B30123D8
:1074D00080221749B0F98C01FCF780F9D8B104F586
:1074E000C47528460121FBF74BF9B4F88E3143F0FF
:1074F0000403A4F88E314FF4E163A4F89A314FF4F9
:107500001673A4F89631C823A4F898312846BDE82C
:107510003840FBF765B9B4F88E31B4F98C010449F1
:1075200023F00403A4F88E31BDE83840FCF77EB99F
:1075300005FE000808B510220449054806F04EF97A
:107540000028034808BF002008BD00BF25FE000832
:10755000F44500202DE9F0470024054600F1160708
:107560004FF00109A2464FEAD40804F0070617F8C5
:10757000083009FA06F633420AD0E0B2FEF772FB91
:1075800080F810A017F8083023EA060607F808600C
:107590000134102CE7D10026AC695CB12368AB61E3
:1075A0006368A168B3F98C01FCF740F92660666056
:1075B000A660F1E710222146284606F03FFA2C612A
:1075C000BDE8F0872DE9F04F87B003F1080901917C
:1075D0008346494605A890461E46FCF76BF90746C8
:1075E000002840F0A0804846FFF726FF0446002808
:1075F00000F09980F3885BBA9AB21AB942F210731C
:10760000838290E0838200F11603A8F110080293B0
:10761000B8F1000F57DD07F11003019AD518D35CBC
:10762000032B02D0222B32D046E05846FBF7B4FFA2
:107630006B780090042B2AD105F1100A08223B49EF
:10764000504606F0CBF810B32B7CFF2B04D16B7C9B
:1076500003F00F03022B1AD0EB785A0617D41B063F
:1076600015D46B689BB151465846FCF78DF9AA7842
:10767000039051460098FFF7F5FE40B14268039B26
:107680002AB9009A42608360A3690360A061AB7865
:107690003F2B6B7801D8022B00E0032B0CD1EB7849
:1076A0000121C3F3C00203F0070301FA03F30299B7
:1076B000895C0B4302998B546B7807EBC307BFB20D
:1076C000A8EBC308A4E773885BBA9BB22361B288B6
:1076D00052BA43EA02432361D9F80000D9F80410F2
:1076E000234603C356F8100F7168022203C300211A
:1076F00004F1160006F0A2F90023A361A58A0C4B41
:1077000004F11C0630465D43F9F7EEF940F22323FD
:107710006386084B6463B3F9003004F130022946F4
:10772000304603F0B5F807B0BDE8F08FD5FD00088E
:1077300000879303AC3400202DE9F0418846C1084E
:10774000064614460831069A22201F46FCF76BFFB6
:107750000546A0B18068002164BA01714171C480FE
:10776000867080F80380EA6800F10804083A204631
:1077700006F064F932463946204600F0EFFC284610
:10778000BDE8F08170B505460E46144618211A462C
:107790002320FCF748FF80B183686ABA2D0C6DBACC
:1077A00076BA5A809D80DE8022689A606268DA60CC
:1077B00054F8082F1A6162685A6170BDF8B50F4617
:1077C000054618B90D490320F9F73CFAFFF734FED6
:1077D000044688B1002606618782696803462868E6
:1077E00003C355F8080F6968022203C3314604F148
:1077F000160006F023F9A6612046F8BD00F800083F
:1078000070B5044615460E4601B11AB91149032058
:10781000F9F718FA104B984214D33833984211D81C
:10782000527C29463046FFF71DFE70B143687BB994
:10783000A26902602269466001328560A06122610E
:10784000184670BD6FF0010070BD6FF00B0070BD89
:10785000002070BD00F80008F445002010B501B10B
:107860001AB910490320F9F7EDF90F4B984218D3D4
:107870003833984215D88369002193B19C68A2429D
:107880001C680BD109B9846100E00C6000221A6009
:107890005A609A6003690133036110BD194623469B
:1078A000EBE710BD00F80008F4450020124B9842A9
:1078B00030B517D33833984214D80F2915D8CC08CF
:1078C00000F1160501232A5D01F0070103FA01F119
:1078D00012EA01030CD111432955026901320261F8
:1078E000184630BD6FF0010030BD6FF0150030BD9F
:1078F0006FF06F0030BD00BFF44500200C4B984284
:1079000010B513D33833984210D80F290ED8CA08AF
:1079100000F11604012301F0070103FA01F1A35C51
:1079200023EA0101A15403690133036110BD00BFC3
:10793000F44500200C4AB2F90030984210B512D03C
:10794000B2F90640002B0CBF13460023A0420AD018
:1079500024B90632002B08BF134600E01BB10122F8
:10796000188059801A7110BD44460020084AB2F9A7
:107970000030834205D0B2F90630834206D101239C
:1079800000E00023062000FB032070470020704722
:10799000444600200021FAF753B8F8B50746848919
:1079A0000E46154600204DB900230822B96800F0A4
:1079B00073FB96F91030022B25D10DE0BD42F3D0B8
:1079C000B542F1D02346AA89A96800F065FBEB68AF
:1079D0006D681C44A4B2E6E702194FF6EE739A42B2
:1079E000C4BF013080B2B16811342044002320228A
:1079F000083180B200F050FB4FF6FF73984203D07D
:107A0000C04380B2F8BD0020F8BD000070B5102260
:107A100098B000210DEB020006F010F84D4B0593D5
:107A20004D4B1B88ADF81C3040F20523ADF80A30F1
:107A300008216FF0850308A80393FBF7BDF804A99C
:107A40000420FDF70FFF6846FBF7B3F8BDF80230DE
:107A50006FF400721344032BF5D8DFE803F0023B08
:107A60007575019D2846F9F7F9FF044608B92846BF
:107A700067E00221FDF76FFF064618B9374903207A
:107A8000F9F7E0F8606830B190F91030042B02D1BA
:107A9000C368082B06D0042208212046F9F7F8FE17
:107AA00000284DD0002385682374EB885BBA9BB215
:107AB000002B45D022463146FFF76FFF4FF6FF738C
:107AC00098423DD1698849BA234640F2012289B2E1
:107AD000042031E0019E304696F91050F9F7BEFFC0
:107AE000044608B930462CE0406826460028C5D038
:107AF00090F91030042B07D0F9F7B0FF0346F8B126
:107B0000706040681E46F1E7F9F7A8FFC0B18268CF
:107B100070600023C16840680B440028FAD15BBA4A
:107B200093806B1C08BF63680A4908BF93F9105023
:107B300040F2022223462846FDF7C0FC002882D1ED
:107B40002046FFF727FF7EE702A96846FBF700F80B
:107B500079E700BF0000FFFF9C02002000F800084A
:107B600010B5044668B161B190F91030042B0BD107
:107B70004268FFF712FF50B1A36840BAD8800020D6
:107B800010BD6FF00D0010BD6FF04C0010BD6FF018
:107B9000010010BD38B50D4614460423082200210B
:107BA000F9F75CFE38B1836800226DBA64BA1D80B3
:107BB0005C809A71DA7138BD1FB50A4CB4F9003097
:107BC00063B9094A0193094B0292009305220823E5
:107BD0004FF480610648F9F7D5F82080B4F9000029
:107BE00004B010BD504A0020A0FB00080D7A000828
:107BF0005046002008B504210448FAF7DDFF044B85
:107C0000B3F9000002F01CFD002008BD5450002014
:107C1000525000207FB52D4D0446B5F9000008B93B
:107C20002B4820E02B4BB3F90020BDF920309A42BD
:107C300001D0294817E0082600960DEB0603002224
:107C40003146FDF78FFC00280CDB0DEB06013246B8
:107C5000A01905F0F5FD2146204800F044FA28B1AE
:107C60001F4800E01F4805F0F1FF2DE040231A46B1
:107C70002146B5F90000FBF7B1FD1849B5F9000040
:107C8000FBF7D4FD184804F05AF9204600F092FAA8
:107C9000164806F065F810221549104805F09EFDBB
:107CA00068B10E49B5F90000FBF7C0FD114804F0BA
:107CB00046F90A4800F07EFA0C4806F051F8102206
:107CC0002146064805F0BCFD04B070BD745000208C
:107CD000A4FB000852500020FEFB00087650002054
:107CE00093FC00084BFC0008CCFC000805FD0008D4
:107CF00025FE000809FD00082DE9F04F93B00DF1B5
:107D0000240B5846F9F70EFCDFF80881DFF8DC9009
:107D100007900024079BDFF8FCA0A3420CD1334C52
:107D2000BAF90010B4F90020314805F08FFFBAF914
:107D30000030002B43D145E0022CF0D03BF9145029
:107D4000002300931A4624212846FDF70BFCB8F9BE
:107D5000006026BB012822D10AAF2649A8F80050AE
:107D6000384600F0F1FA3346402239462846FBF700
:107D700035FD21490EA800F0E7FA2049384600F009
:107D8000E3FA4FF0FF3304931023039602938DE838
:107D9000C0000EAA29461A4803F054FE06E0B9F9BD
:107DA00000301BB9012818BFA9F80050B8F90030FD
:107DB0001BB1B9F90030002BB1D10134AAE7B4F9F5
:107DC00000301BB90F4805F041FF0CE00E4B029349
:107DD000002301930D4B0093062208234FF4C0614A
:107DE0000B48F8F7CFFF13B0BDE8F08F74500020B8
:107DF0004FFD00083FFD0008671D010847FD000812
:107E00007834002097FD0008CEFD0008F57B0008BF
:107E1000524A002052500020F8B504469DF82450E4
:107E200025701E4605F0070310250F46657006985D
:107E30009DF8281015460AB1002F68D018B1002E01
:107E400069D13046F8BD23B1022B02D00DB900280C
:107E500073D0A17080B39DF82030E37002289DF8A4
:107E60002130237104D0082816D0002851D120E0F9
:107E700002463249304605F0B1FC18B9237823F0A8
:107E800020032370637843F0080363707378637191
:107E90003378A371072040E01C236370221D06F194
:107EA000080313F8011D02F8011F9E42F9D10D20AD
:107EB00033E005201DB9F8BD0320002D3DD0431C43
:107EC0009DF81C2022549DF81D20E2540230022D02
:107ED00003D0082D0CD0E5B9F8BD637863F07F03BB
:107EE00063707A782254431C3A78E2540230F8BD29
:107EF000637863F03F03637007F10803044413F8E9
:107F0000012D04F8012BBB42F9D10830F8BD3846E9
:107F1000F8BD0020F8BD63B90DE075B1BDF81C20B7
:107F2000BDF820309A42CAD1237843F04003237031
:107F3000CDE7022B8AD1A1708DE7F8BDD3FD0008F3
:107F4000427802F00C03082B07D00C2B07D0CBB9DA
:107F50000178490614D4032302E0072300E00D232F
:107F600012F0C0020CD00178490658BF0233802AB3
:107F700001D1981C7047C02A04D103F10800704752
:107F8000184670470020704770B501B11AB92649EC
:107F90000320F8F757FE437803F00C03082B07D1B2
:107FA00003785C0617D5C37813700379537012E019
:107FB0000C2B07D103785B060FD5C37813700379B8
:107FC00053700AE013B16FF0150070BD03785E06C0
:107FD000F9D4032302E0072300E00D23447814F0D2
:107FE000C00411D005786D0605D4C65C16705D1C02
:107FF0000233455D5570802C08D1C25C4A70034441
:1080000002205B780B7070BD204670BDC02CDAD1A9
:10801000034401F1080213F8010B02F8010D8A4232
:10802000F9D1082070BD00BF00F8000808B501B103
:108030001AB918490320F8F705FE437803F00C033A
:10804000082B09D1C37813700379537043794B70AF
:1080500083790B70022008BD0C2B0ED1C3781370EE
:1080600010F8043F537001F1080310F8012F03F8D2
:10807000012D8B42F9D1082008BD3BB9037813F0DC
:10808000400F14BF6FF01500002008BD6FF0150001
:1080900008BD00BF00F80008F0B51AB3DC0705D52D
:1080A00011F8014B013A204492B20133570801EB19
:1080B00047054C1C03350234AC4207D014F803ECDE
:1080C00014F8026C06EB0E263044F4E71A44D3078A
:1080D00003D511F8173000EB0320030C80B201D058
:1080E0001844FAE7F0BD30B54B68456804680A6883
:1080F0009D4208BF944209D1C568CB6884688A68EC
:108100009D4206BF94420120002030BD002030BDBA
:1081100030B510B3E1B188421CD0013801390022DA
:1081200010F8015F11F8014FA54202F1080303D1D5
:10813000DAB2802AF4D10FE085EA0401D8B20B0646
:108140000AD40132D2B249008242C9B2F7D130BD5D
:10815000084630BD802030BD104630BD802A28BF83
:108160008022F8B5D50814462A4606460F4605F083
:1081700067FB63070ED0A4EBC504725DFF23C4F157
:10818000080403FA04F422EA040272557B5D1C40E1
:1081900014437455F8BD10F8013F43B18B42FAD136
:1081A00000230370437813B1013005F09FB81046E7
:1081B0007047000000B501468BB018B9064903208E
:1081C000F8F740FD2822684600F008F8684603F0FA
:1081D000B6FE0BB05DF804FB00F800082DE9F0478F
:1081E00007468AB008B90020A8E00029FBD000208B
:1081F0004FF0FF3406462346054631F810E0BEF145
:10820000000F07D1B3F1FF3F13BF013503B20125C2
:108210002DB20BE0B3F1FF3F08D0B4F1FF3F01D026
:10822000B54201DD2E461C464FF0FF3301300828D1
:10823000E3D1581C04D0601C7DD0B54202DD7AE049
:10824000601C03D0012ED8BF4FF0FF343D480025FD
:108250006B46E8464FF03A09AC4203D183F80090F0
:10826000A5194EE015B183F80090013311F815E01F
:108270001EF0F00F4FEA450C17D04FEA1E1A0EF011
:108280000F0E10F80AA010F80EE083F801E001EBE1
:108290000C0E83F800A09EF801E04FEA1E1E033387
:1082A00010F80EE003F801EC21E0BEF1000F10D051
:1082B00010F80EA09E460EF802AB01EB0C0A9AF8DD
:1082C00001A04FEA1A1A10F80AA083F801A0734619
:1082D0000DE001EB0C0E9EF801E01EF0F00F1FBF49
:1082E0004FEA1E1E10F80EE083F800E001338C44C4
:1082F00001359CF801E00EF00F0E10F80EE083F847
:1083000000E0072D03F10103A6DD611C05D0344414
:10831000082C02BF3A2119700133002103F8011B18
:10832000C8EB030393423FF65EAF4146384605F083
:1083300075FF384602E02E461C4683E70AB0BDE8CA
:10834000F08700BF45FE00082DE9F0470F460546BF
:1083500010B90020BDE8F0870029FAD010220021D2
:1083600005F06CFB3B783A2B04D00024A14626464E
:10837000A04619E07A783A2A07F10103E9D11F46AD
:10838000F3E751462B4805F071FD98B951462A484C
:1083900005F06CFD80B1284BC01A40EA0616B6F510
:1083A000803FD6D24FF0010917F801ABBAF1000FA8
:1083B000E7D119E01F4BEFE7BAF13A0FC9D1B9F194
:1083C000000F05D1B8F1000FC3D105EB0408EBE7AE
:1083D000A21C102ABDD8631CDBB2310A2955814684
:1083E000EE54D4B20646DFE7B9F1000F08D0A21C64
:1083F000102AAED8631CDBB2310A2955EE54D4B230
:10840000B8F1000F10D02C44C8EB040805F110029D
:1084100001230021434504F1FF3407DC207802F8F2
:10842000010D01332170F5E7102C92D12846BDE8EB
:10843000F08700BF45FE000856FE00080C4B0146C1
:10844000186882689368013B002B10B4936005DACA
:108450009469A34208DBCBB20A2B05D01368581CE1
:108460001060197010BC704710BC06F03FB900BF17
:108470002802002008B53E20FFF7E0FF2020FFF78C
:10848000DDFF034B1B689868BDE8084005F006B89F
:10849000280200202DE9804885B0814600AF0E46B5
:1084A0009246FFF7E7FFB0460AF1FF340025C6EB1E
:1084B0000803A342F5DA844B186841684B68013B16
:1084C000002B4B6004DA05F053FC002804DAE8E7DF
:1084D0000B685A1C0A6018780D2801D00A280FD1A1
:1084E00000240D2088F80040FFF7A8FF0A20FFF7BE
:1084F000A5FF4645D5D033462246254620462BE0EB
:10850000082801D07F280DD14645D0D0082008F892
:10851000015CFFF793FF2020FFF790FF08F1FF3B7E
:10852000082003E008F1010B88F80000FFF786FF40
:10853000D846BCE7222913D15C781CB35C2C25D02B
:1085400001331C788C42F7D1597820291AD801358B
:10855000197811B303F8010B19782029F8D9E9E744
:10856000272906D1E8E74B1C497822290AD020297F
:10857000EDD91C785C2C1946F5D1591C5B78013279
:10858000002BF0D1514805F0EBFB8AE79C1C9B784F
:108590000132002BF6D02346D3E7002D81D0AB006B
:1085A0000E3323F00703EB46ADEB030D6C464DF89D
:1085B0002510304690F800E003460130BEF1000F70
:1085C000F8D0BEF1220F02D0BEF1270F00D1013347
:1085D00044F821301846013390F800E0BEF1000F56
:1085E000F8D101318D42E5D1201FBAB150F8043FD6
:1085F000A3B1194613F801EBBEF1000FF5D0BEF19F
:108600005C0FF6D191F800E0BEF1000F04D091F8B4
:1086100001E001F801EBF5E7013AEAD12C4B2268C1
:10862000FB60C7F80890002307F1080151F8238088
:10863000B8F1000F0DD10133022B16D0F4E711462B
:108640003B607A6005F080FC7A683B6830B108F1E5
:108650000C08D8F800000028F1D1ECE7D8F8083071
:108660001BB12146284698472CE02168194805F09F
:108670006BFC054610BB184A1849194805F0E6FA84
:10868000184805F06DFB124BC7F80890FB602C46AC
:1086900007F1080353F824500DB10C3503E0013401
:1086A000022CF5D10EE00C3555F8181C0029F6D037
:1086B00055F8142C0A4805F0C9FAF4E721680A486D
:1086C00005F0C4FADD46ECE62802002067FE00084B
:1086D0003800010880FE000885FE000891FE0008B1
:1086E00099FE00083F160108A3FE000808B503F034
:1086F00051F8002008BD08B5F9F76EFA002008BD52
:10870000012810B506D10020F9F700FF0446014604
:10871000074805E0486804F0E9FD044601460548BD
:1087200005F094FA2046F9F7C9FA002010BD00BF01
:10873000BC000108E200010808B5F9F7C5FA0146D6
:10874000024805F083FA002008BD00BF8B1F010816
:108750000146062814D8DFE800F004060B0D0F11BF
:108760000900094800E0094805F070BA0848FBE72D
:108770000848F9E70848F7E70848F5E70848F3E745
:10878000084805F063BA00BF0401010808010108A8
:108790000E010108160101081B0101081E01010854
:1087A0002101010827010108102828D00BD803282F
:1087B0001BD003D8E8B1022815D07047052816D081
:1087C00006281AD07047262815D004D8162818D0A5
:1087D000202818D070472A2817D02B2817D02728F0
:1087E00018D10D4814E00D4812E00D4810E00D4876
:1087F0000EE00D480CE00D480AE00D4808E00D4879
:1088000006E00D4804E00D4802E00D4800E00D4888
:1088100005F01CBA704700BFB30101082C01010824
:108820003C010108490101085F01010867010108D5
:108830006C0101087F01010891010108A6010108EE
:10884000CA010108D501010808B50146034805F031
:10885000FDF90348BDE8084005F082BAE4010108CB
:108860000902010813B5044601A8F8F75BFE70B1D0
:10887000BDF90430A34207D0012807D9BDF906008D
:10888000031B5842584102E0012000E0002002B0E2
:1088900010BD00002DE9F04790B002AF002605465C
:1088A000FE70FAF779FE29460446CB4805F0CEF96A
:1088B000082300933246FB1802212846FCF752FE9B
:1088C000061E1CDB06EB460808F1070323F007032E
:1088D000E946ADEB030D0DF1080AC04805F0B6F905
:1088E000334607F108024146504603F0E5FD0146D4
:1088F000BB4805F0ABF9BB4805F0A8F9CD4602230B
:108900000022009311463B1D2846FCF72BFE002851
:1089100003DBB988B44805F099F9022300930022DB
:108920003B1D26212846FCF71DFE002803DBB988E5
:10893000AE4805F08BF90223009300223B1D06216F
:108940002846FCF70FFE002803DBB988A84805F08D
:108950007DF9A84805F07AF9082300930022FB1856
:1089600003212846FCF7FEFD061E1EDB06EB46082B
:1089700008F1070323F00703E946ADEB030D0DF102
:10898000080A9D4805F062F9334607F1080241469E
:10899000504603F091FD0146984805F057F9984874
:1089A000CD4605F053F9012600E00026022300938E
:1089B0000022BB1D10212846FCF7D4FD002804DB53
:1089C000B7F906108F4805F041F901230093002202
:1089D000BB1C18212846FCF7C5FD002808DB8A4887
:1089E00005F034F9B878FFF7B3FE7E4805F02EF9AC
:1089F000012300930022FB1816212846FCF7B2FD44
:108A0000002803DB7978814805F020F94FF0010850
:108A1000CDF8008007EB0803002220212846FCF750
:108A2000A1FD002810DBCDF80080FB1C00221F21D7
:108A30002846FCF797FD002806DBFB78434503D169
:108A40007978734805F002F96A4805F0FFF80123C8
:108A500000930022FB1C13212846FCF783FD00280D
:108A600008DB97F80380B8F1010F03D1694805F0DE
:108A7000EDF84646012300930022FB1C14212846F2
:108A8000FCF770FD002808DB97F80380B8F1010FB0
:108A900003D1614805F0DAF846460123009300222D
:108AA000FB1C15212846FCF75DFD002808DB97F824
:108AB0000380B8F1010F03D1584805F0C7F84646C6
:108AC000012300930022FB1C12212846FCF74AFDDB
:108AD000002808DB97F80380B8F1010F03D1504854
:108AE00005F0B4F84646012300930022FB1C19212F
:108AF0002846FCF737FD002808DB97F80380B8F11B
:108B0000010F03D1474805F0A1F846460123009321
:108B10000022FB1C1F212846FCF724FD002808DB4F
:108B200097F80380B8F1010F03D13F4805F08EF8A4
:108B30004646012300930022FB1C1E212846FCF719
:108B400011FD002808DB97F80380B8F1010F03D16D
:108B5000364805F07BF84646012300930022FB1CB3
:108B600023212846FCF7FEFC002808DB97F8038049
:108B7000B8F1010F03D12E4805F068F84646FCB164
:108B8000B4F890112B4805F061F894F892112A4836
:108B900005F05CF8B4F88E31D80702D5274805F007
:108BA00055F8B4F88E31990702D5254805F04EF8EE
:108BB000B4F88E315A0702D5224805F047F801264D
:108BC0002846FEF7D3FE002840D00379002B3DD085
:108BD0001D4805F03BF83AE0A3050108DA05010855
:108BE000EA060108F2050108AF050108BE05010803
:108BF000CA050108D2060108D6050108E4050108E6
:108C0000E8050108F4050108070601081006010837
:108C10002406010837060108410601084B06010831
:108C2000550601085F06010869060108700601087B
:108C30007A06010889060108930601089B060108C7
:108C4000A1060108A7060108B106010816B13348BC
:108C500004F0FCFF0223009300223B1D052128465F
:108C6000FCF780FC002803DBB9882D4804F0EEFFF8
:108C7000002C4BD0B4F88E312A492B4813F0800FCA
:108C80002A4B08BF194604F0E1FF244804F0DEFF38
:108C900004F5C47510222649204604F09FFD0028E3
:108CA00031D0244804F0D2FF2822214607F11000D9
:108CB000FFF794FA08B3627C1F4807F1100104F033
:108CC000C5FF08221D49204604F088FD38B12378ED
:108CD000FF2B06D1637803F00F03022B01D1184854
:108CE00000E0184804F0B2FF237CDB0708D52378A6
:108CF000FF2B0CBF1448154800E0154804F0A6FFF0
:108D0000064804F0A3FF3834AC42C3D1114805F043
:108D100027F83837BD46BDE8F08700BFD206010806
:108D2000B806010894050108DF0601089A05010844
:108D300025FE0008ED060108FA060108D5FD000829
:108D4000090701080F070108160701082307010892
:108D50002E0701083FF800081FB504AB012403F8F3
:108D6000012D00940022FCF723FC002804DA0948B6
:108D700004F0F6FF20460BE09DF80F10064B074A63
:108D80000748002914BF1146194604F05FFF002070
:108D900004B010BD45070108420701083FF800086C
:108DA00061070108A0F13003DAB2092A04D9A0F161
:108DB0006103DAB2052A01D8184670474138C3B2B8
:108DC000052B88BF4FF0FF30704700007FB50C4681
:108DD000082105460DEB0100164603F099FB08B982
:108DE00011480FE0009002AB002221462846FCF714
:108DF000DFFB00280ADA0D4804F028FF2046FFF7C1
:108E0000D3FC0B4804F0ACFF01200BE0094804F050
:108E10001DFF2046FFF7C8FC32462946064804F0ED
:108E200015FF002004B070BD78070108EB070108AA
:108E30003FF80008010801080F0801087FB5064641
:108E400010460D4604F052FA04AB012403F8010D5C
:108E50000022009429463046FCF7AAFB00280ADAD3
:108E60000C4804F0F3FE2846FFF79EFC0A4804F085
:108E700077FF20460CE0094804F0E8FE2846FFF79B
:108E800093FC9DF80F200648314604F0DFFE0020D9
:108E900004B070BDEB0701083FF8000801080108A5
:108EA000280801087FB506460D461046531E13F8E4
:108EB000014F1CB1303C092CF9D908E00A222146A7
:108EC00005F0FCFB0390013009D11C481CE0102286
:108ED000002105F0F3FB03900130F6D00124039B41
:108EE000B3F5803FF1D202230093002203AB294661
:108EF0003046FCF75DFB00280ADA114804F0A6FEB4
:108F00002846FFF751FC0F4804F02AFF012012E029
:108F10000D4804F09BFE2846FFF746FC31460B48FF
:108F200004F094FE039924B1094804F08FFE002058
:108F300001E00848F9E704B070BD00BF410801082E
:108F4000EB0701083FF80008010801088F08010835
:108F5000A5080108321E01082DE9F04F012889B04B
:108F6000814602AF0E4612DC07F10800F8F7DAFA84
:108F7000044648B1B7F90800FFF78CFC012C03D96F
:108F8000B7F90A00FFF786FC002400F00DBC486822
:108F9000431E13F8018FB8F1000F21D0A8F130085B
:108FA000B8F1090FF5D93168A34804F04FFE3068D5
:108FB000FFF74AFC3168A14804F048FE3168A04838
:108FC00004F044FE31689F4804F040FE31689E483A
:108FD00004F03CFE31689D4804F038FE0124E3E3D0
:108FE00004F084F905B22846FFF73CFC002800F0A5
:108FF000D783B9F1020F01D12846C3E79449B0687D
:1090000004F0A2FF002840F02082B9F1040F01DC37
:10901000306817E2D6F80C808E48D6F80090366992
:10902000414604F091FF10B9324602210CE041465E
:10903000894804F089FF0028F6D04146874804F0AB
:1090400083FF28B9324603212846FFF7BFFE71E3AC
:109050004146834804F078FF10B93246002151E0C0
:109060004146804804F070FF0028F6D041467E4813
:1090700004F06AFF10B93246262143E041467B489E
:1090800004F062FF10B9324606213BE041467848C1
:1090900004F05AFF0028F6D04146764804F054FF09
:1090A0000028F0D04146744804F04EFF044610BB3F
:1090B000304604F01BF907F11803022223F8100DC3
:1090C0001021009228462246FCF772FA002807DA9F
:1090D0006A4804F0BBFD6A4804F0B8FD694860E3E3
:1090E000694804F0B3FD664804F0B0FDB7F9082004
:1090F00066482946CCE24146654804F025FF28B978
:10910000324605212846FFF7CDFE13E3414661486C
:1091100004F01AFF0446002863D131465E4804F08B
:1091200013FF08B9002332E031465C4804F00CFF1D
:109130000028F7D031465A4804F006FF08B9012349
:1091400025E03146574804F0FFFE0028F7D03146AD
:10915000554804F0F9FE08B9022318E03146534897
:1091600004F0F2FE0028F7D03146514804F0ECFE3E
:1091700008B905230BE031464E4804F0E5FE00280F
:10918000F7D031464C4804F0DFFEB8B9062301267B
:109190003B720022009607F1080318212846FCF7CD
:1091A00007FA002812DA454804F050FD387AFFF734
:1091B000CFFA344804F0D4FD3446F5E23146404855
:1091C00004F0C2FE0028E1D03E48EAE229463E48CB
:1091D00004F03CFD387AFFF7BBFA2A4804F0C0FDE2
:1091E000E2E24146394804F0AFFE10B9324616219A
:1091F0000EE04146364804F0A7FE10B93246202161
:1092000006E04146334804F09FFE28B93246272144
:109210002846FFF713FE8DE241462F4804F094FEE6
:109220000446002840F0938031462C4804F08CFE20
:10923000002855D101235FE0B30F0108D50C0108C8
:10924000580D0108460F0108830B0108880C01081E
:109250008A090108480901084D090108580901084F
:109260005F01010862090108670101086709010837
:109270006B0901086F09010876090108EB0701086D
:109280007F0101083FF800080108010828080108CB
:109290007C090108FCF800088409010804010108A0
:1092A000210E01080801010880F8000816010108D4
:1092B00088090108210101088E090108D709010860
:1092C0000E01010896090108F60901081E0A0108A5
:1092D000260A0108330A0108410A01083F0701086C
:1092E0003146B24804F030FE0028A3D03146B048E1
:1092F00004F02AFEC8B900234FF001083B72002297
:10930000CDF8008007F108032A212846FCF750F920
:10931000002812DAA74804F099FCA74804F096FC4C
:10932000A64804F01DFD44463EE23146A44804F040
:109330000BFE0028DFD0A34833E2A34804F086FCEC
:109340009D4804F083FC32462946A048A0E14146EE
:109350009F4804F0F9FD0446002872D1304604F01D
:10936000CFFF4FEA500909F1070323F00703EA464C
:109370000E28ADEB030D83460DF1080801D1954889
:1093800006E0102801D1944802E0202804D1934837
:1093900004F05CFC002117E0302801D19048F7E789
:1093A000402801D18F48F3E7802801D18E48EFE7AC
:1093B0008E4804F04BFC17E0421C12D04A0800EB28
:1093C000031008F8020002318B450FD9705CFFF7DB
:1093D000E9FC721878605078FFF7E4FC7B685A1C4F
:1093E000EAD1834804F0BCFC012428E0CDF80090C9
:1093F000434600222B212846FCF7DAF8002807DA3A
:109400006C4804F023FC7B4804F020FC6B48E9E73F
:109410006D4804F01BFC774804F018FC2946764898
:1094200004F014FC4546C144A94505D015F8011BBC
:10943000724804F00BFCF7E7604804F091FCD54655
:10944000B2E14846FFF700FAC8E56D49B06804F09C
:109450007BFD044600286AD1B9F1030F01D13168C0
:1094600027E0A9F10309B9F1010FD6F80C8022D049
:109470006449D6F800A0404604F066FD20B9D6F84D
:1094800010804FF0020A17E05F49F06804F05CFDBD
:1094900020B9D6F810804FF0010A0DE05B49F06862
:1094A00004F052FD20B9D6F810804FF0000A03E016
:1094B0005146574890E582462F2140224046FEF70C
:1094C0006AFE431E802B0646414628BF402607F110
:1094D00008005FFA86FBFEF737FF002838D0B9F1A5
:1094E000010F07D03B7AFF2B04D1BAF1010F07D04F
:1094F000484856E1BAF1020F14BF4023412300E06F
:1095000040235A4607F108012846FAF767F918B9C7
:10951000414804F09BFB61E54FF0FF3343618361F9
:1095200032462B4641463D4804F090FB3CE13C4925
:10953000B06804F009FD0446A8B9B9F1030F3FF47F
:1095400049ADF66807F108003146FEF7FDFE08B99F
:10955000344826E107F108012846FAF767F92A4658
:109560003146314894E03149B06804F0EDFC0446DE
:10957000002869D1B9F1030F02D131682C482BE5DD
:10958000F06803F0B3FEA0F5A063B3F57B4F064689
:1095900005D34FF6FF724FF4A06126486AE02846D3
:1095A000F9F7FAFF002849D12348FAE0490A0108EF
:1095B00084090108EB070108CA0101083FF8000807
:1095C000040101084C0A0108010801080F080108FC
:1095D0005F0B01087C0A0108990A0108B60A010814
:1095E000D40A0108F20A0108100B01082E0B010829
:1095F000480B0108D5010108630B01087A0B01082B
:109600007F0B0108CF0B0108D70B0108E10B010804
:10961000830B01080E0C01083A0C01085D0C0108CF
:10962000840C0108E90B0108AB0C0108D10C0108FE
:10963000D50C0108F00C0108180D0108A0F8906184
:109640002A4631465B4823E05B49B06804F07CFC65
:10965000044600BBB9F1030F02D131685748BBE49F
:10966000F06803F043FEFF28064606D954484FF63B
:10967000FF72002104F0EAFAB0E42846F9F78CFF03
:1096800008B950488DE080F892614F482A4631462B
:1096900004F0DCFA88E0D6F808904C4999F80030DC
:1096A000D6F800A02D2B08BF09F1010948460CBFD0
:1096B0004646012604F048FC10B93246132136E034
:1096C0004349484604F040FC10B9324612212EE0CE
:1096D0004049484604F038FC10B93246142126E0CF
:1096E0003D49484604F030FC10B9324615211EE0D1
:1096F0003A49484604F028FC10B93246192116E0D0
:109700003749484604F020FC10B932461F210EE0CC
:109710003449484604F018FC10B932461E2106E0D0
:109720003149484604F010FC30B93246232128461E
:10973000FFF712FB044637E02C49484604F004FCCE
:10974000044678B92846FEF711F908B9284828E0F8
:1097500026B101230371294626481BE006712946DC
:10976000254817E02549484604F0EEFB0446A0B919
:109770002846F9F711FF08B9214812E02EB101215E
:10978000F9F734FF29461F4804E03146F9F72EFF68
:109790001D48294604F05AFA06E051461B481BE4CE
:1097A0001B4804F0DDFA19E420461C37BD46BDE82D
:1097B000F08F00BF320D0108550D0108580D01084A
:1097C000720D0108A00D0108C00D0108E90D010886
:1097D000F10D0108F90D0108010E0108090E01083B
:1097E0000D0E0108120E01081A0E0108270E0108BD
:1097F0002C0E01084A0E0108710E0108990E01088D
:10980000A10E0108D50E01080D0F0108460F010831
:10981000D60801082DE9F04F87B006AF0546884607
:1098200091469A4604F06CFD28448542A0EB05045D
:1098300013D010F801392F2B05D1601C284403F0F8
:1098400055FD06460BE03A2B01D02E2BEDD12846D4
:1098500004F056FD0026044601E00024264604F1EB
:10986000080323F00703ADEB030D0DF1180B621C89
:109870000021584604F0E2F829462246584603F0F3
:10988000DFFF404604F03CFD59461648FEF75CFDFC
:10989000D0B1144D102441461348FEF755FDD0B108
:1098A000114B102200213606039102920193CDF84C
:1098B00010A0009623462A4649460C4802F0C2F8FA
:1098C0000437BD46BDE8F08F03F018FD6A2303603E
:1098D000074D0424DFE703F011FD6A23036004222F
:1098E000044BDFE79650002086500020783400209B
:1098F000AA500020A650002001282DE9F34105467A
:109900000C4603D17A4802F0FDF9BBE002281AD1D7
:109910004968784804F018FB002800F0B1806168BD
:10992000754804F011FB08B97448B8E061687448E0
:1099300004F00AFB014620B96D4802F029F971488C
:10994000ADE07148ABE053DD49686A4804F0FCFAC9
:1099500058B16168684804F0F7FA30B16168684846
:1099600004F0F2FA08B1694899E0032D25D1616845
:10997000634804F0E9FA054690B9A06803F0B6FC24
:1099800004B22046F7F7E0FD214628B1584802F01E
:10999000FFF821465E4800E05E4804F057F9A2E077
:1099A000A1685D48FEF7D0FC054600286CD0102267
:1099B00059494F4802F0CEF864E0052D18D161688E
:1099C0004C4804F0C1FA002868D1E168534804F01B
:1099D000BBFA0546002861D101A8F7F7A3FD0128CD
:1099E00031D14FF0FF33BDF904202169A0683DE07B
:1099F000072D3ED161683F4804F0A6FAC8B9E16876
:109A0000464804F0A1FAA0B96169454804F09CFAFF
:109A1000054670B901A8F7F785FD012813D1A069A3
:109A2000BDF90480A668276903F060FC424603463E
:109A30001AE061682F4804F087FA20B9E1683748D6
:109A400004F082FA08B1374829E06169364804F029
:109A50007BFA05460028F6D1A069A668276903F0BD
:109A600045FC4FF0FF3302B239463046FFF7D2FED5
:109A700039E0092D12D161681E4804F065FA90B1F1
:109A80002A480CE000252EE003F038FC6A2303602E
:109A900004222749164802F05DF824E0254804F026
:109AA0005FF901251FE0E1681C4804F04DFA002829
:109AB000E6D161691C4804F047FA0028E0D1E16969
:109AC000174804F041FA05460028D9D1A069A668D4
:109AD000276903F00BFC8046206A03F007FC0FFAAD
:109AE00088F20346C0E7284602B0BDE8F08100BF17
:109AF000783400207F0B0108840C0108A8110108AC
:109B00003C1201084212010863120108E012010828
:109B100030130108641301089650002082130108D5
:109B2000F81401088613010801150108C80F01087F
:109B3000AA5000200515010813B5044601A8F7F73F
:109B4000F1FC70B1BDF90430A34207D0012807D958
:109B5000BDF90600031B5842584102E0012000E015
:109B6000002002B010BD000000F00700072813D845
:109B7000DFE800F00406080A0C0E121008480CE09A
:109B800008480AE0084808E0084806E0084804E0F9
:109B9000084802E0084800E0084804F057B800BF51
:109BA00055150108621501086F1501087C1501089B
:109BB0008915010896150108A3150108B0150108BB
:109BC00000F03000202805D0302805D0102805D11D
:109BD000044804E0044802E0044800E0044804F0BB
:109BE00035B800BFBD150108C0150108C51501082D
:109BF00065160108F0B5012893B006460D4607D159
:109C00006C4804F0ADF86C4804F0AAF8002005E0B8
:109C100049686A4804F098F930BBF1E702F0E0FBCC
:109C20000446002800F0C3802822211D08A8FEF762
:109C3000D5FA237FB4F91E60054604F114021821F9
:109C400002A802F039FC3246034629465C4803F07C
:109C5000FDFF607FFFF788FF607FFFF7B1FF594886
:109C600004F07EF82046D9E7012E40F39880022EBA
:109C700074D06968544804F067F90446002857D145
:109C8000023E012E02D0022E0CD022E008A8F7F7E7
:109C900049FC012898BFBDF92060AF6888BF2646FF
:109CA00000251CE0AF6808A83946FEF74DFB28B92F
:109CB000A86803F01BFBEF6806B2F1E702A8F7F70C
:109CC00031FC012898BFBDF90860ED6888BF2646C1
:109CD00005E0A86803F00AFBEF682D6906B230467C
:109CE000FFF72AFF08B9394805E0394608A8FEF70A
:109CF0002BFB20B9364804F033F8012457E04DB16E
:109D000008212A460DEB010002F002FC034610B9BF
:109D10003048F0E72B460022009208A902AA3046FC
:109D200002F0B0FA08B92C48E5E739462B4812E0B2
:109D300069682B4804F008F9044678B9AD6808A8AA
:109D40002946FEF701FB0028D4D008A9204602F0DE
:109D50003BFB2448294603F079FF28E06968224844
:109D600004F0F2F80446D0B902F03AFB2346054667
:109D70005DB123B1191DB3F91E0002F025FB284681
:109D800002F02EFB2B460546F2E723B1191DB3F96D
:109D90001E0002F019FB154803F058FF07E02B687E
:109DA00000931A461946124803F050FFA5E72046D3
:109DB00013B0F0BDC9150108181601080B00010801
:109DC000671601083FF800087F0B01087C160108A0
:109DD000E90B01089C160108C7160108F7160108CF
:109DE000840C010829170108880901085217010885
:109DF0007117010870B501288AB00C460DDD48685E
:109E000003F074FA05B22846FFF796FE30B92168D0
:109E1000164803F01BFF012025E00025144803F03D
:109E20009FFF144803F09CFF002002F0F1FA044663
:109E3000C8B1B4F91E600DB1AE4212D12822211D65
:109E40006846FEF7CBF9314602460B4803F0FEFEAA
:109E5000607FFFF789FE607FFFF7B2FE074803F0DF
:109E60007FFF2046E1E70AB070BD00BF1D18010862
:109E700036180108331601086A1801083FF800086F
:109E800008B501460B4803F0E1FE0B4803F068FFFC
:109E90000A4803F065FF0A4803F062FF094803F02F
:109EA0005FFF094803F05CFF0848BDE8084003F085
:109EB00057BF00BF78180108D4180108DE18010840
:109EC000EC180108461901085A1901086B19010814
:109ED0000C4AF0B514880830260AE5B200238B42FC
:109EE00009D2FF2C85BFC718C654C5547D708CBFDE
:109EF00002330133F3E781BF138809181B0A01F805
:109F0000013CF0BD240200202DE9F0430D4685B050
:109F100002210446FBF71FFD032107462046FBF7FD
:109F20001AFD07B108B9274845E08668264AB38874
:109F3000F48812885BBA9BB264BA9A42A4B239D14F
:109F40002249234B0A881B889A4203D9944203D39F
:109F5000012307E0944204D39C428CBF00230123D9
:109F600000E0002333B3BF68D0F80C901948944246
:109F700098BF013207F1080898BF0A80282241469D
:109F8000FEF72CF94FF47A72B388B5FBF2F102FBBD
:109F9000115502910395FA7901925BBA02469BB280
:109FA000494600940C4803F051FE404602F038FA4E
:109FB000012003E0094803F0D3FE002005B0BDE80E
:109FC000F08300BF8619010824020020D65000202B
:109FD000D8500020AE500020BD190108001A010819
:109FE0002DE9F04F99B081460C461022002114A8AB
:109FF00003F024FD812315939C4BB9F1010F1B88BD
:10A00000ADF85C303BDDB9F1020F00F0C88160684B
:10A0100003F06CF9051ED4BF4FF000084FF00108A3
:10A0200008F101034FEA830754F82330089308F13D
:10A030000203D8BF0325994505DDE319586803F0ED
:10A0400055F9049001E00423049308F103039945B2
:10A0500005DDE319986803F049F9064601E04FF47D
:10A060007A7608F10408C14505DD2744F86803F055
:10A070003DF9099000E00995049B002B03DA206864
:10A08000FFF7FEFE3DE04FF0FF3225210898FEF776
:10A0900082F804B2621C089910A808BF0024FEF7D9
:10A0A00053F908B972482AE00822724910A803F04F
:10A0B00095FB50B19DF84030FF2B05D19DF8413004
:10A0C00003F00F03022B00D0ECB10EA8F7F72AFA29
:10A0D0007CB1002800F05E81BDF93830A34212D077
:10A0E000012840F25781BDF93A30A34240F0528135
:10A0F00009E0012802D1BDF9384004E05E4803F0D0
:10A100002FFE012053E114A90320FBF7ABFB00282D
:10A1100001DA5A48F3E7F6F771FC4FF47A737343A8
:10A120000D9300220023CDE90A010027CDE9062383
:10A130004FF0FF332E460593BA46BB46013E731CD3
:10A140004F4A00F006814E4B19884E4B1A88013257
:10A1500092B21A80049B00938020002301F0BAFF82
:10A16000804698B104998068FFF7B2FE10AA0021DA
:10A17000404602F00FF8814640B1ACB14FF0FF33DA
:10A1800008220021F7F76AFB814618B93E4803F020
:10A19000E7FDD3E7836800221A705A705A719A71EA
:10A1A0001A715A8083685C800020F8F7AFF94B463B
:10A1B000804640F2022235490220FBF77FF90C90DD
:10A1C00038B9334803F0CCFD0C994846F7F738FC12
:10A1D000B4E7304A00230EA800F074FB00282DDB02
:10A1E000BDF83A2040F201239A4220D10020F8F72E
:10A1F0008DF9DDF83C90C8EB000841464846FFF772
:10A2000083FE002183444846F7F71AFC059B474527
:10A2100038BF4746434528BF43460593DDE906233B
:10A2200012EB080243F10003CDE906231AE00F4BBD
:10A2300019880EA809B2F8F717FC13E0164803F0C6
:10A240008FFD0FE00EA8F8F7B1FC002828DDBDF85F
:10A250003A304345F6D1114803F0F8FC00210F983D
:10A26000F7F7EEFB40F20128ECE700BF9C0200206C
:10A270001D1A0108D5FD0008361A0108841A0108C4
:10A2800024020020D8500020180901080000FFFF18
:10A29000A41A010840420F00CF1A0108DC1A010875
:10A2A0001EB100210D9800F0C9FA099B0AF1010ABC
:10A2B000534502D0002E7FF441AFF6F79FFB08997B
:10A2C00080463C4803F0C2FCBBF1000FC6EB050A18
:10A2D00038DD5246DDE90601D31702F07BFEDDE9E9
:10A2E0000A23B8EB02029046334AB8FBF2F164232A
:10A2F00002FB11828DE806000C905A46514603FB82
:10A300000BF32E4893FBFAF3C3F1640303F09EFCB6
:10A310004FF47A72B7FBF2F002FB107E01900C98BA
:10A320000C9BB3FBF2F302FB130000900598059918
:10A33000CDF808E0B1FBF2F102FB1102204803F076
:10A3400085FC03E051461F4803F080FC4FF0000AF3
:10A35000F4E61D4B00211980138814A90133032052
:10A360001380FBF7A1FA40F201240EA8F8F71EFCB7
:10A3700000280BDDBDF83A30A342F6D1134803F0B4
:10A3800065FC00210F98F7F75BFBECE7BBFA8BF05D
:10A3900040090CE021460E4803F058FCB1E6636822
:10A3A000089304274FF00008032504974DE619B0E1
:10A3B000BDE8F08F211B010840420F003D1B010842
:10A3C000861B0108BA1B0108D8500020DC1A0108BE
:10A3D000F11B010838B5447C074B04F00F0400253D
:10A3E000057421461868FDF789FA044B142202FB14
:10A3F0000434E56038BD00BFDC500020E050002090
:10A4000008B50146054803F021FC054803F0A8FC07
:10A410000448BDE8084003F0A3BC00BF171C0108B6
:10A42000601C0108A91C010873B501AD2846F7F7A7
:10A4300079F800240646B44211D035F91400F9F732
:10A44000ABF850B1B0F88E31DB0706D500231A46C1
:10A45000194635F91400FAF7C9FB0134EBE702B0ED
:10A4600070BD000030B511488DB003F079FC104884
:10A4700003F076FC0024E0B2FBF7F4FB054678B16C
:10A480000146282202A8FDF7A9FE6A8A2B7C0192C8
:10A490006A7C1209009221460246064803F0D6FB68
:10A4A0000134102CE7D100200DB030BDC81C0108CC
:10A4B0002B160108001D0108F0B5064689B00846B4
:10A4C00015461F4602F012FF0F28044603D93046F6
:10A4D000FFF796FF24E0284603AA234903F0B0FFC4
:10A4E00005460028F3D003AA1F49002003F0A8FF67
:10A4F0000028ECD002F0FAFE431E802B064601D95C
:10A500001A480BE0294604A8FDF71EFF102218493F
:10A510000DEB020003F062F920B9164803F020FCAD
:10A5200001201EE0144D2B6813B9FDF703F82860D5
:10A53000E4B221462868FDF7B9F9002801DA0F488E
:10A54000ECE7384602F0D2FE01230093F2B283B268
:10A5500004A92046FBF7A6FB0028F0D0FFF764FF14
:10A56000002009B0F0BD00BF221D0108241D010814
:10A5700025FE00084E1D0108DC5000206A1D010860
:10A5800038B50446084602F0B1FE0F2803D920462C
:10A59000FFF736FF1AE0104C142303FB0044E56874
:10A5A00085B9C0B2FBF75EFB90B1437C458223F0D6
:10A5B00010034374094B2061E36009492046F6F714
:10A5C000A5FA05E00146074803F040FB012038BD2D
:10A5D000FFF72AFF002038BDE0500020D5A3000877
:10A5E00000A3E111851D0108012870B505460C4640
:10A5F00003DCFFF737FF002070BD49680E4803F009
:10A60000A3FC48B9042D12DD04F1080120680EC92D
:10A61000BDE87040FFF750BF6168084803F094FC44
:10A6200028B9A1682068BDE87040FFF7A9BF20687D
:10A63000FFF7E6FE012070BD7F0B0108840C0108C6
:10A64000F0B5C5B00446182200210BA803F0F6F9B6
:10A6500004271822A6B243F23905002111A80B974E
:10A66000ADF84060ADF8425003F0E8F91C4911978D
:10A6700012A8ADF85860ADF85A50FDF765FE194BB9
:10A680000393402200238DF811200BA91A461DA820
:10A690008DF8103001F0B8FF134803F061FB11ABE7
:10A6A000062203A91DA802F073F817AB009305A9B1
:10A6B0000E4B16221DA801F0FDFF011E0BDD05A8A3
:10A6C000BDF87230009418AA00F05CF80021084828
:10A6D00000F0B4F8E0E7074803F042FBDCE700BF16
:10A6E000AC1D010855484350B71D010880969800DD
:10A6F00000879303D51D010838B50C462E2201466C
:10A700002046FDF76BFD054628B902F0F7FD1C2336
:10A710000360284638BD204638BD00002DE9F041D1
:10A7200005469EB00E46304606A990461F46FFF7E6
:10A73000E3FF6C790734E41002ABC4F110029818FF
:10A74000002103F07BF92246A91D02A803F078F846
:10A7500012A902A8FFF7D0FF6B790093424612AB13
:10A7600006A9074803F072FA6979009733464FF655
:10A77000FF7202A8FDF74EFA1EB0BDE8F08100BFDF
:10A78000F61D01082DE9F0418CB01F460D46044628
:10A79000694610461646FFF7AFFF3A466946164827
:10A7A00003F054FA052D01D8144816E02268144B22
:10A7B0009A4201D0134810E0237903F00F081B09D7
:10A7C00002D0114803F0CCFAB8F1010F0FD1637930
:10A7D000DB0806339D4203D20C4803F0C1FA08E0BF
:10A7E000129B3A4631462046FFF798FF01E00848A1
:10A7F000F3E70CB0BDE8F0811A1E0108361E01080F
:10A80000554843504F1E01086A1E0108891E010861
:10A81000A31E0108F7F7E4BFB0F90010F8F700B97C
:10A8200038B504460020F7F771FE05460020F7F71B
:10A830006DFE401BA042F9D338BD000030B587B093
:10A8400004460D46F5F717FE40B11DB10E49032031
:10A85000F6F7F8F92046FFF7E3FF13E00B4B009003
:10A8600003900290012168460493CDF814D0F7F7C5
:10A8700087FF214601A82A46F6F768F901216846B4
:10A88000F7F77EFF07B030BD00F8000815A80008F4
:10A8900030B4034DC560026130BC1380F6F736B9A1
:10A8A00019A8000870B41146039ABDF91050044E5F
:10A8B000C660026115801A4670BCF6F747B900BF42
:10A8C00019A8000870B58AB00021079106911049B7
:10A8D000098803AC09B2054643F23906019105A87F
:10A8E0000094ADF80E600494FFF7DCFF2846F8F7FB
:10A8F00060F96B88B34202D16B68A34204D005A80B
:10A90000F6F7F2F8012001E04FF0FF300AB070BD19
:10A910009C02002010B5084B0446182240F8203B4A
:10A9200002F08EFF082384F83A30002384F8383090
:10A9300084F83B3010BD00BFF01E010837B5044657
:10A9400000F02EFB94F838301BB90321204600F0AC
:10A9500052FA002508216846A576A58301F0CEFFAE
:10A960009DF80030019A23F0010343F002038DF8B3
:10A970000030009B12BA1BBA204600F0F6F8BDF872
:10A98000001049BA204689B200F0DEF820462321A3
:10A9900000F01CF920461A2100F00BF92946204648
:10A9A00000F030F920460122202100F0ABF92046CA
:10A9B00001224FF4807100F0A5F92A4620464FF499
:10A9C000005100F09FF9204601224FF4804100F031
:10A9D00099F901232373802220460C2100F051FABB
:10A9E0000421204600F05FFA042100F0FD02204619
:10A9F00000F047FA0321204600F055FA032100F049
:10AA0000F002204600F03DFA082220460E2100F018
:10AA100038FA0F21204600F046FA1621204600F0B1
:10AA2000EAF903B030BD10B590F83B30013304466D
:10AA300080F83B30204600F08EFAA0F11103DBB223
:10AA4000012BF7D9192818BF84F83A00192120469C
:10AA500000F0D1F9022384F8393010BD70B51D46DD
:10AA600090F839306E1C1344144680F83930134680
:10AA70000A46F1B200F029FA601970BD10B5012341
:10AA800000F139020021044600F01FFA02221146AB
:10AA9000204600F0F6F963683BB1A28B120504D59D
:10AAA00020460321BDE81040184710BDF8B5082125
:10AAB000044600F0A0F915210746204600F0F3F9FE
:10AAC00060F07F02D2B215210646204600F0D9F987
:10AAD0000621204600F08FF90821204600F0E3F916
:10AAE00060F07F02D2B20821204600F0CAF90121AD
:10AAF000204600F0D8F903060546F8D53246204630
:10AB0000152100F0BEF90821204600F074F93946FD
:10AB1000204600F070F9C5F38010F8BD38B50D4639
:10AB20000221044600F0ADF9162D07D0204600F0B2
:10AB300012FA8542FAD184F8385038BD204600F028
:10AB40000AFA1F28FAD0F6E710B50A0A044601F0FF
:10AB50007F0142740174202100F093F9227C204689
:10AB60002121BDE8104000F08CB92DE9F8430546DD
:10AB700016461F4600F1110800246FF00709E20095
:10AB80003046394602F01AFA09FB04F208F8010FC0
:10AB900038323046394602F011FA04F12401C2B2CB
:10ABA000C9B22846013400F06CF9082CE7D1BDE8A1
:10ABB000F883A1F10B020F2A05D8C27E8A4202D087
:10ABC000C17600F009BA70470020704737B50D0A0A
:10ABD000C181CAB22221044600F053F92A4623213A
:10ABE000204603B0BDE8304000F04BB908B5052160
:10ABF00000F059F9024B00F00F0033F9100008BDC6
:10AC0000D01E0108113109B21429A8BF142121EA6C
:10AC1000E171024B5A5C052100F033B9BB1E0108FB
:10AC200008B52C2100F03FF9C0F3071008BD38B576
:10AC30000C462C21054600F036F9072C28BF0724C6
:10AC400000F00F0040EA0412D2B228462C21BDE8E1
:10AC5000384000F016B908B52C2100F024F9C0F3F3
:10AC6000420008BD0529A8BF0521002938B50C46BA
:10AC7000A8BF0C464FF02C010546B8BF072400F0D2
:10AC800012F920F00E0040EA4402D2B228462C21EC
:10AC9000BDE8384000F0F5B838B505460C4699B126
:10ACA0000A782D2100F0EDF82E21284600F0FBF85F
:10ACB000637800F0F80203F007031A4328462E21B8
:10ACC000BDE8384000F0DDB838BD08B5092100F016
:10ACD000EAF800F00F0040005B3840B208BD0029E0
:10ACE000C4BF494249B25B31C1F3430242F0C002E2
:10ACF000092100F0C6B808B5072100F0D4F85B3888
:10AD000040B208BD10B5838B0446B2B30B43B1F516
:10AD1000807F83830AD002D8202925D010BDB1F5C9
:10AD2000007F0ED0B1F5005F20D010BD00F1120100
:10AD3000FFF7B2FF04212046FFF794FF53222F2193
:10AD400053E02E2100F0AFF840F01002D2B22E21D5
:10AD5000204600F096F81721204600F0A4F840F0B5
:10AD60000202D2B2172140E02E212BE00E2100F08A
:10AD70009AF840F00402D2B236E023EA0103B1F5BA
:10AD8000807F83830AD002D8202921D010BDB1F55D
:10AD9000007F09D0B1F5005F21D010BD4FF0FF3129
:10ADA000BDE81040FFF75EBF172100F07CF81721C7
:10ADB00000F0FD02204600F064F8A38B9B0619D535
:10ADC0002E21204600F06FF800F0EF022E210CE05B
:10ADD0002E2100F068F840F01002D2B2F6E70E2102
:10ADE00000F061F800F0FB020E212046BDE81040A3
:10ADF00000F047B810BD70B504460D46204600F07F
:10AE0000AAF8A0F11103DBB2012B0646F6D91F28E0
:10AE1000F4D0032D02D12A46082126E0A84227D0EB
:10AE2000162801D1192D02E0192807D1162D0AD1B3
:10AE3000092211462046FFF771FE04E00F2802D1D7
:10AE4000204600F094F80F2D0DD103212046FFF786
:10AE5000D2FF2946204600F026F8206BF7F7CCFAFF
:10AE600084F8385004E02A4629462046FFF756FE6B
:10AE7000304670BD90F82430816A006A0022F7F7EE
:10AE80002BB970B504460D461646FFF7F3FF33465F
:10AE900045F0C002A16A206A01F071FE206ABDE897
:10AEA0007040F7F759B938B504460D46FFF7E2FF91
:10AEB00045F080020023A16A206A01F060FE054689
:10AEC000206AF7F749F9284638BDF7B504460F461A
:10AED00015461E46FFF7CEFFA16A206A40230122D5
:10AEE00001F03CFE3B46A16A206A012201F036FED9
:10AEF0000022206A019600922B46A16AF7F748F9D2
:10AF0000206A03B0BDE8F040F7F726B910B5044653
:10AF1000FFF7B0FFA16A206A20230122BDE810409C
:10AF200001F01CBE07B58DE806000023816A006AA7
:10AF30000122F7F72DF903B05DF804FB10B50446C4
:10AF4000816A006A0123002201F008FE206ABDE840
:10AF50001040F7F701B908B590F838300F2B04D03E
:10AF60000121FFF7A0FF00F01F03184608BD10B530
:10AF70000446FFF7F0FF0F2811D1206BF7F745FAD1
:10AF800000214FF49970FFF759FC01212046FFF78B
:10AF90008AFF00F01F00082884F83800F5D110BDA2
:10AFA00010B50446406BF7F730FA00213E20FFF75A
:10AFB00045FC606BF7F720FA00213E20FFF73EFCCE
:10AFC00001212046FFF76FFF00F01F0310F0170F5D
:10AFD00084F83830F4D110BD38B508210446FFF7A5
:10AFE0000AFF082105462046FFF75DFFE37E00F0DB
:10AFF000E00203F01F0320461A430821FFF741FF38
:10B0000029462046BDE83840FFF7F5BE43680BB13E
:10B0100000211847704700002DE9F0470446884694
:10B0200016461F46FFF797FF8146002C00F0D3809D
:10B030000F2840F0DF80B8F1180F66D02046FFF7E8
:10B0400096FFB8F1270F00F22B81DFE818F04200DD
:10B05000290128003300290129013B002901290188
:10B060002901290129012901290129012901550065
:10B0700029018B008F007E0029018400290129010C
:10B080002901930097009B009F002901A300AA00BB
:10B09000290129012901290129014E00BA00022FA5
:10B0A00003D98B490320F5F7CDFD31882046FFF702
:10B0B0004BFD94E0082FF4D8D6E900232046FFF793
:10B0C00054FD8CE0022FECD831882046FFF77EFD3E
:10B0D00085E0012FE5D03178A1F10B030F2B00F2B1
:10B0E000EC802046FFF765FD79E0012FD9D0337859
:10B0F000002B40F0E2806CE0022FD2D8B6F90010AD
:10B100002046FFF77FFD0225D9E0012FC9D833780B
:10B11000013B052B63D8DFE803F00507620C14033D
:10B12000082102E00F2100E016212046FFF763FE10
:10B13000CBE0A38B5A0540F1C8802046FFF79EFC68
:10B14000C3E02046FFF7FAFBBFE03278202120461B
:10B15000FFF7D8FD43E0012FA3D831782046FFF751
:10B1600066FD36E032784FF4806116E032784FF4B5
:10B17000007112E032784FF400510EE032784FF453
:10B1800080410AE032784FF4006106E032784FF4F3
:10B19000805102E032784FF480712046FFF7B2FD13
:10B1A00017E0012F3FF67DAFA38BDB0503D4337887
:10B1B000052B40F2828096F900102046FFF752FDE1
:10B1C00007E0012F3FF66DAF96F900102046FFF71C
:10B1D00086FD012573E06FF01200BDE8F087B9F13C
:10B1E0000F0F5DD03B46324641462046BDE8F04752
:10B1F00001F038BCB8F1270FF4D801A353F828F0B8
:10B20000D3B00008E5B100089FB00008B5B0000851
:10B21000E5B10008E5B10008C5B00008E5B10008D7
:10B22000E5B10008E5B10008E5B10008E5B10008A6
:10B23000E5B10008E5B10008E5B10008E5B1000896
:10B24000F9B00008E5B1000865B100086DB100086B
:10B250004BB10008E5B1000857B10008E5B100089E
:10B260000BB10008E5B1000875B100087DB1000818
:10B2700085B100088DB10008E5B1000895B100085E
:10B28000A3B10008E5B10008E5B10008E5B1000888
:10B29000E5B10008E5B10008EBB00008C3B1000853
:10B2A000B8F1180F9ED06FF085050F212046FFF7EB
:10B2B000A2FD15F1860F05D194E76FF01505B9F1E0
:10B2C0000F0FF2D02846BDE8F0870120BDE8F087D7
:10B2D00000F800082DE9F0410446FFF73CFE0F2876
:10B2E00006464CD00F212046FFF7DDFD0221074620
:10B2F0002046FFF7D8FD7B07054603D5636801218B
:10B300002046984738073AD5162E01D0112E05D180
:10B31000A38B590433D5636802212CE0192E01D088
:10B32000122E2CD194F83B301BB916490320F5F7A7
:10B3300089FC013BDBB284F83B3023B994F83A1026
:10B340002046FFF758FD6368CBB1A28BD20416D517
:10B3500005F0E000202809D002D838B1BDE8F0811E
:10B36000602807D0A02803D0BDE8F081042102E0C6
:10B37000062100E007212046BDE8F0411847BDE85E
:10B38000F08100BF00F8000813B50446816A006A26
:10B39000F6F774FE0121206BF6F76AFF206BF7F7D2
:10B3A00034F80121606BF6F763FF606BF7F724F860
:10B3B000094B009401220021E06AF6F793FF204632
:10B3C000FFF7BCFA1C212046FFF76DFD033818BFBC
:10B3D0004FF0FF3002B010BD0DB000082DE9F34171
:10B3E00004460F4690461E46FFF790FD01220DF1E0
:10B3F00003012046FFF796FD9DF8035005F07F05F9
:10B40000023D07B3454505D92046FFF797FD6FF08C
:10B4100068051BE02A4639462046FFF783FD0222D5
:10B4200001A92046FFF77EFD6EB10122B11820462A
:10B43000FFF778FD2046FFF781FD07212046FFF743
:10B4400032FD307002E02046FFF778FD284602B05A
:10B45000BDE8F0812DE9F04107460D469046FFF723
:10B46000E2FA0026344646450FD06A68A31C13440E
:10B470007F2B05F1080511D8234655F8081C3846DE
:10B48000FFF7ECFA01360446EDE7BB8B5B0502D40F
:10B490003846FFF7F3FA2046BDE8F0816FF08A00E6
:10B4A000BDE8F08108B5FFF756FD0838C0B2112895
:10B4B0009ABF024B185C022008BD00BF081F01089C
:10B4C0002DE9F8430F46164698460546002800F039
:10B4D000B780A1F11103152B4DD8DFE803F0182731
:10B4E000344C4C4C4C204C383C40444C484C4C4C1C
:10B4F0004C4C4C0BB8F1010F03D857490320F5F71A
:10B50000A1FB00237370FFF75FFB307004E0B8F11C
:10B51000010FF2D9662333800220BDE8F883B8F129
:10B52000000FEAD0FFF7BEFF307009E0838B13F401
:10B53000806F03D001203070BDE8F88300233370A2
:10B540000120BDE8F883838B13F4007FF1E7838B40
:10B55000C3F34033F3E7838BC3F38033EFE7838B8D
:10B56000C3F3C023EBE7838BC3F30033E7E7838B9D
:10B57000C3F30023E3E74346324601F0CDF910F16F
:10B58000860F044660D12846FFF7E5FC0F28814668
:10B5900011D12846FFF7EBFC162F1CD004D8012F41
:10B5A00035D0102F0ED046E0272F28D02F2F36D0A1
:10B5B000202F1DD03FE0162F0DD013D8012F26D0FD
:10B5C000102F44D1B8F1010F97D92846FFF70EFB91
:10B5D000022430802CE0B8F1000F8ED02846FFF70F
:10B5E0001FFB23E0272F0AD02F2F18D0202F2ED17A
:10B5F000B8F1000F81D02846FFF72DFB16E0B8F117
:10B60000000F3FF47AAF2846FFF75FFB0EE0B8F17A
:10B61000000F3FF472AF2846FFF748FA06E0B8F192
:10B62000000F3FF46AAF2846FFF765FB3070012436
:10B63000B9F10F0F08D10F212846FFF7DCFB03E01B
:10B640006FF01200BDE8F8832046BDE8F8836FF084
:10B650008500BDE8F88300BF00F80008094B70B50D
:10B660001C6806460D4620460821F4F7FFFD2146DA
:10B670003046F5F767FB2846F4F7FAFEBDE8704060
:10B68000F5F746BBA00200202DE9F04104460E4626
:10B690001546F4F7E5FE27688046A7B13B682360AE
:10B6A00096E803007B6883E803000A21A7F10800FD
:10B6B000F4F7DCFD17F8034C4046F4F7D9FE2046BA
:10B6C000F4F714FE1FE0A268E3689B1A2269934214
:10B6D00007DDDDB14146201DFFF7C0FFF4F7C0FED6
:10B6E00080460D4BE1681B8833804B1CE360236967
:10B6F00062690B4096E8030002EBC30383E8030092
:10B700004046F4F7B5FE0120BDE8F081F4F7B0FE45
:10B710002846BDE8F08100BF9C020020F8B5044631
:10B720000F461546F4F79CFEA168E3688B42064677
:10B730001CD04B1CA3602369626965680B4002EB57
:10B74000C30393E8030087E80300E5B128460A2114
:10B7500050F808396360F4F789FD15F8034C30465A
:10B76000F4F786FE2046F4F7C1FD0FE03DB1084B2B
:10B770001B680146DF602046FFF770FF06E0F4F724
:10B7800077FE2846F8BD3046F4F772FE0120F8BD7A
:10B79000A0020020BFF34F8F0549064BCA6802F490
:10B7A000E0621343CB60BFF34F8F00BFFDE700BFE4
:10B7B00000ED00E00400FA050121F6F7E1BF10B545
:10B7C0000446406908B101F059FAE06908B101F096
:10B7D00055FA00200022002360612061E061A06131
:10B7E0002080C4E9022310BDF5F708B92DE9F04F18
:10B7F00089B08A4615469B460446FFF7F5FFCDE91A
:10B800000401EB000393079355445346AB4205D024
:10B8100013F8012B002AF9D0002300E001230027B0
:10B8200002936FF075030193B846B9463E46A2688D
:10B83000974270D222687D0102EB050EDEE902011B
:10B84000002908BFB0F1FF3F23D0DDE9042399426E
:10B8500008BF90421DD200220023CEE902232268B5
:10B860002A44166122682A44966122685653226847
:10B870002A44506920B101F001FA22682A44566135
:10B8800022682A44D06920B101F0F8F922682A44DC
:10B89000D661039B98453CD222682A44506900280F
:10B8A00037D007AA514601F01FFA38B923681D4462
:10B8B000129BCBF800500120186034E0029B13B1BA
:10B8C00002282DD1F2E7012814D1226815442969F4
:10B8D00011F07F4F1BD0079AB2EB116F17D3B8F15D
:10B8E000000F01D0904512D20023CBF800509046B3
:10B8F00001930AE002280AD1B8F1000F07D12268AB
:10B90000CDF804801544CBF800504FF00109039B9B
:10B91000079301378BE7129B0198C3F8009002E070
:10B920000128F4D1D1E709B0BDE8F08F38B505465C
:10B930000C46FFF759FF4FF47A736B43C01841F17F
:10B940000001C4E9000138BD2DE9F04788B097290E
:10B9500090461BBF109A0792424605AA8A461CBF12
:10B96000CDF814808DF81830ADF806100292DF0083
:10B9700000F1120500F1200600F11C046FF001092E
:10B9800035F9023FDBB1BAF1970F03D000976A4651
:10B99000414607E0D8F8183019684B78DB0000936F
:10B9A0006A460231306801F09FF9023007D0B5F9DC
:10B9B000002003A901A8F7F79DF84FF00009A54260
:10B9C00006F10406DCD1484608B0BDE8F087000067
:10B9D00030B587B006AA102302AD294642F8143DBF
:10B9E00001F064F9A842014620D1019B102B08D137
:10B9F00028220F48FCF7F2FB01460E4802F026F918
:10BA000014E00024019BA34204D3295D0A4802F0FC
:10BA10001DF902E0094802F019F90134102CF1D1A6
:10BA20000724074802F012F9013CFAD107B030BDF3
:10BA3000205200201A1F01087A0B0108F1050108A5
:10BA4000F20501082DE9F04F00F10C0787B004461C
:10BA500038469A468B469046149EFFF7ADFE01236A
:10BA60000493B8F1000F01D0119B2BB93846F6F7BB
:10BA7000B7FE6FF00D006AE004AB0093524605ABD1
:10BA800041462046FFF7B2FE012802D04FF00009E0
:10BA90001CE012991198059C01F08EF8054610B92A
:10BAA0006FF00B044FE0E06901F0E8F8139BE561EB
:10BAB000721CA36102D004F1080139E04FF0FF329B
:10BAC0000023C4E902233DE009F10109A268914580
:10BAD000E6D222684FEA49152A44D2E9020150EA27
:10BAE0000103F1D151464046039201F065F8039AF3
:10BAF000506122682A44516971B1109B1361226818
:10BB0000129911982A44039201F056F8039A139B54
:10BB1000D06122682A44936122682A44D1690029AD
:10BB2000D2D0A2F800B0731C216805D02944083196
:10BB30003046FFF7FBFE05E00D444FF0FF320023D7
:10BB4000C5E9022300243846F6F74AFE204607B02E
:10BB5000BDE8F08FF0B500F10C0485B00546204635
:10BB60000E461746FFF728FE0123029302AB00930F
:10BB70003A4603AB31462846FFF738FE012802D18A
:10BB80000398FFF71CFE2046F6F72AFE05B0F0BD2D
:10BB9000F8B500F10C06054630460F46FFF70CFEDF
:10BBA0000024AB689C420AD22868630117B1C25EC8
:10BBB000BA4202D11844FFF702FE0134F1E73046E1
:10BBC000BDE8F840F6F70CBE2DE9F04F00F10C048B
:10BBD00085B0054620469B46894692460F9EFFF754
:10BBE000EBFD01230293B9F1000F04D0BBF1000F6C
:10BBF00001D00E9B2BB92046F6F7F2FD6FF0150031
:10BC000049E016B1BAF1000F05D12046F6F7E8FD7C
:10BC10006FF00D003FE002AF009703AB109A314682
:10BC20002846FFF7E3FD0128804615D9119B0093B4
:10BC30003246109B99212846FFF786FE48B901231A
:10BC40000293009703AB109A31462846FFF7CEFDCA
:10BC50008046B8F1010F0CD8039B5A465146D8696B
:10BC600001F024F858B92046F6F7BAFD6FF06800E5
:10BC700011E02046F6F7B4FD6FF075000BE0039B72
:10BC8000B3F90020A9F800200E9A9B6913602046A2
:10BC9000F6F7A6FD002005B0BDE8F08FF8B5064622
:10BCA000002546F80C5F04463046FFF785FD04F199
:10BCB000120204F11C0304F1300122F8025F43F880
:10BCC000045F8B424FF00007F7D123792761022BE5
:10BCD000A2680BD1236852013946186801F0AEFE04
:10BCE00023689A685868D200394602E020685201F9
:10BCF000394601F0A3FE01F059F83046BDE8F8409E
:10BD0000F6F76EBD2DE9F04F044600F10C0585B045
:10BD10002846FFF751FDFFF767FD2379012B804689
:10BD200089466AD1674A684B684969488DE80C00C2
:10BD3000684B01F08BFF4FF0000BA3689B456BD263
:10BD400021684FEA4B1A5144D1E90223134351D0E1
:10BD50004869FFF73DFE23685F485344196901F0C5
:10BD600075FF23685344196911F07F4F04D0090E01
:10BD70005A4801F06BFF02E0594801F067FF236861
:10BD80005344D869FFF724FE236853485344996904
:10BD900001F05CFF23685344D3E90267002F08BF1A
:10BDA000B6F1FF3F1CD0B6EB080667EB0907002E83
:10BDB00077F1000301DA4B4913E0304639464A4A2D
:10BDC000002301F007F9002303923046464A394622
:10BDD00001F000F9039A0146444801F037FF03E0FF
:10BDE0004349444801F032FF2368434833F90A10BD
:10BDF00001F02CFF0BF1010B9FE7022B0CD1324B12
:10BE000000933E4A3E4B3F493F4801F01FFF4FF031
:10BE1000000BA3689B4505D3284605B0BDE8F04F4D
:10BE2000F6F7DEBC236819684FEA4B1A5144D1E992
:10BE30000223134343D08B691868FFF7C9FD2368B9
:10BE40001B6853445B691868FFF7C2FD23682F48DD
:10BE50001B685344196901F0F9FE23681B685344B9
:10BE6000D3E90267002F08BFB6F1FF3F1CD0B6EB45
:10BE7000080667EB0907002E77F1000301DA19497C
:10BE800013E030463946184A002301F0A3F8002396
:10BE900003923046144A394601F09CF8039A014651
:10BEA000124801F0D3FE03E01149124801F0CEFE22
:10BEB000236811481B6833F90A1001F0C7FE0BF123
:10BEC000010BA6E75D200108182001087320010876
:10BED000EF1F0108E61F0108202001082A200108A1
:10BEE000332001083B20010840420F004A2001088E
:10BEF00054200108432001083F1F01086320010866
:10BF00005A200108702001087F200108A1200108A3
:10BF100003461A78591C0AB10B46FAE7181A7047FB
:10BF200038B505460C464CB122462946012002F0A0
:10BF3000D1FB002802DB241A0544F4E738BD10B514
:10BF40000446FFF7E5FF01462046BDE81040FFF735
:10BF5000E7BFF8B5064684890F46154600206DB93F
:10BF60000023B289B168FCF797F84FF6C573021940
:10BF70009A4239680EDD013080B20BE0AE42EFD05C
:10BF80002346AA89A968FCF787F8EB686D681C440A
:10BF9000A4B2E4E73A34204400232022083180B2DE
:10BFA000FCF77AF8C04380B2F8BD00002DE9F341F8
:10BFB0000C46804603212046F9F7CDFC054618B90A
:10BFC0002E490320F4F73EFE0221F9F7C4FC074690
:10BFD0000028F5D0EB68032B4CD900F1080122466C
:10BFE0002846AE68FFF7B5FF002843D13378803B81
:10BFF000082B30D8DFE803F0052F2F2F2F0C151E4C
:10C000002700AB89B9683246404600F081F822E04B
:10C01000EB680093BA68334621464046F8F758F873
:10C0200019E0EB680093BA68334621464046F8F7BA
:10C03000D1F810E0EB680093BA68334621464046D9
:10C04000F7F784FE07E0EB680093BA6833462146B1
:10C050004046F7F747FF3178234640F2012203209C
:10C06000F9F72CFA014628B9204602B0BDE8F041A4
:10C07000F5F7E6BC02B0BDE8F08100BF00F80008AB
:10C0800038B50D46144600211A460323F5F7E6FBA2
:10C0900028B1836800221D705C709A70DA7038BD18
:10C0A00010B5044668B190F91030032B0CD14268EA
:10C0B0000831FFF74EFF50B1A36840BA5880002006
:10C0C00010BD6FF00D0010BD6FF04C0010BD6FF093
:10C0D000010010BD2DE9F041DDF818801546002261
:10C0E0000E461F46014608F108031046FFF7C8FF39
:10C0F000044650B1806876BA6DBA8680C58027B193
:10C1000042463946083001F09BFB2046BDE8F081ED
:10C11000F7B506460C46002A38D0072B36D9918849
:10C12000D088083B40BA49BA009389B202F10803AB
:10C1300082B28120FFF7CEFF074638B3237EFF2B64
:10C1400004F108020CBF002104F1180100F022F8EC
:10C15000054610B90146384613E000231A46194631
:10C160001846F9F749FB836809495E800446456033
:10C17000034640F202220220F9F7A0F9014628B94D
:10C18000204603B0BDE8F040F5F75ABC03B0F0BD5F
:10C190000000FFFFF8B50F461646022328220021B3
:10C1A000F5F75CFB054600B38468102204F1080033
:10C1B000394617B101F044FB01E001F03FFC04F106
:10C1C00018001022314616B101F03AFB04E001F0EC
:10C1D00035FC012384F82730602200232270FF22DF
:10C1E0006370A370E370A271E3712846F8BD00008C
:10C1F00008B51022034901F0F1FAB0FA80F04009C5
:10C2000008BD00BF25FE000870B505460C46002697
:10C2100023686BB158680021F5F712FC23685E6053
:10C220002368002BF4D01A68226000221A60EFE71E
:10C2300004F19000F4F758FC2846F7F7ADF938B14F
:10C24000D0F8DC319C4203D100F5E270F4F74CFCED
:10C2500004F17400F4F748FC04F12000F4F744FC06
:10C2600004F13C00F4F740FC04F15800F4F73CFC06
:10C2700010220021201D01F0E1FB00236377E383FE
:10C2800070BD00002DE9F74F914600901E469DF8C5
:10C2900030808A4609B9002069E0082BFBD808469F
:10C2A000FFF7A6FF0028F6D1DFF8C8B00546044620
:10C2B000B82303FB05F73A1D5A4410465146019234
:10C2C000FBF711FF2B4B019A98B1B9F1000F0CD07D
:10C2D0005EB1D819324649461430009301F0B0FAE5
:10C2E000009B1F443E7787F81D80B82000FB053077
:10C2F0003DE01046FFF77CFF10B10CB90BEB0704D3
:10C300000135102DD4D1002CC5D0BDF80030E38309
:10C310002046002340F8043B2A46514601F090FA9B
:10C32000B9F1000F07D036B13246494604F1140086
:10C3300001F086FA267784F81D8008F00708B8F126
:10C34000020F04BF032384F8B4304FF40973A4F838
:10C35000A6304FF40473E3864FF40573C4F8A84085
:10C36000A463A4F88A30C4F88C406465204603B006
:10C37000BDE8F08F48520020F8B507460E4609B9CF
:10C380000020F8BD0846FFF733FF0028F8D10C4D18
:10C390000446B5F91A3013B10FB1BB4209D1314689
:10C3A0002846FBF7A0FE20B1064BB82000FB043066
:10C3B000F8BD0134102C05F1B805EAD1E0E700BF63
:10C3C0004C5200204852002010B50446FFF7D4FF1D
:10C3D000014620B12046BDE81040FFF715BF10BD53
:10C3E00038B510B100F1B80400E0074C074DAC427D
:10C3F00005D2201DFFF7FCFE18B1B834F7E7002086
:10C4000038BD204638BD00BF48520020C85D00201E
:10C4100008B5FFF7E5FF10B1437F1B07F9D508BD4D
:10C42000F8B501460020FFF7A7FF044610B3437F8D
:10C4300013F0050F1ED0B0F91E00F7F7ADF80E4B44
:10C44000D0F8A061B3F9007004F13C052846F4F778
:10C450004BFB40F21723A4F8523004F150023B4644
:10C4600031462846FEF714FA637F23F0070343F0B2
:10C47000070363772046F8BDAC34002010B514469E
:10C4800000B119B90B490320F4F7DCFB2AB1537F43
:10C4900003F00703013B012B01D8002010BD137FDF
:10C4A0000B70127F04F1140101F0CAF9B4F91E00F7
:10C4B00010BD00BF00F80008F0B503EB43048C4248
:10C4C0004FF0000122D8017005465E1E0F464FF066
:10C4D0003A0E994219D014782409092C94BF3034AB
:10C4E000573494462C709CF8004004F00F04092C3B
:10C4F00094BF30345734B1426C700CBF3C46744624
:10C50000AC70013201310335E3E7F0BD0846F0BD00
:10C510002DE9F04112B90020BDE8F0811378002B1D
:10C52000F9D01446264601347378002BFAD1074619
:10C530004FF0010C964217D33478A4F130055FFA1E
:10C5400085F8B8F1090F06F1FF3E23D9A4F14105A2
:10C55000052D02D8A4F137051CE0A4F16105052DD5
:10C5600011D8A4F1570515E0BCF1000FD3D1013F5C
:10C57000B84205D23A780178397000F8012BF6E715
:10C580001846BDE8F081BCF1000FC4D14FF0010C9A
:10C590007646CFE7724518D8A6F1020E16F8016C60
:10C5A000A6F130045FFA84FCBCF1090F0ED9A6F1A4
:10C5B0004104052C02D8A6F1370407E0A6F1610476
:10C5C000052C02D8A6F1570400E0002401338B4269
:10C5D000A1D845EA04143C704FF0000C0137D7E7AE
:10C5E00008B518B907490320F4F72CFBC31C133016
:10C5F00013F8012F1AB98342FAD1012008BD002097
:10C6000008BD00BF00F800082DE9F0410C461546B2
:10C610009846064618B926490320F4F713FB11B1D2
:10C62000CB8A002BF7D02DB1EB8A002BF3D00CB1C5
:10C63000A28AB2BB06F1680718220021384601F031
:10C64000FDF95CB12368042B03D06FF06900BDE8ED
:10C65000F08118222146384601F0F2F806F18007F1
:10C6600018220021384601F0E9F97DB12B68042B2E
:10C67000EBD12846FFF7B4FF18B16FF01500BDE805
:10C68000F08118222946384601F0DAF824B1E28A0E
:10C690000421304600F0B8FBA6F898800020BDE8E1
:10C6A000F081AB8A002BC5D09A42C3D0E5E700BF2A
:10C6B00000F800082DE9F04188B090460E461A4671
:10C6C0000E9F044618B111B1B8F1000F03D12E49E5
:10C6D0000320F4F7B7FA836E002B50D008AD01A900
:10C6E00045F8183D2B4600F0A7FB002849DB0198D0
:10C6F000C368984505D20021F5F7A2F96FF06800EC
:10C700003FE00421F9F727F90028E0D0D0F80880AD
:10C7100047B118222946384601F092F8B8F800309F
:10C720005BBAFB82D4F88030E3B1B8F80030B4F8DB
:10C7300096205BBA9BB29A4206D001980021F5F789
:10C740007FF96FF046001CE0843410220F49204628
:10C7500001F044F830B1102203A9204601F03EF860
:10C760000028EAD1019B30469968DA6801F068F840
:10C7700001980021F5F764F9019BD86801E06FF09A
:10C780007C0008B0BDE8F08100F8000825FE000834
:10C790002DE9F0410F4686B090461D46044628B963
:10C7A000002B7CD142490320F4F74CFA0AB100294E
:10C7B000F8D0ADB1EB8A13B96FF0150074E02846DC
:10C7C000FFF70EFF0028F7D12B68042B5ED16CB168
:10C7D000B4F87C2042B1AB8A33B19A4204D0EBE783
:10C7E000D4F88030002B54D0A36EF3B91822002166
:10C7F000684601F023F92F4A138803EB03166FEA0A
:10C8000086466FEA96460133B6B21380ACB1A4F8FF
:10C810007E6015B9D4F8803000E02B68A3663246FC
:10C820000421204600F0F0FA07E0182204F1680124
:10C830006846B4F87E6001F003F825B904F180057C
:10C84000B4F8964000E0EC8A009A2B680AB900938D
:10C8500001E09A42B0D10023394642461846F4F727
:10C86000FDFF0746C0B131462246FBF793F901466A
:10C8700018B93846F5F7E4F80EE011232A46694660
:10C8800000F03EFB00280FDD08380DE06FF0690076
:10C890000AE06FF07F0007E06FF00B0004E0002A71
:10C8A00088D0002986D17DE706B0BDE8F08100BFC1
:10C8B00000F80008C85D00207FB50C46054600B1B1
:10C8C00019B90D490320F4F7BDF90A4601AE232139
:10C8D00001F0B4F8304600F03BF90023B3FBF4F26A
:10C8E00004FB1232F15CA85C013341400C2BA954CB
:10C8F000F4D104B070BD00BF00F8000810B50446C4
:10C90000FFF7DAFF034B1A78511C19702378534054
:10C91000237010BD26020020062938B50C461546A6
:10C9200035D006D803291FD027D8A9B302290DD0A6
:10C9300091E0172948D004D808294FD0152930D0C4
:10C9400089E019293AD0252944D084E0012B03D865
:10C9500043490320F4F776F90A4600F1100128460E
:10C9600000F06EFF204638BD072BF1D900F112010F
:10C970000822284600F064FF70E0022BE8D1828B89
:10C98000520701D5082205E02B80184638BD022B3E
:10C99000DED1C2892A80F8E7022BD9D1C37E138069
:10C9A0000AE0012BD4D1838B13F0200F02D0012396
:10C9B0002B70EAE700232B70012038BD012BC7D173
:10C9C000838B13F0020FF1E7012BC1D190F90C20FA
:10C9D0002A70DAE7022BBBD10322DBE7072BB7D99A
:10C9E000838B5B074CBF0B4602234FF000024CBF0A
:10C9F00012301030042B6A702A7018D0082B03D024
:10CA0000022B2BD1134619E0027882F002022A7021
:10CA100042786A708278AA70C278EA7002792A71C4
:10CA200042796A718279AA71C279EA71ADE70378B5
:10CA300083F002032B7043786B700223FF210022E6
:10CA4000E970FE21AA7029716A71C25CAA7118444A
:10CA50004378EB7102E06FF0850038BD082038BDE7
:10CA600000F8000870B515461C46192968D8DFE89B
:10CA700001F00D6718283838486767676767676788
:10CA8000676767676767674D67606757022C03D002
:10CA90002E490320F4F7D6F81388FF2BF8D8C37675
:10CAA0004CE0022CF4D800F110060222002130469E
:10CAB00000F0C4FF22462946304600F0C1FE0220A5
:10CAC00070BD082CE4D800F112060822002130467F
:10CAD00000F0B4FF22462946304600F0B1FE08209F
:10CAE00070BD022CD4D11388022B06D0082B2AD17A
:10CAF000838B43F00403838320E0838B23F00403C0
:10CB00000CE0022CC4D11388C38117E01278838B08
:10CB100012B143F0200301E023F020038383CEE72A
:10CB20001278838B12B143F00203F7E723F002037C
:10CB3000F4E7012CACD192F900300373204670BDAC
:10CB40006FF0850070BD6FF0690070BD00F80008DF
:10CB50000C22014900F074BE107AFF1F10B586B098
:10CB600006AC04F8093D012301930DF1170300936E
:10CB70002346F5F70DFB9DF8170006B010BDF0B584
:10CB800085B01F4604AB002403F8012D01220546A1
:10CB90000E4601920094F5F7FBFA3B4622463146D9
:10CBA0002846FFF7DBFF05B0F0BD0000012101487A
:10CBB000F5F7E6BDCC5D00202DE9F04780460E4636
:10CBC000FFF7F4FF294C002514F8013C9E420AD1DE
:10CBD00032464146204600F001FE20B9244B122483
:10CBE00004FB053428E001350A2D04F11204EBD1D1
:10CBF000204B1B68092B33D81D4B0025122202FB4A
:10CC000005F91B4F19F803A0BAF1000F25D107EB66
:10CC1000090463789E4207D010225146A01C00F000
:10CC20000DFF07F809A06670122000FB0570324660
:10CC30004146023000F004FE23780F480133DBB296
:10CC4000012B08BF0B4A237002BF13680133136026
:10CC5000F5F7C6FD2046BDE8F08701350A2DCED197
:10CC60000548F5F7BDFD0020BDE8F087D65D002042
:10CC7000D45D0020D05D0020CC5D002010B50446BE
:10CC8000FFF794FF4CB123783BB1013BDBB223703B
:10CC90001BB9044A1368013B13600348BDE8104008
:10CCA000F5F79EBDD05D0020CC5D002070B5154627
:10CCB00006460C46FFF77AFF72782B6893420AD338
:10CCC000B11C204600F0BCFD73782B600548F5F7D9
:10CCD00087FD204670BD2A600248F5F781FD0020DF
:10CCE00070BD00BFCC5D00202DE9F041174606461F
:10CCF0008846FFF75BFF72783B68B3EBC20F05D144
:10CD0000B01C002501244FF0FF3316E02648F5F74C
:10CD100067FD6FF00100BDE8F081591C37D190F834
:10CD200000E018F80510714537D02B46C4B1BEFAA3
:10CD30008EF46409A4B1013501309542EDD33CB1C4
:10CD400000233B601848F5F74BFD0220BDE8F08159
:10CD50005D1C05D11448F5F743FD2046BDE8F08180
:10CD60001E4418F80310B2784A40072142FA01F431
:10CD7000E40748B202D40139F8D1084600EBC303F6
:10CD80003B600948F5F72CFD0120BDE8F081002C3F
:10CD9000E6D00478B4FA84F4CBE7002CCBD0B1FA17
:10CDA00081F46409C7E700BFCC5D002070B5FFF7D0
:10CDB000FDFE0A4C002504F1B40604F8025C04F8F8
:10CDC000015C204610220021123400F037FEB442EC
:10CDD000F3D10348BDE87040F5F702BDD65D0020F1
:10CDE000CC5D002013B5074A044692E803000022F8
:10CDF0008DE80300694604F11000FEF745FC02B01F
:10CE000010BD00BFAC20010803460846002110B445
:10CE100083E80600072401221C621A7203F1280429
:10CE200003F11002196159619961D9615C62DA609C
:10CE3000194610BCF8F716BD70B51C46531E0333D7
:10CE40000E4688B0114600F1100506D8294B079010
:10CE500003A80693F3F75AFE00E02AB1012201A9C4
:10CE60002846FEF75BFC05E001A92846FEF756FCC4
:10CE7000002838D003A8F3F737FEBDF8063040F29B
:10CE8000012293420CD048F2744293422ED1029A6E
:10CE9000194B9A4214BF6FF003006FF0730027E044
:10CEA000029D02212846F8F756FD10B1C368272BD2
:10CEB00003D812490320F3F7C5FE81681022083118
:10CEC000201D00F0BDFC042323604FF0FF312846F5
:10CED000F8F741FD08B9A08202E083685B88A3826D
:10CEE0003560002004E06FF00A0001E06FF00300FD
:10CEF00008B070BDE5CD0008630B8AF300F80008A8
:10CF00002DE9F0478946064690469A460146002498
:10CF100019B1CB6849681C44FAE7D9F80030D8F851
:10CF20000020934216D1042B14D108F1040209F118
:10CF300004013046FFF72EF90746C8B396F91050A2
:10CF40000DB902253574BB6883F806A0B9F81460E2
:10CF500056B906E03046F4F773FD6FF06900BDE89E
:10CF6000F087B8F8146086B1002319461A461846AF
:10CF7000F8F742FC36B2014618B93846F4F760FDBE
:10CF800016E08B685E804F600F460B493B4640F2CF
:10CF900002222846F8F792FA014630B93846F4F7EB
:10CFA0004FFD6FF04C00BDE8F0872046BDE8F087EC
:10CFB0006FF00B00BDE8F0870000FFFFD0400B1CB6
:10CFC000D1409C46203AD340184352426346934096
:10CFD0001843704753B94AB9002908BF00281CBF3D
:10CFE0004FF0FF314FF0FF3000F07EB9ADF1080C8B
:10CFF0006DE904CE00F006F8DDF804E0DDE9022377
:10D0000004B070472DE9F0478C460E460446089D53
:10D01000002B50D18A4217466CD9B2FA82FEBEF17B
:10D02000000F0BD0CEF1200420FA04F401FA0EF622
:10D0300044EA060C02FA0EF700FA0EF44FEA17491A
:10D04000220CBCFBF9F01FFA87F809FB10C642EA74
:10D05000064600FB08F3B34209D9F61900F1FF3286
:10D0600080F02281B34240F21F8102383E44F61A1A
:10D07000A2B2B6FBF9F309FB136642EA064403FBCE
:10D0800008F8A04509D9E41903F1FF3280F00A81BC
:10D09000A04540F20781023B3C44C8EB040443EA4C
:10D0A00000400021002D62D024FA0EF400232C60F1
:10D0B0006B60BDE8F0878B4207D9002D55D0002169
:10D0C00085E841000846BDE8F087B3FA83F10029FE
:10D0D00040F09080B34202D3824200F2F880841A7A
:10D0E00066EB03060120B446002D40D085E8101001
:10D0F000BDE8F08712B90127B7FBF2F7B7FA87FE50
:10D10000BEF1000F35D1F31B4FEA17481FFA87FC19
:10D110000121B3FBF8F0220C08FB103642EA064668
:10D120000CFB00F3B34207D9F61900F1FF3202D22B
:10D13000B34200F2CE801046F61AA2B2B6FBF8F364
:10D1400008FB136642EA06440CFB03FCA44507D91E
:10D15000E41903F1FF3202D2A44500F2B580134670
:10D16000CCEB040443EA00409CE729462846BDE88E
:10D17000F087CEF1200106FA0EF307FA0EF720FA37
:10D1800001F94FEA1748CE4049EA0309B6FBF8FA1D
:10D190004FEA194408FB1A661FFA87FC44EA064363
:10D1A0000AFB0CF29A4200FA0EF40AD9DB190AF1D2
:10D1B000FF3180F087809A4240F28480AAF1020A0F
:10D1C0003B449B1A1FFA89F9B3FBF8F108FB1133B2
:10D1D00049EA034301FB0CF69E4207D9DB1901F132
:10D1E000FF326BD29E4269D902393B449B1B41EA14
:10D1F0000A418EE7C1F1200E22FA0EF48B40234340
:10D2000020FA0EF706FA01F44FEA134C26FA0EF64E
:10D210003C43B6FBFCF9270C0CFB19661FFA83F89C
:10D2200047EA064609FB08F7B74202FA01F200FA9C
:10D2300001FA08D9F61809F1FF3041D2B7423FD9B7
:10D24000A9F102091E44F61BA0B2B6FBFCF40CFBCC
:10D25000146640EA064704FB08F8B84507D9FF18EA
:10D2600004F1FF3028D2B84526D9023C1F4444EAD5
:10D270000940C8EB0707A0FB02894F4544464E46CC
:10D2800014D329D065B3BAEB040367EB060707FA9A
:10D290000EFECB40CF404EEA030385E88800002114
:10D2A000BDE8F0871346F8E61046E0E6B8EB020466
:10D2B00069EB03060138E5E70446D8E7114695E730
:10D2C0008146C0E78A467CE7023B3C4448E7084683
:10D2D0000AE702383E442FE7C245E7D33E46D1E78E
:10D2E0002946BDE8F08700BF704700BF0A22002131
:10D2F00001F03EB90A23002201F0A6B8014B1868DC
:10D30000704700BF280200208B891A072DE9F041E1
:10D310000D46804635D44A68002A6BDDEC6A002C45
:10D3200047D003F48052002192B2D8F80060C8F8C8
:10D330000010002A62D06A6D5F0705D569686B6BC3
:10D34000521A0BB12B6CD21A0023296A4046A0470F
:10D35000441C39D0AB892A692A60DB044FF00002F3
:10D360006A6045D4696BC8F8006011B305F14403E5
:10D37000994202D0404600F0AFFB00206863BDE850
:10D38000F0810E69AEB10C680E6098070CBF4B6956
:10D390000023A41B8B600AE023463246AF6A296A49
:10D3A0004046B8470028A4EB0004064404DD002CE6
:10D3B000F2DC0020BDE8F081AB8943F04003AB8193
:10D3C0004FF0FF30BDE8F081D8F800201D2AF3D8D7
:10D3D000184BD34003F0010383F00101002BEBD085
:10D3E000AB892C696960D9042C60BBD5002AB9D1FE
:10D3F0006865B7E70A6C002A90DCDAE70123296A3E
:10D400004046A047431C024602D0AB89EC6A93E732
:10D41000D8F80030002BF8D01D2B01D0162B02D1EC
:10D42000C8F80060C5E7AB8943F04003AB81BDE8B5
:10D43000F08100BF010040200B6933B310B50446F2
:10D4400082B008B18369ABB1114B994219D0114B2D
:10D45000994218D0104B994208BFE168B1F90C30DD
:10D4600013B9002002B010BD204602B0BDE8104044
:10D47000FFF74ABF019100F019F90199044B994255
:10D48000E5D16168EAE7A168E8E70020704700BFDE
:10D49000F4200108D4200108B420010820B1054B74
:10D4A00001461868FFF7C8BF034B0449186800F02D
:10D4B00043B900BF280200201421010839D4000814
:10D4C00000207047014900F037B900BF39D4000887
:10D4D0000020704770B568234D1E03FB05F50E460E
:10D4E00005F1740100F03EFB044640B100210C3010
:10D4F000666005F168022160A06000F09FFA204696
:10D5000070BD00BF1F4B70B51D68AB69064613B9EF
:10D51000284600F039F848356B68AC68013B05D502
:10D5200021E0013B5A1C04F168041CD0B4F90C2022
:10D53000002AF6D1002501234FF6FF72E281A38174
:10D5400065662560A560656025616561A561294600
:10D55000082204F15C0000F071FA6563A563A5641C
:10D56000E564204670BD2B680BB11D46D4E704214D
:10D570003046FFF7AFFF286008B10546CCE70C2323
:10D58000336070BD142101083D4B3E491A682DE9F6
:10D59000F04F90424FF000038364C364036508BFFB
:10D5A000012383B008BF836181620746FFF7AAFFAA
:10D5B00078603846FFF7A6FFB8603846FFF7A2FF4D
:10D5C0007D68F86000240423AB812C606C60AC6043
:10D5D0006C66EC812C616C61AC61214605F15C00EC
:10D5E000082200F02BFABE68DFF89CB0DFF89CA0A0
:10D5F000DFF89C90DFF89C80C5F824B00123092255
:10D60000C5F828A0C5F82C90C5F830802D622146B9
:10D61000F381B28134607460B460746634617461A3
:10D62000B46106F15C000822019300F007FAFD687E
:10D63000366212200222C6F824B0C6F828A0C6F826
:10D640002C90C6F830802146A881EA812C606C605D
:10D65000AC606C662C616C61AC6105F15C00082209
:10D6600000F0ECF9019B2D62C5F824B0C5F828A0A4
:10D67000C5F82C90C5F83080BB6103B0BDE8F08FD1
:10D6800014210108C5D40008E1DD000809DE000806
:10D6900045DE000865DE0008024B0349186800F00B
:10D6A0004BB800BF1421010839D40008836903B9BD
:10D6B0006AE77047704700BF704700BF704700BF00
:10D6C000704700BF024B0349186800F00FB800BF55
:10D6D00028020020D1D40008024B0349186800F04A
:10D6E00005B800BF28020020C1D400082DE9F04190
:10D6F00010F148071BD0884600267D68BC68013DB4
:10D700000FD4A389012B05F1FF3506D9B4F90E30EA
:10D710000133204601D0C04706436B1C04F1680466
:10D72000EFD13F68002FE8D13046BDE8F0813E469A
:10D730003046BDE8F08100BF2DE9F84310F14807FD
:10D740001FD0884606464FF000097D68BC68013D41
:10D7500011D4A389012B05F1FF3508D9B4F90E3096
:10D7600001332146304602D0C04749EA00096B1C0C
:10D7700004F16804EDD13F68002FE6D14846BDE8CA
:10D78000F883B9464846BDE8F88300BF70B50F4E30
:10D790000F4D761BB61018BF002405D0013455F884
:10D7A000043B9847A642F9D10A4E0B4D761BF2F77F
:10D7B000EDFCB61018BF002406D0013455F8043B28
:10D7C0009847A642F9D170BD70BD00BF5C22010828
:10D7D0005C2201085C2201085C220108032A70B463
:10D7E00026D940EA01039B0711D004780D78AC429A
:10D7F00022D10244431C05E013F8014B11F8015FEC
:10D80000AC4219D19342F7D1002070BC70470C464E
:10D8100003461E682568AE421846214603F10403FC
:10D8200004F10404E1D1043A032A18462146F0D851
:10D83000002ADAD11046E8E7601B70BC704700BFD1
:10D84000844641EA000313F003036DD1403A41D30B
:10D8500051F8043B40F8043B51F8043B40F8043BCA
:10D8600051F8043B40F8043B51F8043B40F8043BBA
:10D8700051F8043B40F8043B51F8043B40F8043BAA
:10D8800051F8043B40F8043B51F8043B40F8043B9A
:10D8900051F8043B40F8043B51F8043B40F8043B8A
:10D8A00051F8043B40F8043B51F8043B40F8043B7A
:10D8B00051F8043B40F8043B51F8043B40F8043B6A
:10D8C00051F8043B40F8043B51F8043B40F8043B5A
:10D8D000403ABDD2303211D351F8043B40F8043BFA
:10D8E00051F8043B40F8043B51F8043B40F8043B3A
:10D8F00051F8043B40F8043B103AEDD20C3205D30A
:10D9000051F8043B40F8043B043AF9D2043208D001
:10D91000D2071CBF11F8013B00F8013B01D30B8873
:10D9200003806046704700BF082A13D38B078DD051
:10D9300010F003038AD0C3F10403D21ADB071CBF23
:10D9400011F8013B00F8013B80D331F8023B20F88D
:10D95000023B7BE7043AD9D3013A11F8013B00F8C6
:10D96000013BF9D20B7803704B7843708B7883704E
:10D97000604670478842F0B50DD98B1898420AD29C
:10D980008118002A51D09A1A13F8014D01F8014D5F
:10D990009342F9D1F0BD0F2A48D941EA00039B0711
:10D9A00046D100F1100401F11003154653F8106C34
:10D9B00044F8106C53F80C6C44F80C6C53F8086C79
:10D9C00044F8086C103D53F8046C44F8046C0F2DB7
:10D9D00003F1100304F11004E8D8A2F1100323F0BE
:10D9E0000F0302F00F0E1033BEF1030F194403446E
:10D9F00021D91E1F0D467446043C55F8047B46F899
:10DA0000047F032CF8D8AEF1040424F0030404349A
:10DA10002344214402F0030262B1013B0A4411F89D
:10DA2000014B03F8014F8A42F9D1F0BD0346F3E7F9
:10DA30000346F2E7F0BD7246EEE700BF70B484071C
:10DA400046D0541E002A41D0CDB2034602E0621EE9
:10DA5000E4B3144603F8015B9A07F8D1032C2ED9DE
:10DA6000CDB245EA05250F2C45EA054519D903F144
:10DA700010022646103E0F2E42F8105C42F80C5C55
:10DA800042F8085C42F8045C02F11002F2D8A4F1FA
:10DA9000100222F00F0204F00F041032032C134482
:10DAA0000DD91E462246043A032A46F8045BFAD8EA
:10DAB000221F22F003020432134404F003042CB1A9
:10DAC000C9B21C4403F8011BA342FBD170BC7047D0
:10DAD00014460346C2E700BF30B481B151F8043C9C
:10DAE0000439002BB8BFC9181D4B1A682AB18A42E5
:10DAF0000AD908680C18A24225D04A60196030BCC7
:10DB000070478B4203D81A465368002BF9D114682A
:10DB100015198D420CD007D808680C189C4218D0F3
:10DB20004B6030BC516070470C23036030BC7047C1
:10DB300009680C44111999421460E0D10ACB0C44D5
:10DB400053601460DBE7146852684A602044086040
:10DB5000D4E71C685B684B60204408605160CEE7E6
:10DB6000885E002070B5CD1C25F0030508350C2D0E
:10DB700038BF0C25002D06463BDBA94239D8274982
:10DB80000A6852B113685B1B04D436E023685B1B40
:10DB90001AD522465468002CF8D149681F4C002938
:10DBA00036D029463046F2F7F5FA431C21D0C41C82
:10DBB00024F00304A04205D0211A3046F2F7EAFA15
:10DBC000013016D0256004E00B2B0DD923601C44D6
:10DBD000256004F10B0020F00700231DC31A02D0BA
:10DBE0005A42E25070BD70BD94420ED063685360DB
:10DBF000EFE70C233360002070BD0B2B03D8536874
:10DC000014460B60E5E71446E0E713461446F8E7D0
:10DC10003046F2F7BFFA6060C3E700BF885E0020BD
:10DC20000EB410B5044683B018B183690BB9FFF781
:10DC30003DFD06A803460190059AA168204600F024
:10DC4000DFFE03B0BDE8104003B070470FB410B55D
:10DC50000A4B1C6882B024B1A36913B92046FFF7B0
:10DC600025FD05A803460190049AA168204600F00E
:10DC7000C7FE02B0BDE8104004B070472802002083
:10DC80002DE9F0410E46804600283ED08369002BE6
:10DC900039D084682F4B9C4243D02F4B9C4256D0A6
:10DCA0002E4B9C4208BFD8F80C40A3891B073DD5DA
:10DCB0002369002B3AD0013EA36816F8015F013BAF
:10DCC000A360B5B1002B04DB23685A1C22601D70D1
:10DCD000F2E7A769BB4222462946404601DB0A2DEE
:10DCE000F2D100F003FD0130E6D14FF0FF30BDE886
:10DCF000F081002B21DB23680A22591C21601A7055
:10DD00001046BDE8F081FFF7D1FCD8F81830D8F8FC
:10DD10000840002BBED14046FFF7C8FC0D4B9C428B
:10DD2000BBD1D8F80440A3891B07C1D42146404683
:10DD300000F03EFD0028BED0D7E7224640460A212B
:10DD400000F0D4FC0130D0D00A20BDE8F081D8F832
:10DD50000840AAE7F4200108D4200108B4200108F3
:10DD6000024B01461868FFF78BBF00BF2802002056
:10DD700038B50C46054608B18369B3B1114B9C42D6
:10DD800018D0114B9C4217D0104B9C4208BFEC6836
:10DD90002846214601F06AF980B994E80C00013B5D
:10DDA000511C84E80A00107838BDFFF77FFC054B52
:10DDB0009C42E6D16C68EBE7AC68E9E74FF0FF30D6
:10DDC00038BD00BFF4200108D4200108B4200108A8
:10DDD000024B01461868FFF7CBBF00BF28020020A6
:10DDE00010B50C46B1F90E10F2F7F2F9002803DB7A
:10DDF000636D0344636510BDA38923F48053A3813D
:10DE000010BD00BF002070472DE9F0411646B1F962
:10DE10000C201F46D3050C46054607D500220223D9
:10DE2000B1F90E10F2F7E1F9B4F90C20B4F90E10C3
:10DE300022F48052A2813B4632462846BDE8F0419A
:10DE4000F2F7CAB910B50C46B1F90E10F2F7CDF9D8
:10DE5000A389421C0EBF23F4805343F480536065B2
:10DE6000A38110BDB1F90E10F2F7BAB970B411F078
:10DE7000FF0434D085070FD00378002B5AD09C4282
:10DE80002BD0431C05E013F8012B002A4FD09442FD
:10DE900023D09A071846F6D10E0206F47F46264391
:10DEA000036846EA064601E050F8043F86EA0305A7
:10DEB000A5F10132A3F1013122EA050221EA0303AF
:10DEC000134313F0803FEFD0037823B932E010F80A
:10DED000013F002B2ED09C42F9D170BC70478407C3
:10DEE0000BD00378002BF8D0431C03E002780133F9
:10DEF000002AF2D099071846F8D10268A2F101333E
:10DF000023EA020313F0803F08D150F8042FA2F156
:10DF1000013323EA020313F0803FF6D00378002B8D
:10DF2000DBD010F8013F002BFBD170BC70471046CE
:10DF300070BC7047184670BC704700BF00000000FE
:10DF4000A2EB0300704700BF02780B78012A28BFBC
:10DF50009A42F5D16DE9044540EA0104CDE9026732
:10DF60006FF0000C4FEA447212B380EA010414F01F
:10DF7000070F6AD100F0070420F0070004F0030542
:10DF800021F007014FEAC505F0E8042314F0040F5F
:10DF9000F1E804670CFA05F462EA040266EA040692
:10DFA0000AD063EA0403624667EA0407664603E0B0
:10DFB000F0E80423F1E8046782FA4CF582EA0604EB
:10DFC000A4FA8CF46CBB83FA4CF583EA0705A5FA36
:10DFD0008CF595B950E9022351E9026782FA4CF5B4
:10DFE00082EA0604A4FA8CF483FA4CF583EA070566
:10DFF000A5FA8CF52543DBD09CB92DBAB5FA85F48A
:10E0000024F0070427FA04F1DDE9026723FA04F398
:10E0100003F0FF0001F0FF01FDE80445A0EB010063
:10E02000704724BAB4FA84F424F0070426FA04F101
:10E03000DDE9026722FA04F202F0FF0001F0FF01BD
:10E04000FDE80445A0EB0100704714F0030F3CD13C
:10E0500010F0030428D150F8082B51F8083B82FA3D
:10E060004CF582EA0305A5FA8CF55DB950F8042C4D
:10E0700051F8043C82FA4CF582EA0305A5FA8CF5C6
:10E08000002DE8D02DBAB5FA85F424F0070423FA60
:10E0900004F122FA04F202F0FF0001F0FF01FDE8B2
:10E0A0000445A0EB010070474FEAC40420F00300D0
:10E0B00050F8082B21F0030151F8083B0CFA04F446
:10E0C00062EA040263EA0403C9E710F003041AD009
:10E0D000A1EB040120F00300E40750F8042B06D064
:10E0E0000FD28B785FFAA2F4E41A06D12BB1CB7869
:10E0F0005FFAB2F4E41A00D11BB920465DF8104B68
:10E10000704701F1040150F8042BCC0721F0030102
:10E1100051F8043B48D824D222F07F4482FA4CF5CF
:10E1200094EA1325A5FA8CF50AD165B951F8043B98
:10E1300084EA0204B4EB036F0ED150F8042BEBE732
:10E140004FEA132355E035F07F454DD10878FDE8BF
:10E150000445C0F1000070474FEA126203F0FF036C
:10E1600047E002EA1C4482FA4CF594EA1345A5FA0A
:10E170008CF50AD165B951F8043B84EA0204B4EB8A
:10E18000034F0CD150F8042BEBE74FEA134330E078
:10E1900015EA1C4528D10B884FEA124229E04FEAC4
:10E1A000124203EA1C4324E002F0FF0482FA4CF519
:10E1B00094EA1365A5FA8CF50AD165B951F8043BC8
:10E1C00084EA0204B4EB032F09D150F8042BEBE7E7
:10E1D0004FEA13630DE015F0FF0F05D10B684FEA0E
:10E1E000122223F07F4304E04FF00000FDE80445D5
:10E1F000704712BA1BBA82FA4CF482EA0304A4FAFA
:10E200008CF5B5FA85F402FA04F203FA04F34FEA46
:10E210001260FDE80445A0EB1360704780EA01023C
:10E22000844612F0030F4FD111F0030F32D14DF895
:10E23000044D11F0040F51F8043B0BD0A3F101324F
:10E240009A4312F0803F04BF4CF8043B51F8043B62
:10E2500016D100BF51F8044BA3F101329A4312F0DA
:10E26000803FA4F101320BD14CF8043BA24312F0E1
:10E27000803F04BF51F8043B4CF8044BEAD02346DE
:10E280000CF8013B13F0FF0F4FEA3323F8D15DF890
:10E29000044B704711F0010F06D011F8012B0CF858
:10E2A000012B002A08BF704711F0020FBFD031F8D0
:10E2B000022B12F0FF0F16BF2CF8022B8CF8002057
:10E2C00012F47F4FB3D1704711F8012B0CF8012BDA
:10E2D000002AF9D1704700BF0000000000000000D4
:10E2E000000000000000000000000000000000002E
:10E2F000000000000000000000000000000000001E
:10E3000090F800F06DE9024520F007016FF0000C75
:10E3100010F0070491F820F040F049804FF000041D
:10E320006FF00700D1E9002391F840F000F10800F8
:10E3300082FA4CF2A4FA8CF283FA4CF3A2FA8CF330
:10E340004BBBD1E9022382FA4CF200F10800A4FA97
:10E350008CF283FA4CF3A2FA8CF3E3B9D1E90423EB
:10E3600082FA4CF200F10800A4FA8CF283FA4CF322
:10E37000A2FA8CF37BB9D1E9062301F1200182FADC
:10E380004CF200F10800A4FA8CF283FA4CF3A2FAE2
:10E390008CF3002BC6D0002A04BF04301A4612BAF0
:10E3A000B2FA82F2FDE8024500EBD2007047D1E9F3
:10E3B000002304F00305C4F100004FEAC50514F082
:10E3C000040F91F840F00CFA05F562EA05021CBF53
:10E3D00063EA050362464FF00004A9E7F0B420B3F6
:10E3E00007460D4617F8016B01E0A64216D015F856
:10E3F000014B002CF9D1EEB13E460C4616F8015BFC
:10E4000000E073B114F8013B9D42FAD15DB10023E5
:10E410003B70166006463046F0BC704763B1384624
:10E42000DEE73746E8E72E46F3E710680028D7D145
:10E430000646F0E71660EEE7176006460370EAE767
:10E440000123FFF7CBBF00BF2DE9F04F474C8346B8
:10E450000E46D4F800E000E02646344614F8015B8E
:10E460000EEB0500407800F0080000F0FF080028DF
:10E47000F2D12D2D5CD02B2D04BF7578B41C002B50
:10E480003ED0102B60D09A46B8F1000F0CBF6FF051
:10E4900000404FF000400027B0FBFAF9BC460AFBF1
:10E4A00019000CE0303DAB4219DD7E1C05D0CC4597
:10E4B00023D820D00AFB0C5C012714F8015B0EEB7B
:10E4C0000506767816F0040FECD116F0030606D098
:10E4D000012E14BF57263726AD1BAB42E5DC7B1C53
:10E4E00016D0B8F1000F10D16046002A39D0DFB93C
:10E4F0001160BDE8F08F8542DCDD4FF0FF37DCE7CF
:10E50000302D1AD00A239A46BEE7CCF1000CEBE777
:10E51000B8F1000F4FF022030CBF6FF000404FF036
:10E520000040CBF80030F2B1611E1160BDE8F08F01
:10E53000B41C75784FF00108A1E7237803F0DF03DE
:10E54000582B08D008239EE7302D9CD1207800F06E
:10E55000DF00582897D14FF0100A657853460234EF
:10E5600092E7BDE8F08FBDE8F08F00BF8C0200207D
:10E5700010B4044C13460A460146206810BCFFF74D
:10E5800063BF00BF280200202DE9F04F494C8246AE
:10E590000E46D4F800E000E02646344614F8015B4D
:10E5A0000EEB0500407800F0080000F0FF0C00289A
:10E5B000F2D12D2D54D02B2D04BF7578B41C5BB136
:10E5C000102B5ED04FF0FF38B8FBF3F803FB08FBCD
:10E5D0006FEA0B0B994607E0302D46D00A23DFF88F
:10E5E000D88099464FF0050B002738460CE0303DA7
:10E5F000AB4219DD7E1C05D0404522D81FD009FB57
:10E600000050012714F8015B0EEB0506767816F032
:10E61000040FECD116F0030606D0012E14BF5726C6
:10E620003726AD1BAB42E5DC002F0FDBBCF1000F42
:10E6300000D0404242B17FB91160BDE8F08F5D4526
:10E64000DDDD4FF0FF37DDE7BDE8F08F2223CAF8AC
:10E6500000304FF0FF305AB3611E1160BDE8F08FFB
:10E66000B41C75784FF0010CA9E7237803F0DF03A1
:10E67000582B0DD0082399464FF0070B6FF06048D8
:10E68000B2E7302D0ED1207800F0DF00582809D1F4
:10E690004FF0100965784B464FF00F0B02346FF0C6
:10E6A0007048A1E74FF00F0B6FF0704899469BE759
:10E6B000BDE8F08F8C0200209999991910B4044C90
:10E6C00013460A460146206810BCFFF75DBF00BF35
:10E6D0002802002010B4044C13460A460146206864
:10E6E00010BCF1F779BD00BF28020020F8B50E4636
:10E6F0001446054610B18369002B41D0254B9C423E
:10E7000043D0254B9C4242D0244B9C4208BFEC682E
:10E71000A389A269A2601A0721D52369FBB12268E7
:10E720006169D31A8B42F7B221DA0133A168501C18
:10E730000139A1602060167062699A4206D0A389EF
:10E74000DB0701D50A2F01D03846F8BD21462846FF
:10E75000FEF772FE0028F7D04FF0FF37F4E72146AE
:10E76000284600F025F80028F6D12369D7E721468E
:10E770002846FEF761FE0028EED122680123D5E786
:10E78000FEF794FF034B9C42BBD16C68C0E7AC68BA
:10E79000BEE700BFF4200108D4200108B42001081E
:10E7A000024B0A4601461868FFF7A0BF2802002066
:10E7B000384B70B51D6806460C4615B1AB69002B89
:10E7C00042D0354B9C4245D0344B9C4258D0344BC0
:10E7D0009C4208BFEC68B4F90C2093B219070CD521
:10E7E0002069A8B113F001021ED0636900225B42C8
:10E7F000A361A260F0B1002070BDDD0642D55807CC
:10E800002AD4206942F00803A3819BB20028E9D1F1
:10E8100003F42072B2F5007FE4D03046214600F0C8
:10E820006FF8A3892069DDE7990758BF6269A26084
:10E830000028E0D1B4F90C301A06DDD543F04003CE
:10E84000A3814FF0FF3070BD2846FEF72FFF124B1B
:10E850009C42B9D16C68BEE7616B51B104F14403CD
:10E86000994204D03046FFF737F9B4F90C20002361
:10E87000636300232069636022F024022060C1E703
:10E88000AC68A8E742F04002092333604FF0FF3044
:10E89000A28170BD28020020F4200108D4200108C4
:10E8A000B420010870B50C46B1F90E10002990B0E3
:10E8B00015461E4613DB01AAF1F79CFC00280EDB6F
:10E8C000029A02F47042A2F50052B2FA82F25209A0
:10E8D0004FF48063002032602B6010B070BDA389BC
:10E8E00000221B06326004D5402300202B6010B0AC
:10E8F00070BD4FF4806300202B6010B070BD00BF6E
:10E900008A8992070B4606D501F1470201211A6058
:10E910001A6159617047F0B583B001AB6A460C4685
:10E920000546FFF7BFFF009906462846FFF71AF98C
:10E93000B4F90C30D0B1019A124F0099AF6243F094
:10E940008003A3812060206161611AB93343A381F0
:10E9500003B0F0BD2846B4F90E10F1F750FCB4F93D
:10E960000C300028F2D043F00103EFE79A05EFD412
:10E9700004F1470243F002030121A38122602261D6
:10E980006161E5E7C5D400089368013B002B10B432
:10E99000936007DBCCB21368581C106019702046D6
:10E9A00010BC70479469A34202DBCCB20A2CF2D1AE
:10E9B00010BCFFF79BBE00BF93B1F8B514460F46DD
:10E9C0000646D51801E0AC4208D03A4614F8011BBF
:10E9D0003046FFF7D9FF431CF5D1F8BD0020F8BD44
:10E9E00000207047936810B5144613B95360184659
:10E9F00010BD00F0D1FB0023A360636010BD00BF19
:10EA00002DE9F04F9DB0884614460393814618B116
:10EA10008369002B00F00B818B4B984500F00D8132
:10EA20008A4B984500F00C81894B984508BFD9F86E
:10EA30000C80B8F80C301D0740F1EF80D8F810308A
:10EA4000002B00F0EA8030238DF82A302378814DA6
:10EA5000DFF804A20021202209918DF82920002B43
:10EA600000F08580252B264603D117E0252B00F0EA
:10EA7000868016F8013F002BF8D1B6EB040B76D058
:10EA800022465B4641464846FFF796FF01306ED06E
:10EA9000099B32785B440993002A68D000234FF029
:10EAA000FF31721C0493079306938DF853301A9329
:10EAB0000591012604E0049906FA03F30B4304933D
:10EAC000144664482178052200F0EAFC621C431BCE
:10EAD0000028F0D1049BD80644BF20228DF8532093
:10EAE0001907217844BF2B228DF853202A2968D09A
:10EAF000A1F13002092A0BD8079B14F8011F03EB80
:10EB0000830302EB4303A1F13002092AF5D90793ED
:10EB10002E293FD00322504800F0C2FC48B104998E
:10EB2000CAEB0000402202FA00F041EA000301347F
:10EB30000493217849488DF828100622013400F00A
:10EB4000AFFC00285FD0464BEBB103AB00934246CD
:10EB5000444B04A94846AFF3008007467A1C06D010
:10EB6000099B3B4409932378002B7FF47BAFB8F8D3
:10EB70000C305B0658D409981DB0BDE8F08FB6EB99
:10EB8000040B8BD07CE7039B073323F00703083388
:10EB90000393E5E761782A291DD0A1F13002002313
:10EBA000092A04F101040593B4D814F8011F03EBFA
:10EBB000830302EB4303A1F13002092AF5D905933F
:10EBC000A8E7039A116804320029039215DB079124
:10EBD000617801349CE7039B1A680592002A03F1CF
:10EBE00004030393B8BF4FF0FF3204F10203AEBF3A
:10EBF000A178A17805921C468CE7494243F00203B4
:10EC000007910493E4E703AB00934246154B04A934
:10EC1000484600F0CDF80746A0E741464846FFF7D2
:10EC2000C7FD00283FF40FAF4FF0FF30A4E7FEF719
:10EC30003DFD054B98457FF4F3AED9F80480F8E626
:10EC4000D9F80880F5E600BFF4200108D4200108B7
:10EC5000B420010820220108282201082C220108E2
:10EC600000000000B9E9000810B4044C13460A463D
:10EC70000146206810BCFFF7C3BE00BF2802002079
:10EC80002DE9F0470C4691460969A268DDF820801D
:10EC90008A42B8BF0A46C9F8002094F843100646D5
:10ECA0001F4611B10132C9F80020236899065DD5CD
:10ECB000D9F800200232C9F80020236813F0060FAB
:10ECC00019461DD1E1688A1A002AD8BF194617DDF6
:10ECD00004F1190A002505E0E368D9F800209B1A21
:10ECE000AB420CDD0123524639463046C047013065
:10ECF00005F10105F0D14FF0FF30BDE8F087216844
:10ED000094F84330003318BF01238A060AD5E1186E
:10ED10005A1C302081F84300224494F8451082F8B0
:10ED20004310023304F1430239463046C0470130F4
:10ED3000E1D0236803F00603042B29D0A3682269DD
:10ED40009342C8BF4FF000092FDD9B1A99441A3433
:10ED5000002501E04D4528D00123224639463046A2
:10ED6000C047013005F10105F4D1C4E713F0060FE7
:10ED700008D1E168D9F800208A1A002AD8BF1946BC
:10ED8000A6DCBDE794F84330003318BF0123C9E780
:10ED9000D9F80000E168A3682269091A934221EAC0
:10EDA000E179D2DCB9F1000FD1D10020BDE8F087C4
:10EDB0002DE9F0430C46097E85B06E2906461746BC
:10EDC0000C98984604F1430C5AD01AD8632900F0E5
:10EDD000128100F2D68000295CD0582940F0F580DD
:10EDE00084F8451022680368DFF864E2150603F131
:10EDF00004011ED4550653BF1B6801601B880160C7
:10EE000019E0732900F0CF807ED86F2900F0E480EC
:10EE1000702940F0DA80226842F0200222607823D4
:10EE200084F845300368DFF82CE2150603F104018D
:10EE3000E0D51B680160D00744BF42F02002226089
:10EE4000002B40F09080226822F0200222601021E6
:10EE5000002284F843206068A0600028C0F2888007
:10EE6000226822F004022260002B62D1002840F0C8
:10EE70008180654608296AD0C5EB0C0323610CE04C
:10EE800023681A0640F1D58003686269191D016084
:10EE90001B681A60002365462361CDF800803B465D
:10EEA00003AA21463046FFF7EBFE013021D02A4667
:10EEB000236939463046C04701301AD02368039889
:10EEC00013F0020FE36819D01A1A002A16DD04F1B4
:10EED0001909002504E0E36803981A1AAA420DDD17
:10EEE00001234A4639463046C047013005F1010545
:10EEF000F1D14FF0FF3005B0BDE8F0839842B8BFC4
:10EF0000184605B0BDE8F083752965D078295CD135
:10EF1000226884E76168A1602D200029C3F1000305
:10EF200084F8430021DB22F00402DFF824E12260B0
:10EF30000A216546B3FBF1F201FB123013461EF8BD
:10EF4000002005F8012D002BF4D1082994D1236865
:10EF5000D90791D5626823699A428DDC302305F880
:10EF6000013C013D88E7102172E7DFF8E4E00A2167
:10EF7000002BDED19EF8003084F8423004F14205C7
:10EF800078E7642901D069291FD122680368150632
:10EF900003F104013AD51B680160002BBADBDFF8EE
:10EFA000B0E00A2157E703686268191D01601D6817
:10EFB0000021284600F074FA002846D0401B60600B
:10EFC0002061002384F8433067E7012384F842106E
:10EFD000236104F14205F4E723681A061ED503688D
:10EFE0001A1D1B680260227EDFF864E06F2A14BFDE
:10EFF0000A2108212CE703681A68191D0123016002
:10F0000004F1420584F842202361DAE7550653BF34
:10F010001B680160B3F900300160BEE713F0400FD8
:10F02000036803F1040215BF02601B681B880260BD
:10F03000D9E713F0400F0368626903F1040101602E
:10F040001B6814BF1A801A6024E76068B8E700BF25
:10F050003422010848220108838903F00903092B9F
:10F0600001D000207047FEF719BA00BFF8B50C4672
:10F07000054610B18369002B45D0424B9C4247D0D6
:10F08000414B9C426FD0414B9C4208BFEC68B4F9A5
:10F090000C2093B200219F06616031D45E0722D517
:10F0A000616B61B104F14403994202D02846FEF736
:10F0B00013FD236C636000206063002B43D1236940
:10F0C000002B52D0B4F90C70BEB2B30722D1226922
:10F0D000226028466369656A216AA8470028606043
:10F0E00009DD0020F8BDD80644D519072ED442F01A
:10F0F0000402A281E3E7A3891DD143F02003A38189
:10F100004FF0FF30F8BDFEF7D1FA1E4B9C42B7D14D
:10F110006C68BCE71E4B1F4918680123A38106F0E9
:10F120000906FEF7E3FA092EA781D0D12146284629
:10F13000FEF7EAF8CBE7002243F04003A3816260C8
:10F140004FF0FF30F8BDE36B2360F8BD2146284641
:10F15000FEF772F90028D3D1B4F90C20A060A061A9
:10F1600022F00802C3E7AC6891E721462846FFF782
:10F17000C7FBA7E742F0400209232B604FF0FF30A6
:10F18000A281F8BDF4200108D4200108B4200108B0
:10F190001421010859F000089368002B76D02DE95E
:10F1A000F04F8B8985B00C4619070190164629D57A
:10F1B00022693AB303F002081FFA88F03568002884
:10F1C0002FD04FF00009B44FC846B246B845434669
:10F1D0004A4628BF3B460198B8F1000F50D0216A3B
:10F1E000A66AB047002871DDDAF808301B1A81449E
:10F1F000C0EB0808CAF80830002BE7D1002005B0A2
:10F20000BDE8F08F21460198FFF7D2FA002840F0C0
:10F210003A81A389356803F002081FFA88F00028B4
:10F22000CFD113F001095BD14F4602961FB39A0567
:10F23000D4F808802CD54745C246C0F0A48013F40A
:10F24000906F40F0B180206852464946FEF792FB2D
:10F25000A0682368C8EB00005344A06023603846D0
:10F26000029A93681B1A81443F1A9360002BC5D001
:10F27000A389002FDBD1D5F800906F680835D5E75A
:10F28000D5F80090D5F8048008359FE70020704736
:10F2900020682369984203D861698F4280F0B78063
:10F2A000B84528BFB84642464946FEF763FBA36807
:10F2B0002268C8EB03034244A3602260002B49D1BB
:10F2C00021460198FEF7B8F8002843D0B4F90C3075
:10F2D00043F040034FF0FF30A38105B0BDE8F08F4D
:10F2E0008046029082468146B9F1000F2AD0029BE7
:10F2F000002B4CD0206823696269C845C34628BFEB
:10F30000CB4698425F4604D9A36813449B4500F35B
:10F310009080934520DB1346A76A216A01985246E4
:10F32000B847071ED2DDB8EB070823D0B368DB1B54
:10F33000BA44C7EB0909B360002B3FF45FAFB9F1E2
:10F34000000FD4D10023D5F800A0D5F80490029383
:10F350000835C9E7404683E75A465146FEF70AFB9F
:10F36000A2682368CBEB02025B44B8EB0708A260FB
:10F370002360DBD121460198FEF75EF80028A5D175
:10F38000CDF80880D2E72068B846BA465CE74A461E
:10F390000A21504600F084F800286FD00130012384
:10F3A000CAEB00080293A5E762692068216902EBB5
:10F3B0004208C1EB000A08EBD8780AF101004FEAD5
:10F3C000680838444045424684BF804642465B0553
:10F3D00042D511460198FEF7C5FB8346002855D05B
:10F3E00052462169FEF72CFAA38923F4906343F077
:10F3F0008003A381CAEB08030BEB0A00C4F8148056
:10F40000C4F810B02060A360B846BA461CE76FF09D
:10F410000043BB4228BF3B464A4693FBF1F30198A9
:10F42000A66A01FB03F3216AB04700283FF718AF33
:10F430004CE71A4651460393FEF79CFA2268039B59
:10F4400001981A4422602146FDF7F6FF039B00282D
:10F450007FF43CAF1F4666E7019800F071F88346E1
:10F460000028C7D1019D21692846FEF735FBB4F974
:10F470000C300C2223F080032A6029E7012309F1D4
:10F480000108029336E74FF0FF30B8E6019A0C23EB
:10F490001360B4F90C301BE700FCFF7F0000000094
:10F4A00001F0FF01102A2BDB10F0070F08D010F835
:10F4B000013B013A8B422DD010F0070F42B3F6D139
:10F4C000F0B441EA012141EA014122F007047FF052
:10F4D00000070023F0E80256083C85EA010586EAA9
:10F4E000010685FA47F5A3FA87F586FA47F6A5FAE5
:10F4F00087F68EB9EED1F0BC01F0FF0102F00702F1
:10F5000032B110F8013B013A83EA010313B1F8D19B
:10F510000020704701387047002D06BF354603387C
:10F52000073815F0010F07D1013015F4807F02BFB5
:10F53000013015F4C03F0130F0BC0138704700BF06
:10F54000F9B1F8B506461546B2B10C4600F01CF804
:10F55000854201D82046F8BD29463046FEF702FB19
:10F56000074668B12A462146FEF76AF93046214629
:10F57000FEF7B2FA3846F8BDFEF7AEFA2846F8BDF7
:10F58000F8BD1146FEF7EEBA51F8040C0028BEBFD4
:10F59000091851F8043CC018043870474E4D4920F2
:10F5A00048414E444C4552004D454D204D414E4141
:10F5B00047452048414E444C455200425553204651
:10F5C00041554C542048414E444C455200555341FE
:10F5D0004745204641554C542048414E444C4552E5
:10F5E000004445425547204D4F4E2048414E444C23
:10F5F00045520044554D4D592048414E444C4552CA
:10F60000000A49535220737461636B206F766572F0
:10F61000666C6F77656400537461636B20706F690B
:10F620006E74657220636F727275707465642C20DD
:10F63000726573657420746F20746F70206F66201C
:10F64000737461636B000A436F6E74657874206233
:10F6500065666F726520686172646661756C743A84
:10F660000020202072303A2030782530386C780A1B
:10F6700020202072313A2030782530386C780A20EA
:10F68000202072323A2030782530386C780A2020D9
:10F690002072333A2030782530386C780A002020E8
:10F6A0007231323A2030782530386C780A202020A8
:10F6B0006C723A2030782530386C780A202020701F
:10F6C000633A2030782530386C780A2020707372C5
:10F6D0003A2030782530386C780A0A004653522F89
:10F6E0004641523A0020434653523A203078253062
:10F6F000386C780A0020484653523A20307825303A
:10F70000386C780A0020444653523A20307825302D
:10F71000386C780A0020414653523A203078253020
:10F72000386C780A0020424641523A203078253021
:10F73000386C780A004D4D4641523A2030782530D9
:10F74000386C780A004D697363004558435F524531
:10F75000543A2030782530386C780A00417474654A
:10F760006D7074696E6720746F207265636F6E735D
:10F77000747275637420737461746520666F72208F
:10F78000646562756767696E672E2E2E00496E206C
:10F790004744423A0A2020736574202470633D3048
:10F7A00078256C780A20206672616D6520300A2009
:10F7B0002062740A000A49535220737461636B20FB
:10F7C0006F766572666C6F7765642062792061740C
:10F7D000206C656173742025642062797465732ED2
:10F7E0000A0048415244204641554C542048414E5D
:10F7F000444C455200676E72635F6574686F7300B6
:10F800004641494C454420415353455254494F4E7B
:10F810002E0025700A002A2A2A2052494F54206BB4
:10F8200065726E656C2070616E69633A0A25730AB1
:10F830000A002A2A2A2068616C7465642E0A0A006C
:10F840006D61696E28293A205468697320697320B4
:10F8500052494F5421202856657273696F6E3A20C1
:10F86000323031382E30312D646576656C2D32376B
:10F870002D67386230302D64656269616E290A0037
:10F8800069646C65006D61696E000000250F0008F9
:10F890008D0E0008890E0008830E0008B10E0008C6
:10F8A000851B00087D5E7D5D676E72635F6E6574AB
:10F8B0006465763A20706F737369626C79206C6F3F
:10F8C000737420696E746572727570742E005F5166
:10F8D000F9F9000801FA00080AFA000813FA00080A
:10F8E00019FA000821FA00082AFA000833FA000879
:10F8F0003CFA000844FA00084CFA0008737461747A
:10F9000065006E616D650009706964207C20252D9D
:10F910003231737C20252D397351207C207072691F
:10F92000207C20737461636B2020282075736564CC
:10F9300029207C2062617365206164647220207CD0
:10F940002063757272656E7420202020200A0009E1
:10F9500020202D207C206973725F737461636B209B
:10F9600020202020202020202020207C202D20202E
:10F970002020202020202D207C2020202D207C20B5
:10F98000253669202825356929207C2025313070CD
:10F99000207C20253130700A000925336869207CDD
:10F9A00020252D323073207C20252D387320252EE4
:10F9B0003173207C20253369207C2025366920285E
:10F9C00025356929207C2025313070207C20253187
:10F9D0003070200A007C0053554D000925357320F6
:10F9E000252D3231737C253133732536732025362E
:10F9F000692028253569290A0073746F7070656461
:10FA000000736C656570696E6700626C206D75745B
:10FA1000657800626C20727800626C2073656E6499
:10FA200000626C207265706C7900626C20616E7986
:10FA3000666C00626C20616C6C666C00626C206DA0
:10FA4000626F780072756E6E696E670070656E64C5
:10FA5000696E67000044004000000200030002409D
:10FA60000200024007070026004800400000040092
:10FA7000090C0240080C0240070700270706040291
:10FA800001070705030200000030014007000240A3
:10FA9000060002400500024004000240050000008C
:10FAA0000010000001000000003800400F04024078
:10FAB0000E0402400D0402400C0402400500000048
:10FAC000004000000000000000000040FFFFFFFFBA
:10FAD00001000000001C0000000C0040FFFFFFFFC1
:10FAE0000800000000320000020252494F54206218
:10FAF0006F7264657220726F7574657220657861CB
:10FB00006D706C65206170706C69636174696F6E93
:10FB100000416C6C2075702C2072756E6E696E677A
:10FB200020746865207368656C6C206E6F770000C8
:10FB30000100000003000000060C02400210024019
:10FB4000070C02400A0C02405B6175746F5F696EBE
:10FB500069745F6E657469665D206572726F72208C
:10FB6000696E697469616C697A696E67206174385D
:10FB700036726632787820726164696F2023257549
:10FB80000A006174383672663278780069707636A9
:10FB900000293A11366C6F00FF7F3F1F0F070301EA
:10FBA00075647000676E72635F75686370633A2096
:10FBB000756863705F68616E646C655F70726566BE
:10FBC000697828293A2072656365697665642070D2
:10FBD00072656669782C2062757420646F6E277474
:10FBE000206B6E6F7720616E7920776972656C6526
:10FBF000737320696E746572666163650A00676E6F
:10FC000072635F75686370633A20756863705F68DC
:10FC1000616E646C655F70726566697828293A2048
:10FC200072656365697665642070726566697820BF
:10FC300066726F6D20756E6578706563746564209B
:10FC4000696E746572666163650A00676E72635FF0
:10FC500075686370633A20756863705F68616E648D
:10FC60006C655F70726566697828293A2063616EF9
:10FC70006E6F742067657420494944206F66207751
:10FC80006972656C65737320696E74657266616311
:10FC9000650A00676E72635F75686370633A20750A
:10FCA0006863705F68616E646C655F7072656669D9
:10FCB0007828293A20676F742073616D652070720F
:10FCC0006566697820616761696E0A00676E7263B4
:10FCD0005F75686370633A20756863705F68616E12
:10FCE000646C655F70726566697828293A20636F75
:10FCF0006E66696775726564206E657720707265DF
:10FD000066697820002F363400676E72635F75680D
:10FD10006370633A20756863705F68616E646C65D8
:10FD20005F70726566697828293A2072656D6F7612
:10FD30006564206F6C642070726566697820006667
:10FD40006538303A3A3200666538303A3A31006701
:10FD50006E72635F75686370633A205573696E678E
:10FD600020257520617320626F7264657220696E50
:10FD70007465726661636520616E6420257520611B
:10FD80007320776972656C65737320696E74657230
:10FD9000666163652E0A00676E72635F75686370E3
:10FDA000633A206F6E6C79206F6E6520696E7465A2
:10FDB000726661636520666F756E642C20736B6973
:10FDC0007070696E672073657475702E0A007568AF
:10FDD000637000FFFFFE80000000000000000000D4
:10FDE0000000000000FF0100000000000000000013
:10FDF0000000000001FF0200000000000000000001
:10FE00000000000001FF02000000000000000000F0
:10FE10000000000002FF02000000000000000000DF
:10FE200001FF0000000000000000000000000000D2
:10FE300000000000000000000000000000000000C2
:10FE40000000000001303132333435363738396143
:10FE500062636465660030313233343536373839A1
:10FE6000414243444546007368656C6C3A20696EB4
:10FE7000636F72726563742071756F74696E670069
:10FE800068656C70004465736372697074696F6E45
:10FE900000436F6D6D616E6400252D323073202537
:10FEA000730A007368656C6C3A20636F6D6D616EE8
:10FEB00064206E6F7420666F756E643A2025730A35
:10FEC000007265626F6F74005265626F6F742074A8
:10FED0006865206E6F6465007073005072696E749F
:10FEE0007320696E666F726D6174696F6E206162F6
:10FEF0006F75742072756E6E696E672074687265B6
:10FF00006164732E0070696E67360050696E6720F9
:10FF10007669612049434D5076360072616E646F98
:10FF20006D5F696E697400696E697469616C697A84
:10FF30006573207468652050524E470072616E648C
:10FF40006F6D5F6765740072657475726E732033D0
:10FF50003220626974206F662070736575646F204B
:10FF600072616E646F6D6E657373006966636F6E48
:10FF700066696700436F6E666967757265206E65B6
:10FF800074776F726B20696E7465726661636573F6
:10FF900000666962726F757465004D616E69707597
:10FFA0006C61746520746865204649422028696E3A
:10FFB000666F3A2027666962726F757465205B61AF
:10FFC00064647C64656C5D2729006E6361636865A9
:10FFD000006D616E616765206E65696768626F724A
:10FFE0002063616368652062792068616E640072D5
:10FFF0006F7574657273004950763620646566616A
:020000040801F1
:10000000756C7420726F75746572206C69737400FE
:100010003663747800364C6F5750414E20636F6ED4
:100020007465787420636F6E666967757261746950
:100030006F6E20746F6F6C00C1FE0008C8FE000870
:10004000ED860008D8FE0008DBFE0008F7860008F1
:1000500005FF00080BFF0008E19F00081BFF0008D8
:1000600027FF0008018700083CFF000847FF000841
:10007000398700086BFF000874FF0008598F0008DB
:1000800091FF00089AFF0008F9980008CAFF0008CD
:10009000D1FF0008F59B0008EFFF0008F7FF0008FC
:1000A000F59D00081000010815000108E9A50008E9
:1000B00000000000000000000000000050524E4709
:1000C00020696E697469616C697A656420746F2057
:1000D00063757272656E742074696D653A2025646B
:1000E0000A0050524E4720696E697469616C697AE2
:1000F000656420676976656E2076616C75653A2067
:1001000025640A004F464600534C45455000535461
:10011000414E4442590049444C45005258005458FD
:100120000052455345540025303878002873686FD5
:100130007274292061646472657373006C6F6E67FA
:10014000206164647265737300736F7572636520F8
:1001500061646472657373206C656E6774680063B4
:1001600068616E6E656C0070616765006E657477BE
:100170006F726B206964656E74696669657200549C
:100180005820706F776572205B696E2064426D5DE8
:10019000006D61782E2072657472616E736D697383
:1001A00073696F6E730043534D41207265747269B9
:1001B000657300434341207468726573686F6C64B3
:1001C000205B696E2064426D5D00656E63727970BC
:1001D00074696F6E00656E6372797074696F6E20FA
:1001E0006B65790075736167653A202573203C69FA
:1001F000665F69643E20736574203C6B65793E20C0
:100200003C76616C75653E0A00202020202020533A
:1002100065747320616E2068617264776172652015
:100220007370656369666963207370656369666985
:10023000632076616C75650A2020202020203C6BAD
:1002400065793E206D6179206265206F6E65206F53
:10025000662074686520666F6C6C6F77696E670ADC
:10026000202020202020202A202261646472222065
:100270002D2073657473202873686F727429206150
:100280006464726573730A202020202020202A20B5
:1002900022616464725F6C6F6E6722202D2073652B
:1002A0007473206C6F6E6720616464726573730A87
:1002B000202020202020202A2022616464725F7385
:1002C000686F727422202D20616C69617320666FE3
:1002D00072202261646472220A20202020202020C3
:1002E0002A20226368616E6E656C22202D20736562
:1002F000747320746865206672657175656E6379C4
:10030000206368616E6E656C0A202020202020200A
:100310002A20226368616E22202D20616C6961733E
:1003200020666F7220226368616E6E656C220A20FF
:100330002020202020202A202263736D615F7265B7
:10034000747269657322202D20736574206D617845
:100350002E206E756D626572206F66206368616E17
:100360006E656C2061636365737320617474656D81
:100370007074730A202020202020202A202263630A
:10038000615F7468726573686F6C6422202D2073DE
:100390006574204544207468726573686F6C6420CE
:1003A000647572696E672043434120696E20644220
:1003B0006D0A202020202020202A20226E6964221D
:1003C000202D207365747320746865206E657477C2
:1003D0006F726B206964656E746966696572202846
:1003E0006F72207468652050414E204944290A20CC
:1003F0002020202020202A20227061676522202DC5
:100400002073657420746865206368616E6E656C26
:100410002070616765202849454545203830322ED7
:1004200031352E34290A202020202020202A202285
:1004300070616E22202D20616C69617320666F727D
:1004400020226E6964220A202020202020202A20D9
:100450002270616E5F696422202D20616C69617376
:1004600020666F7220226E6964220A2020202020DC
:1004700020202A2022706F77657222202D20545868
:1004800020706F77657220696E2064426D0A2020AB
:1004900020202020202A202272657472616E73222F
:1004A000202D206D61782E206E756D626572206F33
:1004B000662072657472616E736D697373696F6EB5
:1004C000730A202020202020202A20227372635FBC
:1004D0006C656E22202D207365747320746865200E
:1004E000736F757263652061646472657373206CE9
:1004F000656E67746820696E20627974650A2020D1
:1005000020202020202A2022737461746522202D4F
:10051000207365742074686520646576696365205E
:1005200073746174650A202020202020202A202254
:10053000656E637279707422202D20736574207447
:10054000686520656E6372797074696F6E206F6E76
:100550002D6F66660A202020202020202A20226B72
:10056000657922202D207365742074686520656E7E
:100570006372797074696F6E206B657920696E2083
:1005800068657861646563696D616C20666F726D22
:1005900061740A00776972656400776972656C65D9
:1005A0007373004966616365202532642020002052
:1005B0004368616E6E656C3A202568752000205096
:1005C0006167653A202568752000204E49443A202D
:1005D0003078256878004C6F6E67204857616464F6
:1005E000723A2000257320000A202020202020209D
:1005F000202020002054582D506F7765723A202516
:10060000686964426D20002053746174653A20006B
:10061000206D61782E2052657472616E732E3A20BF
:10062000257520002043534D412052657472696541
:10063000733A202575200050524F4D4953432020D6
:10064000004155544F41434B20200041434B5F52E2
:1006500045512020005052454C4F4144202000522B
:1006600041574D4F444520200043534D4120200029
:100670004155544F4343412020004D41435F4E4F6D
:100680005F534C4545502020004D54553A25687520
:10069000202000484C3A2575202000364C4F202061
:1006A000005254522020005254525F4144562020A0
:1006B0000049504843202000536F757263652061E4
:1006C000646472657373206C656E6774683A202584
:1006D00068750A2020202020202020202020004C87
:1006E000696E6B20747970653A20257300696E65B8
:1006F000743620616464723A200025732F257520BA
:100700002073636F70653A20006C6F63616C0067E3
:100710006C6F62616C00205B6D756C7469636173F2
:10072000745D00205B616E79636173745D00657256
:10073000726F7220696E20636F6E76657273696F77
:100740006E00756E006572726F723A20756E61622E
:100750006C6520746F20736574206F7074696F6EA0
:1007600000737563636573733A2025737365742032
:100770006F7074696F6E0A006572726F723A2075DD
:100780006E61626C6520746F2070617273652061A8
:100790006464726573732E0A4D75737420626520EC
:1007A0006F6620666F726D6174205B302D39612D2C
:1007B00066412D465D7B327D283A5B302D39612DB7
:1007C00066412D465D7B327D292A0A28686578209E
:1007D00070616972732064656C696D697465642009
:1007E000627920636F6C6F6E7329006572726F722D
:1007F0003A20756E61626C6520746F207365742099
:1008000000737563636573733A2073657420002009
:100810006F6E20696E746572666163652025686914
:1008200020746F2025730A00206F6E20696E746536
:1008300072666163652025686920746F2025690AE6
:10084000006572726F723A20756E61626C65207419
:100850006F2070617273652076616C75652E0A4D2C
:1008600075737420626520612031362D62697420B1
:10087000756E7369676E656420696E74656765720D
:100880002028646563206F7220686578290A00203B
:100890006F6E20696E746572666163652025686994
:1008A00020746F20003078253034780A0075736129
:1008B00067653A202573203C69663E205B3C4C32DC
:1008C00020616464723E7C62636173745D203C6489
:1008D0006174613E0A006572726F723A20696E76C9
:1008E000616C696420696E74657266616365206716
:1008F0006976656E006263617374006572726F720F
:100900003A20696E76616C69642061646472657313
:100910007320676976656E006572726F723A207037
:1009200061636B6574206275666665722066756CBE
:100930006C006572726F723A20756E61626C652030
:10094000746F2073656E6400616464720061646436
:10095000725F73686F727400616464725F6C6F6E53
:1009600067006368616E006E69640070616E00709C
:10097000616E5F696400706F776572007372635FA8
:100980006C656E006F6666007265736574007374E3
:10099000616E6462790075736167653A20696663A8
:1009A0006F6E666967203C69665F69643E207365A7
:1009B00074207374617465205B6F66667C736C650C
:1009C00065707C69646C657C72657365747C737436
:1009D000616E6462795D006572726F723A20756E45
:1009E00061626C6520746F20736574207374617428
:1009F0006520746F2000737563636573733A2073A9
:100A00006574207374617465206F6620696E746507
:100A100072666163652025686920746F20007265C5
:100A20007472616E730063736D615F726574726975
:100A30006573006363615F7468726573686F6C648B
:100A400000656E6372797074004F4E007573616754
:100A5000653A206966636F6E666967203C69665F08
:100A600069643E2073657420656E63727970746981
:100A70006F6E205B6F6E7C6F66665D000A4E6F74F2
:100A80006963653A2073657474696E672035362032
:100A9000626974206B65792E000A4E6F7469636514
:100AA0003A2073657474696E672036342062697405
:100AB000206B65792E000A4E6F746963653A207366
:100AC000657474696E672031323820626974206BF6
:100AD00065792E000A4E6F746963653A20736574F8
:100AE00074696E672031393220626974206B6579D0
:100AF0002E000A4E6F746963653A207365747469D9
:100B00006E672032353620626974206B65792E005D
:100B10000A4E6F746963653A2073657474696E6711
:100B20002035313220626974206B65792E00657240
:100B3000726F723A20696E76616C6964206B6579B8
:100B40002073697A652E0A006572726F723A207599
:100B50006E61626C6520746F207061727365206BCA
:100B6000657900206F6E20696E74657266616365D9
:100B70002025686920746F200A00253032780061D2
:100B800064640075736167653A202573203C69666B
:100B90005F69643E20616464205B616E79636173A8
:100BA000747C6D756C7469636173747C756E696354
:100BB0006173745D203C697076365F616464723E77
:100BC0005B2F7072656669785F6C656E5D0A0061A7
:100BD0006E7963617374006D756C746963617374AD
:100BE00000756E6963617374006572726F723A208A
:100BF000756E61626C6520746F2070617273652020
:100C00004950763620616464726573732E00657294
:100C1000726F723A206164647265737320776173D6
:100C2000206E6F742061206D756C746963617374DC
:100C300020616464726573732E006572726F723A1C
:100C400020756E61626C6520746F20616464204958
:100C500050763620616464726573730A007375633D
:100C6000636573733A2061646465642025732F257E
:100C70006420746F20696E746572666163652025F7
:100C800068690A0064656C0075736167653A2025C0
:100C900073203C69665F69643E2064656C203C6932
:100CA0007076365F616464723E0A007375636365D3
:100CB00073733A2072656D6F7665642025732074B6
:100CC0006F20696E74657266616365202568690AC4
:100CD000006D74750075736167653A202573203C5B
:100CE00069665F69643E206D7475203C6E3E0A0043
:100CF0006572726F723A204D5455206D7573742071
:100D00006265206265747765656E2025687520616F
:100D10006E64202568750A006572726F723A2075DC
:100D20006E61626C6520746F20736574204D54553C
:100D30002E00737563636573733A20736574204D79
:100D4000545520257520696E74657266616365204F
:100D50002568690A00686C0075736167653A20252B
:100D600073203C69665F69643E20686C203C6E3E7F
:100D70000A006572726F723A20486F70206C696D5C
:100D80006974206D7573742062652062657477657F
:100D9000656E2025687520616E64202568750A00DF
:100DA0006572726F723A20756E61626C6520746F45
:100DB0002073657420686F70206C696D69742E00F3
:100DC000737563636573733A2073657420686F701D
:100DD000206C696D697420257520696E7465726672
:100DE000616365202568690A0070726F6D697363BD
:100DF000007072656C6F6164006175746F61636B24
:100E00000061636B5F726571007261770063736D7F
:100E100061006175746F636361006D61635F6E6F24
:100E20005F736C6565700069706863006572726FEE
:100E3000723A20756E61626C6520746F2028756E41
:100E40002973657420495048430073756363657363
:100E5000733A20656E61626C652049504843206F8B
:100E60006E20696E74657266616365202568690A23
:100E700000737563636573733A2064697361626CB0
:100E8000652049504843206F6E20696E7465726614
:100E9000616365202568690A007274725F61647617
:100EA000006572726F723A20756E61626C652074B3
:100EB0006F2028756E2973657420726F7574657262
:100EC000206164766572746973656D656E74206601
:100ED0006C61672E00737563636573733A20656E8A
:100EE00061626C6520726F757465722061647665ED
:100EF00072746973656D656E7473206F6E20696EB0
:100F000074657266616365202568690A007375639C
:100F1000636573733A2064697361626C6520726FF4
:100F200075746572206164766572746973656D6548
:100F30006E7473206F6E20696E746572666163658E
:100F4000202568690A0075736167653A202573205A
:100F50003C69665F69643E205B2D5D7B70726F6DDE
:100F60006973637C6175746F61636B7C61636B5FD4
:100F70007265717C63736D617C6175746F636361AD
:100F80007C6363615F7468726573686F6C647C70A6
:100F900072656C6F61647C6D61635F6E6F5F736CB3
:100FA0006565707C697068637C7274725F61647679
:100FB0007D0A0075736167653A202573205B3C6983
:100FC000665F69643E5D0A000A62726965663A207E
:100FD000616464732061206E657720656E74727938
:100FE00020746F20746865204649422E0A7573612B
:100FF00067653A20666962726F7574652061646422
:10100000203C64657374696E6174696F6E3E20760E
:101010006961203C6E65787420686F703E205B6467
:101020006576203C6465766963653E5D205B6C692E
:10103000666574696D65203C6C69666574696D658B
:101040003E5D0A202020202020203C6465737469C6
:101050006E6174696F6E3E202D2074686520646532
:101060007374696E6174696F6E2061646472657314
:10107000732077697468206F7074696F6E616C207B
:101080007072656669782073697A652C20652E67B1
:101090002E202F3131360A202020202020203C6EA7
:1010A00065787420686F703E202020202D207468A1
:1010B000652061646472657373206F66207468656F
:1010C000206E6578742D686F7020746F776172641C
:1010D0007320746865203C64657374696E6174691B
:1010E0006F6E3E0A202020202020203C6465766917
:1010F00063653E2020202020202D20746865206418
:101100006576696365206964206F66207468652070
:10111000496E7465726661636520746F20757365CE
:101120002E204F7074696F6E616C206966206F6E3F
:101130006C79206F6E6520696E7465726661636597
:1011400020697320617661696C61626C652E0A208A
:101150002020202020203C6C69666574696D653E06
:10116000202020202D206F7074696F6E616C206CC0
:1011700069666574696D6520696E206D7320776896
:10118000656E2074686520656E747279206175746F
:101190006F6D61746963616C6C7920696E76616CE6
:1011A0006964617465730A000A62726965663A204F
:1011B00064656C6574657320616E20656E74727908
:1011C0002066726F6D20746865204649422E0A754C
:1011D000736167653A20666962726F757465206431
:1011E000656C203C64657374696E6174696F6E3EF2
:1011F0000A202020202020203C64657374696E61E1
:1012000074696F6E3E202D20746865206465737468
:10121000696E6174696F6E206164647265737320B6
:101220006F662074686520656E74727920746F2013
:1012300062652064656C657465640A00666C75732C
:1012400068007375636365737366756C6C7920668B
:101250006C757368656420616C6C20656E7472696E
:101260006573000A736565203C666962726F757408
:1012700065205B6164647C64656C5D3E20666F72B2
:10128000206D6F726520696E666F726D6174696F33
:101290006E0A3C666962726F75746520666C757360
:1012A00068205B696E746572666163655D3E20727D
:1012B000656D6F76657320616C6C20656E74726904
:1012C0006573205B6173736F636961746564207714
:1012D00069746820696E746572666163655D0A0091
:1012E0000A756E7265636F676E697A6564207061F6
:1012F00072616D65746572322E0A506C656173653A
:1013000020656E74657220666962726F75746520FF
:101310005B6164647C64656C5D20666F72206D6FD8
:10132000726520696E666F726D6174696F6E2E00F2
:101330007375636365737366756C6C7920666C7521
:101340007368656420616C6C20656E747269657386
:1013500020666F7220696E74657266616365202510
:1013600068750A00696E7465726661636520256838
:101370007520646F6573206E6F742065786973746F
:101380000A00766961000A62726965663A206164E2
:1013900064732061206E657720656E7472792074A5
:1013A0006F20746865204649422E0A75736167652F
:1013B0003A20666962726F75746520616464203CCE
:1013C00064657374696E6174696F6E3E20766961DD
:1013D000203C6E65787420686F703E205B64657693
:1013E000203C6465766963653E5D0A2020202020EC
:1013F00020203C64657374696E6174696F6E3E2071
:101400002D207468652064657374696E6174696FFA
:101410006E20616464726573732077697468206FED
:101420007074696F6E616C20707265666978207384
:10143000697A652C20652E672E202F3131360A20DF
:101440002020202020203C6E65787420686F703E3C
:10145000202020202D2074686520616464726573EB
:1014600073206F6620746865206E6578742D686FD0
:101470007020746F776172647320746865203C64B7
:10148000657374696E6174696F6E3E0A2020202056
:101490002020203C6465766963653E202020202062
:1014A000202D207468652064657669636520696411
:1014B000206F662074686520496E7465726661638A
:1014C0006520746F207573652E204F7074696F6E80
:1014D000616C206966206F6E6C79206F6E65206983
:1014E0006E746572666163652069732061766169F7
:1014F0006C61626C652E0A006C69666574696D6565
:1015000000646576000A756E7265636F676E697A4E
:10151000656420706172616D65746572732E0A5026
:101520006C6561736520656E7465722066696272B0
:101530006F757465205B6164647C64656C5D2066B6
:101540006F72206D6F726520696E666F726D617467
:10155000696F6E2E00554E4D414E41474544202047
:101560002000554E524541434841424C45200049D8
:101570004E434F4D504C4554452020005354414C50
:1015800045202020202020200044454C4159202087
:1015900020202020200050524F4245202020202093
:1015A000202000524541434841424C452020200024
:1015B000554E4B4E4F574E202020202000474300D1
:1015C00054454E54005245470049507636206164D8
:1015D000647265737320202020202020202020208A
:1015E000202020202020202020696620204C32202E
:1015F00061646472657373202020202020202020E5
:101600002020202020202073746174652020202059
:1016100020202074797065002D2D2D2D2D2D2D2D40
:101620002D2D2D2D2D2D2D2D2D2D2D2D2D2D2D2DEA
:101630002D2D2D2D2D2D2D2D2D2D2D2D2D2D2D2DDA
:101640002D2D2D2D2D2D2D2D2D2D2D2D2D2D2D2DCA
:101650002D2D2D2D2D2D2D2D2D2D2D2D2D2D2D2DBA
:101660002D2D2D2D2D2D00252D33307320202532AD
:1016700068692020252D3234732020006572726F36
:10168000723A20696E76616C696420696E74657265
:101690006661636520676976656E2E006572726F9C
:1016A000723A20756E61626C6520746F2070617291
:1016B0007365206C696E6B2D6C6179657220616455
:1016C00064726573732E006572726F723A20756E64
:1016D00061626C6520746F2061646420616464726F
:1016E00065737320746F206E65696768626F72201E
:1016F00063616368652E00737563636573733A2075
:101700006164646564204950763620616464726562
:10171000737320257320746F206E65696768626F2C
:10172000722063616368650A007375636365737330
:101730003A2072656D6F7665642025732066726F3E
:101740006D206E65696768626F72206361636865AA
:101750000A00737563636573733A20726573657409
:10176000206E65696768626F722063616368650AED
:101770000075736167653A202573205B6C6973742B
:101780005D0A2020206F723A202573206164642056
:101790005B3C6966616365207069643E5D203C69FD
:1017A0007076365F616464723E203C6C325F6164C7
:1017B00064723E0A2020202020202A203C69666195
:1017C0006365207069643E206973206F7074696F6F
:1017D0006E616C206966206F6E6C79206F6E65207B
:1017E000696E746572666163652065786973747388
:1017F0002E0A2020206F723A2025732064656C2009
:101800003C697076365F616464723E0A2020206F06
:10181000723A2025732072657365740A00757361CE
:1018200067653A202573205B3C69666163652070BB
:1018300069643E5D0A0069662020526F75746572A6
:101840002020202020202020202020202020202098
:101850002020202020202020202073746174652007
:1018600020202020207479706500253268692020AE
:10187000252D3330732020002573205B3C636F756A
:101880006E743E5D203C6970763620616464723E01
:101890005B25253C696E746572666163653E5D20FB
:1018A0005B3C7061796C6F61645F6C656E3E5D205E
:1018B0005B3C64656C617920696E206D733E5D20D0
:1018C0005B3C737461747320696E74657276616CCD
:1018D0003E5D0A0064656661756C74733A00202091
:1018E0002020636F756E74203D203300202020205F
:1018F000696E74657266616365203D206669727306
:101900007420696E74657266616365206966206F14
:101910006E6C79206F6E652070726573656E742CC5
:10192000206F6E6C79206E656564656420666F72E9
:10193000206C696E6B2D6C6F63616C2061646472E6
:10194000657373657300202020207061796C6F616E
:10195000645F6C656E203D2034002020202064658B
:101960006C6179203D203130303000202020207300
:101970007461747320696E74657276616C203D20A9
:10198000636F756E74006572726F723A204950769B
:101990003620686561646572206F722049434D503E
:1019A000763620686561646572206E6F7420666F9C
:1019B000756E6420696E207265706C7900257520E3
:1019C00062797465732066726F6D2025733A2069A1
:1019D000643D256875207365713D25687520686FC5
:1019E00070206C696D69743D25752074696D652082
:1019F0003D20256C752E2530336C75206D730A00E3
:101A00006572726F723A20756E6578706563746581
:101A10006420706172616D657465727300657272C5
:101A20006F723A206D616C666F726D6564206164DF
:101A30006472657373006572726F723A206C696EBE
:101A40006B206C6F63616C20746172676574206ECB
:101A50006565647320696E74657266616365207084
:101A60006172616D65746572202875736520223C12
:101A7000616464726573733E253C69666E756D3E84
:101A800022290A006572726F723A206E6574776F50
:101A9000726B20726567697374727920697320664E
:101AA000756C6C006572726F723A20756E61626C53
:101AB0006520746F2073656E642049434D507636FF
:101AC000206563686F20726571756573740A0070B4
:101AD000696E672074696D656F75740064726F70EC
:101AE00070696E67206164646974696F6E616C20EF
:101AF000726573706F6E7365207061636B657420BF
:101B00002870726F6261626C7920636175736564BD
:101B1000206279206475706C696361746573290A49
:101B2000002D2D2D2025732070696E672073746140
:101B300074697374696373202D2D2D0A0025642048
:101B40007061636B657473207472616E736D697418
:101B50007465642C2025642072656365697665640C
:101B60002C2025642525207061636B6574206C6FC3
:101B700073732C2074696D6520256C752E303625A5
:101B80006C7520730A00727474206D696E2F617613
:101B9000672F6D6178203D20256C752E2530336CC4
:101BA000752F256C752E2530336C752F256C752E91
:101BB0002530336C75206D730A00256420706163D5
:101BC0006B657473207472616E736D69747465648F
:101BD0002C20302072656365697665642C20313075
:101BE000302525207061636B6574206C6F73730AF8
:101BF000006572726F723A20256869206973206EE1
